:100000000C947C2E0C9481310C94AC310C94D7312F
:100010000C9402320C942D320C9458320C9483328E
:100020000C94AE320C94AD2E0C94AD2E0C94AD2EDF
:100030000C94AD2E0C94AD2E0C94AD2E0C94AD2ED4
:100040000C94AD2E0C9486C70C94AD2E0C94AD2E52
:100050000C94AD2E0C94AD2E0C94EAB90C94AF2EEA
:100060000C94AD2E0C9480A50C942CA60C94AD2E63
:100070000C94AD2E0C94AD2E0C94AD2E0C94AD2E94
:100080000C94AD2E0C94AD2E0C94AD2E0C94AD2E84
:100090000C94AD2E0C94AD2E0C94AD2E0C94AD2E74
:1000A0000C94AD2E0C94AD2E0C94AD2E0C94AD2E64
:1000B0000C94AD2E0C94AD2E0C94AD2E0C94AD2E54
:1000C0000C94AD2E0C94AD2E0C94AD2E0C94AD2E44
:1000D0000C94AD2E0C94AD2E0C94AD2E0C94AD2E34
:1000E0000C94AD2EF72FFC2F01300B3015308E30D5
:1000F0001F3027302F30393043304D305C30663080
:100100008E3070307A308430B230B530A430A830C0
:10011000AE30EC30B930BD30C330C730CB30D13029
:10012000D530D930EC30DF30E330E7308A656A65AE
:1001300070656D6573657665796585657C659765C0
:100140007F658265C6A2C4A2E8A2E5A2E3A21AA3C3
:1001500017A315A373A341A33EA33CA3B3A5B9A5BD
:10016000CAA5D5A5DDA5F2A5E1A5F2A5E5A5E9A558
:10017000F2A5EFA5084AD73B3BCE016E84BCBFFD7C
:10018000C12F3D6C74319ABD56833DDA3D00C77F67
:1001900011BED9E4BB4C3E916BAAAABE0000008000
:1001A0003F05A84CCDB2D44EB93836A9020C50B98F
:1001B000918688083CA6AAAA2ABE000000803F00BB
:1001C0000D94F9370D94D54B0D940D470D94700493
:1001D0004E414E494E495459494E46CDCCCC3D0A2C
:1001E000D7233C17B7D13877CC2B329595E6241F0F
:1001F000B14F0A000020410000C84200401C4620C8
:10020000BCBE4CCA1B0E5AAEC59D7400407A10F39A
:100210005A00A0724E18090010A5D4E80000E87634
:1002200048170000E40B54020000CA9A3B0000008B
:10023000E1F505000080969800000040420F0000A4
:1002400000A08601000000102700000000E8030065
:100250000000006400000000000A0000000000012F
:1002600000000000002C76D888DC674F0823DFC12F
:10027000DFAE59E1B1B796E5E3E453C63AE65199EA
:100280007696E8E6C28426EB898C9B62ED407C6F13
:10029000FCEFBC9C9F40F2BAA56FA5F490055A2ACA
:1002A000F75C936B6CF9676DC11BFCE0E40D47FED6
:1002B000F520E6B500D0ED902E03009435770500CB
:1002C00080841E080000204E0A000000C80C333352
:1002D00033330F986E12831141EF8D2114893BE661
:1002E0005516CFFEE6DB18D1844B381BF77C1D90EA
:1002F0001DA4BBE424203284725E228100C9F12453
:10030000ECA1E53D2700000A0B02090C0D0E0807C1
:1003100003040100000000000000000000000000D5
:1003200000000000000000000000000000000000CD
:10033000001211100000000000000000000000008A
:10034000000000000000000000000001021020205A
:100350000808102040102040800201020108040219
:10036000010102040810204080804020100804028F
:1003700001800402018040201008040201080402E8
:1003800001010204081020408001020408102040EE
:100390008005050505070508080808020202020A8B
:1003A0000A08080404040401010101010101010318
:1003B00003030303030303040707070C0C0C0C0CD3
:1003C0000C0C0C0202020206060606060606060BC6
:1003D0000B0B0B0B0B0B0B0000200023002600293E
:1003E000002C002F0032000001000003010601096B
:1003F0000100002200250028002B002E00310034CF
:100400000002010000050108010B01000021002489
:100410000027002A002D00300033000101000004F5
:100420000107010A0101060D00FE09016602D6203E
:10043000FFFE0BFE0AFE0D0060221969808080809D
:100440008080800080183363A0A0A00357675050BD
:10045000F850F850500259692078A0A0702828F070
:100460002002596948A85010204050A890025868AE
:1004700040A0A040A0989068281363808080113B22
:100480006B2040408080808080404020113B6B800A
:100490004040202020202040408006556520A87044
:1004A000A8200455652020F8202011336360408087
:1004B000065161F811336340E040025969080810A1
:1004C00010204040808002596920508888888888A0
:1004D00050200259692060A02020202020F80259D5
:1004E000697088880810204080F8025969F808105F
:1004F000207008088870025969101030505090F828
:100500001010025969F88080B0C808088870025934
:100510006970888080F088888870025969F80810AE
:10052000102020404040025969708888887088886F
:10053000887002596970888888780808887011382E
:100540006840E040000040E04011386840E0400072
:100550000060408002596908102040804020100847
:10056000045464F80000F802596980402010081013
:1005700020408002596970888808102020002002DD
:10058000596970888898A8A8B08078025969205065
:10059000888888F8888888025969F04848487048EF
:1005A0004848F00259697088808080808088700295
:1005B0005969F048484848484848F0025969F88065
:1005C0008080F0808080F8025969F8808080F08017
:1005D0008080800259697088808080988888700245
:1005E000596988888888F888888888123969E0403D
:1005F000404040404040E00259693810101010104F
:10060000109060025969888890A0C0A090888802E4
:1006100059698080808080808080F802596988884C
:10062000D8A8A88888888802596988C8C8A8A898BE
:1006300098888802596970888888888888887002B4
:100640005969F0888888F080808080015A6A7088B3
:100650008888888888A87008025969F0888888F096
:10066000A090888802596970888080700808887016
:10067000025969F820202020202020200259698872
:10068000888888888888887002596988888888500E
:100690005050202002596988888888A8A8A8A850A6
:1006A00002596988885050205050888802596988BA
:1006B0008850502020202020025969F8081010206E
:1006C000404080F8113B6BE080808080808080809B
:1006D00080E0025969808040402010100808113BDA
:1006E0006BE0202020202020202020E008536320E1
:1006F0005088015161F82A226280400256667008D3
:1007000078889868025969808080F088888888F0A5
:1007100002566670888080887002596908080878D7
:1007200088888888780256667088F88088700259B0
:100730006930484040F04040404000586870888828
:100740008878088870025969808080B0C888888855
:10075000881238684000C040404040E0004A6A10BB
:1007600000301010101090906002596980808090C5
:10077000A0C0A09088123969C0404040404040402D
:10078000E0025666D0A8A8A8A888025666B0C88815
:10079000888888025666708888888870005868F053
:1007A000888888F0808080005868788888887808F1
:1007B0000808025666B0C88080808002566670883D
:1007C000601088700258684040F040404048300255
:1007D0005666888888889868025666888888505047
:1007E000200256668888A8A8A8500256668850201D
:1007F0002050880058688888889868088870025651
:1008000066F810204080F8015B6B1820202020C083
:10081000202020201822196980808080808080809C
:1008200080015B6BC0202020201820202020C008E1
:10083000536348A890FFFFFFFFFFFFFFFFFFFFFF8D
:10084000FFFFFFFFFFFFFFFFFFFFFFFFFFFFFFFFB8
:10085000FFFFFFFFFFFF0D0060221969800080800D
:1008600080808080800358682070A8A0A0A8702095
:1008700002596930484040E0404048B0035666881D
:10088000705050708802596988885050F820F820BC
:1008900020221969808080800080808080124A6ACE
:1008A000609080609090601090601A3262A0A00307
:1008B00059697088A8D8C8D8A88870045767700884
:1008C00078887800F80356662850A0A05028045372
:1008D00063F80808163161E00359697088E8D8D8D0
:1008E000E8D888700A5161F81744646090906003FA
:1008F00057672020F8202000F807356540A02040E9
:10090000E007356540A04020C02A226240800058A0
:10091000688888888898E8808002596978E8E8E8DB
:10092000E868282828262161C020226240800735F7
:100930006540C04040E0045767708888887000F8C0
:10094000035666A050282850A0025A6A40C0404072
:10095000E00818283808025A6A40C04040E01028D1
:10096000081038025A6A40A04020A04818283808C9
:10097000025969200020204080888870025A6A400D
:10098000200020508888F88888025A6A10200020A9
:10099000508888F88888025A6A3048002050888831
:1009A000F88888025A6A28500020508888F8888879
:1009B000025A6A50500020508888F88888025A6A83
:1009C00020502020508888F8888802596958A0A0B3
:1009D000A0B0E0A0A0B8005B6B70888080808080B1
:1009E00088702040025A6A402000F88080F08080A1
:1009F000F8025A6A102000F88080F08080F8025ACD
:100A00006A304800F88080F08080F8025A6A5050BE
:100A100000F88080F08080F8123A6A804000E04060
:100A200040404040E0123A6A204000E040404040F0
:100A300040E0124A6A609000E04040404040E012CE
:100A40003A6AA0A000E04040404040E0025969F00E
:100A5000484848E8484848F0025A6A2850008888C0
:100A6000C8A8988888025A6A4020007088888888B8
:100A70008870025A6A1020007088888888887002FE
:100A80005A6A30480070888888888870025A6A28B4
:100A9000500070888888888870025A6A50500070A8
:100AA0008888888888700355658850205088015B45
:100AB0006B08709898A8A8A8C8C87080025A6A40A5
:100AC000200088888888888870025A6A10200088E8
:100AD000888888888870025A6A30480088888888A0
:100AE000888870025A6A5050008888888888887080
:100AF000025A6A102000888850202020200259695C
:100B000080F0888888F0808080025969609090A089
:100B1000A0908888B00259694020007008788898B1
:100B2000680259691020007008788898680259692D
:100B30003048007008788898680259692850007019
:100B40000878889868025969505000700878889829
:100B500068025A6A304830007008788898680256EF
:100B600066702870A0A850005868708880808870CF
:100B700020400259694020007088F880887002592E
:100B8000691020007088F880887002596930480028
:100B90007088F88088700259695050007088F88019
:100BA0008870123969804000C040404040E01239EE
:100BB00069204000C040404040E012496960900018
:100BC000C040404040E0123969A0A000C040404011
:100BD00040E0025A6A50206010708888888870024D
:100BE0005969285000B0C88888888802596940200F
:100BF0000070888888887002596910200070888881
:100C00008888700259693048007088888888700226
:100C10005969285000708888888870025969505036
:100C200000708888888870035767202000F80020AB
:100C300020015868087098A8A8C8708002596940B7
:100C40002000888888889868025969102000888860
:100C50008888986802596930480088888888986828
:100C6000025969505000888888889868005B6B102A
:100C700020008888889868088870005A6A8080B048
:100C8000C88888C8B08080005B6B50500088888816
:100C9000986808887001050700FE0500FB01F22036
:100CA000FFFE05FE05FE0200400215258080800043
:100CB00080053242A0A002556550F850F850014618
:100CC000562070C030E02002556590102040480248
:100CD0005565608068906805122280800225354045
:100CE000808080400225358040404080043343A00E
:100CF00040A003334340E0400122324080043141B0
:100D0000E0021121800255650810204080024555FF
:100D10006090909060022535C040404040024555AB
:100D2000E0106080F0024555E0106010E00245558B
:100D30002060A0F020024555F080E010E00245550B
:100D40006080E09060024555F0102040400245551B
:100D500060906090600245556090701060031323AE
:100D6000800080021424800080800235452040806D
:100D70004020033343E000E00235458040204080BE
:100D8000024555E0106000400255657088B8A870B3
:100D9000024555609090F090024555E090E090E05B
:100DA0000235456080808060024555E0909090E07B
:100DB000023545E080E080E0023545E080E080805B
:100DC0000245557080B090700245559090F090901B
:100DD000023545E0404040E002455530101090603B
:100DE00002455590A0C0A09002354580808080E0EB
:100DF00002556588D8A8888802455590D0B0909053
:100E00000245556090909060024555E09090E080DA
:100E1000014656609090906010024555E09090E039
:100E20009002455570806010E0023545E04040403A
:100E30004002455590909090600245559090A0A03A
:100E40004002556588A8A8A850024555909060902A
:100E5000900245559090701060023545E02040802A
:100E6000E0022535C0808080C0025565804020109A
:100E700008022535C0404040C005324240A0024132
:100E800051F0052232804002445470909070024527
:100E90005580E09090E002344460808060024555C7
:100EA000107090907002445460B0C06002354520CC
:100EB00040E04040004656709090701060024555EA
:100EC00080E0909090021525800080808000273778
:100ED000400040404040800245558090A0E0900294
:100EE00015258080808080025464F0A8A8A8024460
:100EF00054E090909002445460909060004656E018
:100F00009090E080800046567090907010100234EF
:100F100044A0C0808002445470C030E00235454097
:100F2000E0404020024454909090700244549090CD
:100F3000A040025464A8A85050023444A04040A0ED
:100F4000004656909090701060024454F02040F09B
:100F50000235456040804060021525808080808099
:100F6000023545C0402040C005425250A0FFFFFF5F
:100F7000FFFFFFFFFFFFFFFFFFFFFFFFFFFFFFFF81
:100F8000FFFFFFFFFFFFFFFFFFFFFFFFFFFF02006D
:100F900040FFFFFFFFFFFFFFFFFFFFFFFFFFFFFF20
:100FA000FFFFFFFFFFFFFFFFFFFFFFFFFFFFFFFF51
:100FB000FFFFFFFFFFFFFFFFFFFFFFFFFFFFFFFF41
:100FC000FFFFFFFFFFFFFFFFFFFFFFFFFFFFFFFF31
:100FD000FFFFFFFFFFFFFFFFFFFFFFFFFFFFFFFF21
:100FE000FFFFFFFFFFFFFFFFFFFFFFFFFFFFFFFF11
:100FF00001050800FF060121023520FFFF07FF065B
:10100000FF090050221656808080800080153353DF
:10101000A0A0A00257575050F850F8505002575710
:101020002070A07028702013355580A040A02002A9
:10103000475740A0A040A0A05025135380808012A5
:101040002656408080808040122656804040404096
:10105000800245559060F060900255552020F820A0
:1010600020113353604080044151F011335340E06C
:101070004002465610102040808012365640A0A0F4
:10108000A0A04012365640C0404040E002465660A4
:1010900090106080F0024656F0206010906002468A
:1010A000562060A0F02020024656F080E0109060AC
:1010B0000246566080E0909060024656F010202074
:1010C00040400246566090609090600246566090A4
:1010D00090701060122555C0C000C0C01136566017
:1010E00060006040801236562040808040200343DC
:1010F00053F000F0123656804020204080123656C1
:1011000040A020400040015858304898A8A890407E
:1011100030024656609090F09090024656E090E083
:101120009090E0024656609080809060024656E0C3
:1011300090909090E0024656F080E08080F0024669
:1011400056F080E0808080024656609080B09060CB
:101150000246569090F0909090123656E0404040F3
:1011600040E002465670202020A04002465690A043
:10117000C0A0A0900246568080808080F002465633
:1011800090F0F090909002465690D0F0B0B090025F
:101190004656609090909060024656E09090E080B5
:1011A00080014757609090D0B06010024656E090A2
:1011B00090E0909002465660904020906012365623
:1011C000E04040404040024656909090909060022F
:1011D0004656909090906060024656909090F0F045
:1011E00090024656909060609090025656888850C3
:1011F000202020024656F010204080F0123656E0A3
:1012000080808080E0024656808040201010123698
:1012100056E020202020E016325240A0014151F03B
:1012200016225280400244547090907002465680BC
:1012300080E09090E0123454608080600246561046
:10124000107090907002445460B0C0600246562006
:101250005040E04040014555609070106002465695
:101260008080E09090901236564000C04040E011DF
:1012700037572000202020A040024656808090E072
:101280009090123656C040404040E0025454D0A8DE
:10129000A8A8024454E0909090024454609090605A
:1012A000014555E090E08080014555709070101028
:1012B000024454A0D0808012345460C020C0024642
:1012C000564040E0405020024454909090701234B8
:1012D00054A0A0A04002545488A8A850024454909E
:1012E0006060900145559090709060024454F020E9
:1012F00040F0024757304020C02040302216568030
:101300008080808080024757C02040304020C00647
:10131000425250A0FFFFFFFFFFFFFFFFFFFFFFFF55
:10132000FFFFFFFFFFFFFFFFFFFFFFFFFFFFFFFFCD
:10133000FFFFFFFFFF0900502216568000808080CB
:10134000800146562070A0A070200246562050E032
:101350004050A002555588705070880256568850EB
:10136000F820F82022175780808000808080024774
:10137000577080E0907010E0173151A002565670FF
:10138000A8C8C8A87014355560A06000E003435396
:1013900050A050123353E02020143151E002565631
:1013A00070E8D8E8D870173151E015335340A040A9
:1013B00012355540E04000E014355540A02040E093
:1013C000143555C020C020C016225240800145551A
:1013D000909090E08002565678E8E868282824111A
:1013E0005180112252408014355540C04040E014D5
:1013F000355540A04000E0034353A050A00247579A
:10140000808080A060F0200247578080A0D010200C
:101410007002475780408060A0F02012365640008E
:101420004080A04002475740206090F090900247D3
:101430005720406090F0909002475760906090F085
:10144000909002475750A06090F0909002475790BC
:10145000006090F0909002475760906090F09090FC
:1014600002465670A0A0F0A0B0014757609080805F
:101470009060400247574020F080E080F0024757DC
:101480002040F080E080F00247576090F080E080DC
:10149000F00247579000F080E080F012375780400C
:1014A000E0404040E01237572040E0404040E0122A
:1014B000375740A0E0404040E0123757A000E040DE
:1014C0004040E00256567048E8484870024757507E
:1014D000A090D0B0909002475740206090909060CC
:1014E000024757204060909090600247576090609C
:1014F0009090906002475750A06090909060024793
:101500005790006090909060123353A040A0024624
:101510005670B0B0D0D0E0024757402090909090E5
:10152000600247572040909090906002475760902B
:101530009090909060024757900090909090600239
:1015400057571020885020202002465680E0909067
:10155000E0800246566090A0A090A002475740202D
:101560000070909070024757204000709090700279
:1015700047572050007090907002475750A000705D
:1015800090907002465650007090907002475760DD
:10159000906070909070025454F068B07811355596
:1015A000608080604002475740200060B0C0600209
:1015B000475720400060B0C060024757609000600D
:1015C000B0C060024656500060B0C060123757800D
:1015D0004000C04040E0123757204000C04040E08B
:1015E00012375740A000C04040E0123656A000C05D
:1015F0004040E0024757A040A0107090600247575B
:1016000050A000E0909090024757402000609090DA
:1016100060024757204000609090600247576090FA
:10162000006090906002475750A000609090600268
:1016300046569000609090601235554000E00040A2
:1016400002445470B0D0E002475740200090909080
:10165000700247572040009090907002475760906A
:1016600000909090700246569000909090700148C3
:101670005820400090907090600147578080E09023
:10168000E08080014757900090907090602020206B
:101690002000202020202020200025753A253032EF
:1016A0007500253032753A25303275002575642075
:1016B000253032753A25303275003FFFF038007022
:1016C0003186302387102787902F87D02F03D02093
:1016D00030102078102078102030102F03D02F8762
:1016E000D02787902387103186303800703FFFF075
:1016F0003FFFF038007030FC3020FC1020781020C4
:1017000030102C00D02E31D02F7BD02F7BD02E311B
:10171000D02C00D020301020781020FC1030FC306D
:101720003800703FFFF00410400208200208200437
:101730001040082080104100104100082080041053
:10174000400000001FFFF81FFFF81FFFF81FFFF801
:101750001FE020102010201010201020201020103A
:1017600030300840048003001FE03FF03FF03FF0BE
:101770001FE01FE03FF03FF03FF00FC00780030085
:101780004572723A207574663820666F6E74206EEA
:101790006F7420696E697469616C697A65642E0082
:1017A0004572723A207574663820666F6E74206ECA
:1017B0006F7420696E697469616C697A65642E0062
:1017C0004572723A207574663820666F6E74206EAA
:1017D0006F7420696E697469616C697A65642E0042
:1017E000506C656173652052657365740050524991
:1017F0004E5445522048414C54454400687474701E
:101800003A2F2F6D61726C696E66772E6F7267006A
:10181000322E302E302E313638007F80FFC0FFC090
:10182000FFC07F807F80FFC0FFC0FFC03F001E0061
:101830000C00FFFFFF0E000E000E000E000E000E4B
:10184000000E000E007FC03F801F000E0004000449
:10185000000E001F003F807FC00E000E000E000E25
:10186000000E000E000E000E0000FE0003FF8007B9
:1018700083C00E01C00E00E01C00E07F00E03E00CF
:10188000E01C00E00800E00000E00001C00E01C024
:101890000F078007FF0001FC0001FC0007FF000F9D
:1018A00007800E01C00001C00000E00800E01C003D
:1018B000E03E00E07F00E01C00E00E00E00E01C012
:1018C0000783C003FF8000FE00000C0D00FE07022E
:1018D0002603BC017FFE08FE08FE0508080600007E
:1018E00040F0C88888987810050808060000C0F8FD
:1018F0008888888888F80505050600012030F830BA
:10190000200508080600002070F820202020E005AF
:1019100009090600FF2070A8A8B88888702005066D
:1019200006060001E08CEA8C8A0A0509090600FF18
:10193000F8A88888888888A8F8050A0A0600FE2082
:101940005050505088A8A888700303030600034035
:10195000A040FFFFFFFFFFFFFFFFFFFFFFFFFFFFB5
:10196000FFFFFFFFFFFFFFFF0000000605FF01076D
:101970000706020080808080800080030303060148
:1019800005A0A0A005060606000050F85050F8502B
:101990000509090600FF2070A8A07028A87020057E
:1019A0000707060000C8C8102040989805070706DA
:1019B000000040A0A040A890680103030602058033
:1019C00080800309090601FF20404080808040405C
:1019D000200309090601FF8040402020204040806C
:1019E00005070706000020A8702070A8200505053F
:1019F0000600012020F820200203030601FFC0405A
:101A000080050101060003F8020202060100C0C0C1
:101A10000507070600000810102040408005070752
:101A2000060000708898A8C88870030707060100A0
:101A300040C040404040E0050707060000708808AD
:101A4000102040F8050707060000F8081030088845
:101A50007005070706000010305090F810100507B9
:101A600007060000F880F0080888700507070600E0
:101A700000304080F0888870050707060000F808ED
:101A80001010202020050707060000708888708845
:101A900088700507070600007088887808106002C3
:101AA0000505060100C0C000C0C00206060601FF11
:101AB000C0C000C0408003050506010120408040F1
:101AC00020050303060002F800F8030505060101DE
:101AD0008040204080050707060000708810202005
:101AE00000200507070600007088B8A8B8807005B8
:101AF0000707060000708888F888888805070706A9
:101B00000000F04848704848F005070706000070DC
:101B1000888080808870050707060000F0484848E4
:101B20004848F0050707060000F88080F08080F83C
:101B3000050707060000F88080F080808005070711
:101B400006000070888080988870050707060000EE
:101B5000888888F8888888030707060100E04040E5
:101B6000404040E0050707060000381010101090B4
:101B7000600507070600008890A0C0A090880507B0
:101B800007060000808080808080F8050707060037
:101B90000088D8A8888888880507070600008888F4
:101BA000C8A8988888050707060000708888888874
:101BB0008870050707060000F08888F0808080059F
:101BC000070706000070888888A890680507070640
:101BD0000000F08888F0A0908805070706000070D4
:101BE000888070088870050707060000F82020200C
:101BF00020202005070706000088888888888870CC
:101C000005070706000088888888505020050707C8
:101C100006000088888888A8A850050707060000E5
:101C2000888850205088880507070600008888505B
:101C300020202020050707060000F808102040801B
:101C4000F80309090601FFE080808080808080E041
:101C5000050707060000804040201010080309090E
:101C60000601FFE020202020202020E005030306BD
:101C700000052050880501010600FEF80303030655
:101C80000105804020050505060000700878887869
:101C90000507070600008080F0888888F0050505A4
:101CA000060000708080887005070706000008089D
:101CB00078888888780505050600007088F08070AF
:101CC000050707060000304840E040404005070790
:101CD0000600FE70888888780870050707060000EF
:101CE0008080F0888888880307070601004000C0CC
:101CF000404040E00409090601FE100030101010B9
:101D000010906005070706000080808890E09088AA
:101D1000030707060100C04040404040E0050505BC
:101D2000060000D0A8A8A8A8050505060000B0C8B0
:101D30008888880505050600007088888870050772
:101D4000070600FEF0888888F080800507070600F7
:101D5000FE78888888780808050505060000B0C860
:101D600080808005050506000078807008F0050772
:101D7000070600002020F820202018050505060091
:101D800000888888986805050506000088888850BE
:101D9000200505050600008888A8A8500505050649
:101DA000000088502050880507070600FE888888B4
:101DB00050204080050505060000F8102040F8037B
:101DC00009090601FF2040404080404040200109B1
:101DD000090602FF8080808080808080800309095E
:101DE0000601FF804040402040404080050303063C
:101DF000000248A890FF1FFFFFFFFFFFFF600000E9
:101E0000000001FF400000000000FF800000000013
:101E1000007F83CF00000C303F87FF80000C301F15
:101E2000867980000C000F8C30C7838C30E78C30B3
:101E3000CFC7CC31F38C30DCECEC33B98C30D86CC0
:101E40006C33198C30D06C0C33198C30D86C0C334B
:101E5000198C30DC6C0E3B198C30CF7C079F198CB1
:101E600030C77C038F1940000000000002600000B2
:101E7000000000061FFFFFFFFFFFF800060900FE3D
:101E800006018902FE20FFFE07FE06FE0000000696
:101E900000070106060602008080808000800303A0
:101EA00003060103A0A0A00507070600FF5050F895
:101EB00050F850500509090600FE2070A8A07028AF
:101EC000A870200608080600FF40A84810204854C3
:101ED000080507070600FF6090906098906801036E
:101EE000030602038080800207070602FF4080800D
:101EF000808080400207070602FF8040404040404B
:101F0000800505050600008850F85088050505067F
:101F100000002020F820200204040602FEC04040F9
:101F200080050101060002F8020202060200C0C09C
:101F300004060606010010102040808004060606F4
:101F4000010060909090906003060606010040C07A
:101F5000404040E00406060601006090102040F07A
:101F6000040606060100F020601010E005060606D3
:101F7000000010305090F810040606060100F080B2
:101F8000E01010E00406060601006080E09090601A
:101F9000040606060100F010102040400406060664
:101FA0000100609060909060040606060100609059
:101FB00090701060020505060200C0C000C0C0029B
:101FC00007070602FEC0C000C040408005050506A8
:101FD00000001860806018050303060001F800F88F
:101FE000050505060000C0300830C00407070601DB
:101FF00000609010604000400506060600007090EA
:10200000A8B08070050606060000205088F8888871
:10201000050606060000F088F08888F0040606062B
:102020000100609080809060040606060100E09048
:10203000909090E0040606060100F080E08080F0B9
:10204000040606060100F080E08080800406060693
:102050000100609080B09060040606060100909038
:10206000F0909090030606060100E040404040E0FA
:1020700005060606000038101010906004060606DB
:10208000010090A0C0A09090040606060100808088
:10209000808080F005060606000088D8A8A88888F9
:1020A00004060606010090D0B09090900506060642
:1020B0000000708888888870040606060100E09099
:1020C00090E080800407070601FF609090D0B06028
:1020D00010040606060100E09090E09090040606C9
:1020E000060100609040209060050606060000F89A
:1020F0002020202020040606060100909090909059
:1021000060040606060100909090F06060050606E7
:102110000600008888A8A8D888050606060000885A
:102120005020205088050606060000888850202090
:1021300020040606060100F010204080F003060689
:10214000060100E080808080E00406060601008031
:102150008040201010030606060100E02020202009
:10216000E00503030600032050880501010600FE78
:10217000F802020206020480400404040601007012
:102180009090700406060601008080E09090E004C4
:102190000404060100708080700406060601001029
:1021A000107090907004040406010060B0C07004C8
:1021B0000606060100205040E040400406060601E5
:1021C000FE6090907010600406060601008080E0BA
:1021D0009090900306060601004000C04040E003D6
:1021E00008080601FE200060202020A0400406060A
:1021F0000601008080A0C0A090030606060100C072
:1022000040404040E0050404060000D0A8A888042F
:102210000404060100E090909004040406010060AC
:102220009090600406060601FEE09090E080800435
:1022300006060601FE70909070101004040406015A
:1022400000A0D0808004040406010070C030E004C7
:1022500006060601004040E0405020040404060148
:102260000090909070040404060100909060600556
:10227000040406000088A8A8500404040601009085
:102280006060900406060601FE90909070906004D5
:102290000404060100F02040F003070706010020B7
:1022A0004040804040200107070602FF8080808078
:1022B0008080800307070601008040402040408066
:1022C00004020206010350A0FFFFFFFFFFFFFFFF14
:1022D000FFFFFFFFFFFFFFFFFFFFFFFFFFFFFFFF0E
:1022E000FFFFFFFFFFFFFFFFFF00000006000701E9
:1022F0000606060200800080808080040606060133
:10230000FF2070A0A070200507070600FF3048409E
:10231000F04040F8050505060000A8508850A805C3
:1023200006060600008850F820F82001070706027C
:10233000FF808080008080800407070601FF708096
:1023400060906010E0030101060105A00607070682
:102350000000788494A49484780305050601016044
:10236000A06000E00505050600002850A0502804E4
:102370000303060100F01010040101060102F0063B
:1023800007070600007884B4A4A484780401010639
:102390000105F004030306010260906005070706CB
:1023A00000FF2020F8202000F80305050601014069
:1023B000A02040E0030505060101C0204020C00226
:1023C000020206020440800405050601FF9090B059
:1023D000D08005060606000078E8E8682828010194
:1023E00001060202800202020602FE408003050589
:1023F00006010140C04040E003050506010140A080
:102400004000E0050505060000A0502850A0050882
:10241000080600FF40C040507030781005080806DC
:1024200000FF40C04050680810380508080600FF4B
:10243000C0204030F030781004070706010020006B
:102440002060809060050707060000402020507043
:10245000888805070706000010202050708888052E
:1024600007070600002050205070888805070706DF
:10247000000028502050708888050707060000508B
:102480000020507088880507070600002050205063
:1024900070888805060606000078A0F0A0A0B804A1
:1024A00008080601FE6090808090602040040707C5
:1024B0000601004020F080E080F0040707060100DC
:1024C0002040F080E080F00407070601002050F073
:1024D00080E080F00407070601005000F080E080F3
:1024E000F00307070601008040E0404040E003079A
:1024F000070601002040E0404040E00307070601D6
:102500000040A0E0404040E0030707060100A000B3
:10251000E0404040E00506060600007048E84848F4
:102520007004070706010050A090D0B090900407F7
:1025300007060100402060909090600407070601A4
:102540000020406090909060040707060100205032
:10255000609090906004070706010050A060909082
:10256000906004070706010050006090909060059D
:10257000050506000088502050880408080601FF61
:102580001070B0B0D0D0E0800407070601004020F2
:102590009090909060040707060100204090909072
:1025A000906004070706010020509090909060040E
:1025B00007070601005000909090906005070706FD
:1025C000000010208850202020040606060100800C
:1025D000E09090E0800406060601006090A0A090C4
:1025E000A0040707060100402000709090700407C7
:1025F0000706010020400070909070040707060154
:10260000002050007090907004070706010050A051
:1026100000709090700406060601005000709090C3
:102620007004070706010020502070909070050488
:102630000406000070A8B0780406060601FE70804B
:102640008070204004070706010040200060B0C0F1
:102650007004070706010020400060B0C070040746
:102660000706010020500060B0C070040606060195
:1026700000500060B0C070030707060100804000F2
:10268000C04040E0030707060100204000C0404072
:10269000E003070706010040A000C04040E0030639
:1026A00006060100A000C04040E004070706010044
:1026B0003060107090906004070706010050A00081
:1026C000E090909004070706010040200060909081
:1026D0006004070706010020400060909060040736
:1026E0000706010020500060909060040707060173
:1026F0000050A000609090600406060601005000A3
:10270000609090600505050600002000F800200498
:10271000040406010070B0D0E00407070601004081
:102720002000909090700407070601002040009060
:102730009090700407070601002050009090907060
:1027400004060606010050009090907004090906E6
:1027500001FE2040009090907090600408080601EF
:10276000FE8080E09090E080800408080601FE5022
:1027700000909090709060536E346B3300496E7689
:10278000616465727300427269636B6F7574004DAA
:1027900061696E00536D6F6F7468696E6700536D89
:1027A0006F6F7468696E67005A005A0059005900CB
:1027B00058005800436F7272656374696F6E00430E
:1027C0006F7272656374696F6E004D61696E004669
:1027D000696C616D656E740054656D7065726174CD
:1027E000757265004261636B6C6173680053746558
:1027F00070732F6D6D004A65726B00416363656C89
:1028000065726174696F6E0056656C6F6369747987
:1028100000436F6E66696775726174696F6E00451B
:1028200073746570732F6D6D004573746570732FCD
:102830006D6D005A73746570732F6D6D005A7374EB
:102840006570732F6D6D005973746570732F6D6DA6
:10285000005973746570732F6D6D005873746570D3
:10286000732F6D6D005873746570732F6D6D00411B
:102870006476616E6365642053657474696E677312
:102880000056652D4A65726B0056652D4A65726B60
:1028900000567A2D4A65726B00567A2D4A65726B26
:1028A0000056792D4A65726B0056792D4A65726B18
:1028B0000056782D4A65726B0056782D4A65726B0A
:1028C00000416476616E6365642053657474696E5B
:1028D000677300416D6178204500416D6178204546
:1028E00000416D6178205A00416D6178205A0041A5
:1028F0006D6178205900416D6178205900416D610A
:1029000078205800416D6178205800412D54726143
:1029100076656C00412D54726176656C00412D52D4
:1029200065747261637400412D52657472616374E1
:1029300000416363656C00416363656C00416476CC
:10294000616E6365642053657474696E67730056C5
:1029500054726176204D696E005654726176204D36
:10296000696E00566D696E00566D696E00566D6138
:1029700078204500566D6178204500566D617820BD
:102980005A00566D6178205A00566D6178205900C2
:10299000566D6178205900566D6178205800566D4B
:1029A0006178205800416476616E636564205365E8
:1029B0007474696E67730020082046616374002098
:1029C000082046616374002008204D6178002008CB
:1029D000204D6178002008204D696E002008204DB0
:1029E000696E004175746F74656D70004F666600A6
:1029F0004F6E004175746F74656D7000416476614F
:102A00006E6365642053657474696E6773004C6F00
:102A10006164206D6D004C6F6164206D6D00556EBA
:102A20006C6F6164206D6D00556E6C6F6164206D1C
:102A30006D00416476616E6365204B004164766190
:102A40006E6365204B00416476616E63656420535C
:102A5000657474696E67730044697361626C6520A4
:102A60005374657070657273004D3834004175742D
:102A70006F20486F6D6500473238004D6F766520D6
:102A800041786973004D61696E00457874727564B0
:102A9000657220004175746F20486F6D6500473284
:102AA00038004D6F7665205A004D6F7665205900CD
:102AB0004D6F76652058004D6F74696F6E004578D4
:102AC00074727564657220004D6F76652025736D94
:102AD0006D00004D6F766520302E316D6D004D6FAD
:102AE000766520316D6D004D6F76652031306D6DEE
:102AF000004D6F7665204178697300486F74656E8C
:102B00006420746F6F20636F6C6400457874727515
:102B100064657220004D6F7665205A004D6F7665B2
:102B20002059004D6F76652058004D6F7665205A0C
:102B3000004D6F76652059004D6F76652058005026
:102B400072696E742066726F6D204D6564696100F4
:102B50005072696E742066726F6D204D6564696194
:102B600000022E2E004D61696E005072696E740075
:102B700043616E63656C00537461727420507269B6
:102B80006E7420003F005761697420666F720066A2
:102B9000696C616D656E74207075726765000050B8
:102BA0006C6561736520776169742E00507265737E
:102BB0007320427574746F6E00746F207265737544
:102BC0006D65207072696E74005761697420666F5C
:102BD000720066696C616D656E74206C6F61640073
:102BE000496E736572742066696C616D656E740000
:102BF000616E6420707265737320627574746F6E99
:102C000000746F20636F6E74696E75650050726535
:102C1000737320627574746F6E00746F20686561E1
:102C200074206E6F7A7A6C65004E6F7A7A6C6520CC
:102C300068656174696E6700506C656173652077C3
:102C40006169742E2E2E005761697420666F7200C0
:102C500066696C616D656E7420756E6C6F61640081
:102C60005761697420666F720066696C616D656E8C
:102C700074206368616E676500746F20737461729D
:102C800074005061726B696E672E2E2E004368616E
:102C90006E67696E672046696C616D656E7400557C
:102CA0004E4C4F41442046494C414D454E54004CFA
:102CB0004F41442046494C414D454E540020204E42
:102CC0006F7A7A6C653A20002000456E6420666950
:102CD0006C616D656E74206368616E676500507528
:102CE000726765206D6F726500004368616E67658D
:102CF0002046696C616D656E7400556E6C6F616421
:102D00002046696C616D656E74004C6F616420468D
:102D1000696C616D656E74004D3630302042302034
:102D2000542564004D373032203B2564004D373048
:102D30003220542564004D37303120542564005032
:102D400072656865617420437573746F6D005072AD
:102D5000656865617420437573746F6D00507265AA
:102D60006865617420414253005072656865617402
:102D700020504C41004261636B004E6F204D6564F2
:102D80006961005072696E742066726F6D204D65C6
:102D9000646961004368616E6765204D65646961BF
:102DA000004D32310041626F7574205072696E744B
:102DB0006572004368616E67652046696C616D6588
:102DC0006E74004368616E67652046696C616D656D
:102DD0006E74004D36303020423000436F6E6669AD
:102DE0006775726174696F6E0054656D70657261AC
:102DF00074757265004D6F74696F6E0052657375FE
:102E00006D65205072696E740054756E6500537460
:102E10006F70205072696E74005061757365205038
:102E200072696E7400496E666F2053637265656ED9
:102E30000053746F70004261636B0053746F7020B5
:102E40005072696E74003F0050726F6265205A20A4
:102E50004F666673657400426162797374657020B1
:102E600059004261627973746570205800466C6F36
:102E70007700466C6F770046616E2053706565641D
:102E800020310046616E2053706565642031004238
:102E9000656400426564004E6F7A7A6C65004E6F1F
:102EA0007A7A6C650053706565640053706565647B
:102EB000004D61696E0042616279737465702059DA
:102EC00000426162797374657020580047616D65D6
:102ED00073004669726D7761726520566572736919
:102EE0006F6E004D61696E00436F6F6C646F776E3B
:102EF0000046616E20537065656420310046616E46
:102F00002053706565642031004265640042656449
:102F1000004E6F7A7A6C65004E6F7A7A6C65004D60
:102F200061696E006F6F6F0000001FC07FF0DDD819
:102F3000FFF87FF0444024800000318000002480AE
:102F40004440107CFEFEFE04000E000E007FC0FF19
:102F5000E0FFE0FFE0FFE006000F001F8036C03F0B
:102F6000C009001680294006000F001F8036C03FB0
:102F7000C0168020401080104008801FC037607F3E
:102F8000F05FD050500D80104048905FD077707F38
:102F9000F01FC0104020200F007FE0FFF0E670FF20
:102FA000F0198036C0C0300F007FE0FFF0E670FF00
:102FB000F0198036C0198047414D45204F56455283
:102FC00000526573746F7265206661696C73616627
:102FD00065004C6F61642053657474696E6773009B
:102FE00053746F72652053657474696E6773005013
:102FF000726F6265205A204F666673657400416483
:1030000076616E6365642053657474696E677300DE
:103010004D61696E0050726F6265205A204F66667E
:10302000736574004D6F76696E672E2E2E004D32DB
:1030300034004D323520500A4D3234005072696EE2
:10304000742050617573656400506175736520501C
:1030500072696E74005072696E742041626F72748E
:103060006564004C756C7A426F742054415A203666
:103070002072656164792E005072696E74696E67A2
:103080002E2E2E005072696E742050617573656427
:10309000004D656469612052656D6F766564004D11
:1030A0006564696120496E736572746564004D31B1
:1030B0003137004D33310043616E6E6F7420656EA1
:1030C000746572207375626469723A20002E0A007A
:1030D0006F70656E206661696C65642C2046696C52
:1030E000653A20006175746F25632E670065727202
:1030F0006F722077726974696E6720746F206669D9
:103100006C650A004E6F74205344207072696E74AF
:10311000696E670A005344207072696E74696E6745
:10312000206279746520002E0A0044656C6574691C
:103130006F6E206661696C65642C2046696C653A27
:10314000200046696C652064656C657465643A00AE
:1031500057726974696E6720746F2066696C653A8E
:1031600020002E0A006F70656E206661696C6564D0
:103170002C2046696C653A20002E0A006F70656E3F
:10318000206661696C65642C2046696C653A200094
:1031900046696C652073656C65637465640A00201C
:1031A00053697A653A200046696C65206F70656ED8
:1031B00065643A20002066696C653A200066726595
:1031C000736800646F696E67004E6F772000454E2C
:1031D0004420535542524F5554494E450A0022202F
:1031E000706F73002220706172656E743A22005312
:1031F0005542524F5554494E452043414C4C207442
:1032000061726765743A2200747279696E6720741E
:103210006F2063616C6C207375622D67636F6465EA
:103220002066696C6573207769746820746F6F20FD
:103230006D616E79206C6576656C732E204D4158FA
:10324000206C6576656C2069733A310A004D323422
:10325000004D323320257300534420636172642093
:103260006F6B0A006F70656E526F6F7420666169D4
:103270006C65640A00766F6C756D652E696E697495
:10328000206661696C65640A00534420696E697444
:10329000206661696C0A00286E6F2066696C65297A
:1032A0000043616E6E6F74206F70656E207375627F
:1032B00064697220007C3C3E5E2B3D3F2F5B5D3B92
:1032C0002C2A225C000A003B20454550524F4D20DD
:1032D000496E6465783A20005570646174696E6760
:1032E000207A6F666673657420696E20454550527A
:1032F0004F4D3A20003474682070726F6265207000
:103300006F696E742C2064697374616E63652066E6
:10331000726F6D20706C616E653A200000000000D5
:10332000000000000000000000000000000000009D
:103330000000000000000000000000000000000C81
:10334000000000000000000C00000000000000125F
:103350000000000000000023000000000000002129
:10336000000000000000004C800000000000005E33
:10337000800000000000009240000000000000A15A
:103380004000000000000121200000000000027F3A
:10339000900000000000020010000000000007FF85
:1033A000F800000000000400080000000000080011
:1033B00004000000000008000600000000001000EB
:1033C000020000000000301E010000000000207F0D
:1033D00081000000000041FFE0800000000043FC8D
:1033E000F08000000000873B7840000000018EDB89
:1033F000FC60000000010FEBCC20000000021FED7C
:10340000B610000000021FDEB6100000000439CD27
:103410007F080000000436E0FF08000000087EC0BE
:10342000BB84000000187F005D86000000107FC094
:10343000ED82000000203CC07301000000203B33FF
:103440007F01000000701BE77E03800000C81DEEB6
:10345000DE04C00000880FDEDC04400001240FDF22
:103460003C092000012607DBF8192000027203E75F
:10347000F0139000025101FFE02290000489007FC8
:10348000802448000904801E004824000BFE4000F0
:1034900000DFF40010004000008002001FFFFFFF6B
:1034A000FFFFFE0000000000000000000000000020
:1034B0000000000000000000000000001022103C8E
:1034C0003C0E1F00102210042211040010221008CC
:1034D00022110400102210083C11040010221010C8
:1034E0002211040010221020221104001E1C1E3C78
:1034F0003C0E04000000000000000000000000007E
:1035000000000000000000000000000000000000BB
:1035100000000000000000000000000000000000AB
:10352000000000000000000000000000000000009B
:10353000000000000000000000000000000000008B
:10354000000000000000000000000000000000007B
:1035500000000000000000000000000C0D00FE074D
:10356000022603BC017FFE08FE08FE0508080600CF
:103570000040F0C88888987810050808060000C048
:10358000F88888888888F80505050600012030F845
:1035900030200508080600002070F820202020E0D8
:1035A0000509090600FF2070A8A8B88888702005C2
:1035B0000606060001E08CEA8C8A0A050909060065
:1035C000FFF8A88888888888A8F8050A0A0600FEF7
:1035D000205050505088A8A88870030303060003A9
:1035E00040A040FFFFFFFFFFFFFFFFFFFFFFFFFFC8
:1035F000FFFFFFFFFFFFFFFFFF0000000605FF01C9
:103600000707060200808080808000800303030695
:103610000105A0A0A005060606000050F85050F8CD
:10362000500509090600FF2070A8A07028A8702086
:10363000050707060000C8C810204098980507072E
:1036400006000040A0A040A8906801030306020500
:103650008080800309090601FF204040808080406F
:1036600040200309090601FF8040402020204040FF
:103670008005070706000020A8702070A820050517
:10368000050600012020F820200203030601FFC0E8
:103690004080050101060003F8020202060100C095
:1036A000C0050707060000081010204040800507ED
:1036B00007060000708898A8C888700307070601ED
:1036C0000040C040404040E0050707060000708809
:1036D00008102040F8050707060000F80810300819
:1036E000887005070706000010305090F81010058C
:1036F0000707060000F880F008088870050707062D
:103700000000304080F0888870050707060000F848
:103710000810102020200507070600007088887018
:103720008888700507070600007088887808106090
:10373000020505060100C0C000C0C0020606060161
:10374000FFC0C000C0408003050506010120408085
:103750004020050303060002F800F80305050601F2
:103760000180402040800507070600007088102077
:103770002000200507070600007088B8A8B88070F0
:10378000050707060000708888F8888888050707FD
:10379000060000F04848704848F00507070600009A
:1037A00070888080808870050707060000F0484810
:1037B000484848F0050707060000F88080F0808040
:1037C000F8050707060000F88080F0808080050774
:1037D000070600007088808098887005070706003B
:1037E00000888888F8888888030707060100E04079
:1037F00040404040E0050707060000381010101058
:1038000090600507070600008890A0C0A09088057A
:103810000707060000808080808080F80507070683
:10382000000088D8A88888888805070706000088CF
:1038300088C8A898888805070706000070888888C7
:10384000888870050707060000F08888F08080806F
:1038500005070706000070888888A8906805070794
:10386000060000F08888F0A0908805070706000091
:1038700070888070088870050707060000F820200F
:10388000202020200507070600008888888888886F
:1038900070050707060000888888885050200507B3
:1038A0000706000088888888A8A850050707060032
:1038B00000888850205088880507070600008888FF
:1038C0005020202020050707060000F8081020409F
:1038D00080F80309090601FFE080808080808080F5
:1038E000E00507070600008040402010100803098B
:1038F000090601FFE020202020202020E00503030E
:103900000600052050880501010600FEF8030303A8
:10391000060105804020050505060000700878882E
:10392000780507070600008080F0888888F0050584
:1039300005060000708080887005070706000008F3
:103940000878888888780505050600007088F0806A
:1039500070050707060000304840E040404005077A
:10396000070600FE7088888878087005070706003B
:10397000008080F0888888880307070601004000DF
:10398000C0404040E00409090601FE10003010105C
:103990001010906005070706000080808890E09076
:1039A00088030707060100C04040404040E005058D
:1039B00005060000D0A8A8A8A8050505060000B0C7
:1039C000C888888805050506000070888888700505
:1039D00007070600FEF0888888F080800507070644
:1039E00000FE78888888780808050505060000B07C
:1039F000C880808005050506000078807008F00505
:103A000007070600002020F82020201805050506DD
:103A10000000888888986805050506000088888861
:103A200050200505050600008888A8A85005050552
:103A300006000088502050880507070600FE888889
:103A40008850204080050505060000F8102040F849
:103A50000309090601FF204040408040404020010A
:103A600009090602FF8080808080808080800309B1
:103A7000090601FF8040404020404040800503038C
:103A800006000248A890FF4F4646004F4E0065636F
:103A9000686F3A004572726F723A004572726F72C7
:103AA0002077726974696E6720746F2045455052A3
:103AB0004F4D210A00507265737320627574746FE4
:103AC0006E20286F72204D3130382920746F2068A5
:103AD000656174206E6F7A7A6C650A005072657346
:103AE0007320627574746F6E20286F72204D3130B0
:103AF000382920746F20726573756D650A00496EF0
:103B0000736572742066696C616D656E7420616E98
:103B10006420707265737320627574746F6E2028F0
:103B20006F72204D313038290A004D3630303A203E
:103B3000546F6F20436F6C6400486F74656E64202F
:103B4000746F6F20636F6C640A00486F74656E64F5
:103B500020746F6F20636F6C640A00496E73657226
:103B6000742066696C616D656E7420616E6420708E
:103B70007265737320627574746F6E20286F722083
:103B80004D313038290A0063616E63656C007265DF
:103B900073756D656400726573756D650070617530
:103BA00073656400706F7765726F6666002F2F61B2
:103BB0006374696F6E3A0020573A0020573A004804
:103BC0006F74656E6420436F6F6C696E672E2E2E66
:103BD00000486F74656E642048656174696E672E75
:103BE0002E2E00202F002042403A0020403A004D67
:103BF000383420582059205A204500546865726D89
:103C0000616C2052756E6177617900486F74656EE2
:103C10006420544845524D414C2052554E41574125
:103C2000590042454420544845524D414C2052557C
:103C30004E4157415900202D20496E76616C6964D0
:103C4000206578747275646572206E756D62657238
:103C500020210A0048656174696E67206661696C9D
:103C60006564004265642048656174696E6720463A
:103C700061696C656400546865726D616C20527591
:103C80006E617761790042454420544845524D4168
:103C90004C2052554E415741590048656174696E38
:103CA00067206661696C656400486F74656E6420A6
:103CB00048656174696E67204661696C656400548B
:103CC0006865726D616C2052756E6177617900482C
:103CD0006F74656E6420544845524D414C205255D6
:103CE0004E41574159004D494E54454D5020747234
:103CF0006967676572656400486F74656E64204526
:103D000072723A204D494E54454D50004572723AF8
:103D1000204D494E54454D5020424544004D415898
:103D200054454D5020747269676765726564004838
:103D30006F74656E64204572723A204D4158544547
:103D40004D50004572723A204D415854454D502017
:103D500042454400626564002C2073797374656D7C
:103D60002073746F7070656421204865617465729A
:103D70005F49443A200023646566696E65204445C6
:103D80004641554C545F004B6420004B6920004B6A
:103D90007020000062656400504944204175746FD2
:103DA00074756E652066696E69736865642120505C
:103DB000757420746865206C617374204B702C20BE
:103DC0004B6920616E64204B6420636F6E73746175
:103DD0006E74732066726F6D2062656C6F772069F8
:103DE0006E746F20436F6E66696775726174696F78
:103DF0006E2E680A00504944204175746F74756EC8
:103E000065206661696C6564212074696D656F75F4
:103E1000740A00546865726D616C2052756E61772A
:103E2000617900486F74656E6420544845524D4175
:103E30004C2052554E415741590042454420544868
:103E400045524D414C2052554E415741590048650D
:103E50006174696E67206661696C656400486F749F
:103E6000656E642048656174696E67204661696C9F
:103E70006564004265642048656174696E67204628
:103E800061696C656400504944204175746F7475B4
:103E90006E65206661696C6564212054656D70658E
:103EA00072617475726520746F6F20686967680A43
:103EB00000204B643A2000204B693A2000204B70D0
:103EC0003A20000A20436C617373696320504944AF
:103ED000200A00204B643A2000204B693A20002041
:103EE0004B703A20000A204E6F206F76657273681F
:103EF0006F6F740A002054753A2000204B753A20E9
:103F000000206D61783A2000206D696E3A20002013
:103F1000643A200020626961733A200050494420CD
:103F20004175746F74756E652073746172740A00E4
:103F3000504944204175746F74756E6520666169DF
:103F40006C6564212054656D70657261747572656D
:103F500020746F6F20686967680A001000AD033035
:103F6000016A0150022B0170030A019004F500B0B0
:103F700005E500D006D800F007CE001009C50030D6
:103F80000ABE00500BB700700CB100900DAB00B032
:103F90000EA600D00FA200F0109D00101299003064
:103FA0001395005014920070158E0090168B00B07F
:103FB000178700D0188400F0198100101B7E003094
:103FC0001C7B00501D7900701E7600901F7300B09E
:103FD000207000D0216E00F0226B001024690030A8
:103FE000256600502663007027610090285E00B0AF
:103FF000295C00D02A5900F02B5600102D540030B7
:104000002E5100502F4E0070304B0090314800B0C0
:10401000324500D0334200F0343E0010363B0030D1
:104020003737005038330070392E00903A2900B0ED
:104030003B2300D03C1B00F03D1100103F0100F07D
:104040003F00001000C90210012C01400122017044
:10405000011801B0010E01F00104015002FA00B094
:1040600002F0003003E600D003DC009004D20070C0
:1040700005C800A006BE000008B400B009AA00D020
:104080000BA000600E960060118C000015820020CD
:10409000197800C01D6E00A0226400B0275A00905D
:1040A0002C500000314600E0343C001038320090C3
:1040B0003A2800603C1E00A03D1400803E0A00200B
:1040C0003F00006F70656E005452494747455245A6
:1040D00044003A20007A5F70726F6265007A5F6D0B
:1040E0006178007A5F6D696E00795F6D6178007943
:1040F0005F6D696E00785F6D617800785F6D696EE5
:10410000005265706F7274696E6720656E647374B7
:104110006F70207374617475730A00456E647374F4
:104120006F7073202563202563202563202563009D
:1041300020503A00205A3A0020593A0020583A00BC
:10414000656E6473746F7073206869743A200048F8
:104150006F6D696E67204661696C656400496E76B3
:10416000616C69642065787472756465720A0045D3
:10417000313A200045303A20005A3A2000593A207E
:10418000004D53312C4D53322C4D53332050696E1A
:10419000730A583A20004D6963726F7374657073C7
:1041A00020756E617661696C61626C650A00205AE7
:1041B0003A0020593A0020436F756E7420583A0037
:1041C000C23100001C260000F4190000D80F0000C6
:1041D000EB080000C0040000750200004001000070
:1041E00024F4D43050C38E20C2A24017828B7011A9
:1041F000127A910D816CD90AA861E108C758660747
:10420000615143061E4B5D05C145A7041A411104C7
:10421000093D9803713931034036DB026533910261
:10422000D4305402802E1D02632CEE01752AC50184
:10423000B028A001102781018F2564012B244B0198
:10424000E0223401AC211F018D200D01801FFC00F4
:10425000841EED00971DDF00B81CD200E61BC600CF
:10426000201BBC00641AB200B219A8000A19A000F1
:104270006A189900D117910040178B00B516840079
:1042800031167E00B31579003A157300C7146F001C
:1042900058146A00EE1366008813630025135E004D
:1042A000C7125B006C12570015125400C111510067
:1042B00070114F0021114B00D61049008D1047009E
:1042C0004610440002104200C00F4000800F3E0024
:1042D000420F3C00060F3B00CB0E3800930E370018
:1042E0005C0E3500270E3400F30D3200C10D310095
:1042F000900D3000600D2E00320D2D00050D2C00AC
:10430000D90C2B00AE0C2900850C29005C0C270071
:10431000350C27000E0C2600E80B2400C40B2400EB
:10432000A00B23007D0B23005A0B2100390B210029
:10433000180B2000F80A1F00D90A1E00BB0A1E0035
:104340009D0A1D00800A1D00630A1C00470A1B000D
:104350002C0A1B00110A1A00F7091A00DD091900BE
:10436000C4091900AB091900920917007B0918004C
:10437000630917004C0916003609160020091600BB
:104380000A091500F5081500E0081400CC0814000F
:10439000B8081400A4081400900813007D08120047
:1043A0006B08130058081200460812003408110068
:1043B000230811001208110001081100F007100075
:1043C000E0071000D0071000C0071000B0070F0072
:1043D000A107100091070E0083070F0074070F005C
:1043E00065070E0057070E0049070E003B070D003A
:1043F0002E070E0020070D0013070D0006070D0005
:10440000F9060C00ED060D00E0060C00D4060C00C9
:10441000C8060C00BC060C00B0060C00A4060B007D
:1044200099060C008D060B0082060B0077060B0028
:104430006C060B0061060A0057060B004C060A00CA
:1044400042060A0038060A002E060A0024060A0060
:104450001A060A001006090007060A00FD050900F1
:10446000F4050900EB050900E2050900D90509007A
:10447000D0050900C7050900BE050900B5050800FB
:10448000AD050800A50509009C0508009405080075
:104490008C050800840508007C05080074050800E8
:1044A0006C050700650508005D0507005605080056
:1044B0004E050700470507004005080038050700BE
:1044C000310507002A050700230507001C05060023
:1044D000160507000F05070008050600020507007E
:1044E000FB040600F5040700EE040600E8040600DD
:1044F000E2040700DB040600D5040600CF04060032
:10450000C9040600C3040600BD040600B704060083
:10451000B1040500AC040600A6040600A0040500D2
:104520009B04060095040500900406008A0405001B
:1045300085040500800406007A0405007504050062
:10454000700405006B0405006604050061040500A5
:104550005C04050057040500520405004D040500E5
:1045600048040500430405003E0404003A04050025
:1045700035040500300404002C0405002704040061
:10458000230405001E0404001A0404001604050098
:10459000110404000D0404000904050004040400CF
:1045A00000040400FC030400F8030400F403040006
:1045B000F0030400EC030400E8030400E403040037
:1045C000E0030400DC030400D8030400D403040067
:1045D000D0030400CC030400C8030300C503030098
:1045E00024F404D9201BC40C5C0E9804C4095F0297
:1045F00065077101F405F900FB04B3004804870066
:10460000C10369005803550003034500BE023A0088
:104610008402310053022A002902250004022000EE
:10462000E4011C00C8011900AF0117009801140033
:1046300084011300710110006101100051010E008E
:1046400043010D0036010B002B010B0020010B0074
:10465000150109000C01090003010800FB00080016
:10466000F3000800EB000700E4000600DE0006008F
:10467000D8000600D2000600CC000500C7000500E7
:10468000C2000500BD000400B9000400B50004002C
:10469000B1000400AD000400A9000400A50003005F
:1046A000A20003009F0004009B0003009800030089
:1046B0009500020093000300900003008D000200AB
:1046C0008B000300880002008600020084000300C3
:1046D000810002007F0002007D0002007B000200DA
:1046E00079000200770001007600020074000200E9
:1046F00072000100710002006F0002006D000100F5
:104700006C0002006A0001006900020067000100FD
:104710006600010065000100640002006200010003
:1047200061000100600001005F0002005D00010007
:104730005C0001005B0001005A000100590001000B
:10474000580001005700010056000100550001000B
:10475000540001005300000053000100520001000A
:1047600051000100500001004F0001004E00000008
:104770004E0001004D0001004C0001004B00000004
:104780004B0001004A000100490001004800000000
:1047900048000100470001004600000046000100FB
:1047A00045000000450001004400010043000000F6
:1047B00043000100420000004200010041000000EF
:1047C00041000100400001003F0000003F000100E7
:1047D0003E0000003E0001003D0000003D000100E1
:1047E0003C0000003C0000003C0001003B000000D9
:1047F0003B0001003A0000003A00010039000000CF
:1048000039000100380000003800000038000100C5
:1048100037000000370001003600000036000000BD
:1048200036000100350000003500000035000100B1
:1048300034000000340000003400010033000000A8
:10484000330000003300010032000000320000009D
:104850003200010031000000310000003100010091
:104860003000000030000000300001002F00000088
:104870002F0000002F0000002F0001002E0000007C
:104880002E0000002E0001002D0000002D00000071
:104890002D0000002D0001002C0000002C00000065
:1048A0002C0000002C0001002B0000002B00000059
:1048B0002B0000002B0001002A0000002A0000004D
:1048C0002A0000002A000100290000002900000041
:1048D0002900000029000000290001002800000034
:1048E0002800000028000000280000002800010027
:1048F000270000002700000027000000270000001C
:10490000270001002600000026000000260000000D
:104910002600000026000100250000002500000000
:1049200025000000250000002500000025000100F2
:1049300024000000240000002400000024000000E7
:1049400024000100230000002300000023000000D9
:1049500023000000230000002300000023000100CA
:1049600022000000220000002200000022000000BF
:1049700022000000220001002100000021000000B0
:1049800021000000210000002100000021000000A3
:104990002100010020000000200000002000000095
:1049A0002000000020000000200000002000000087
:1049B000200001001F0000001F0000001F00000079
:1049C0001F0000001F0000001F0000001F0001006A
:1049D0001E0000001E0000001E0000001E0000005F
:1049E00020204D36303320003A0A0020286D6D29F2
:1049F00000205300205A0020590020580020204D4C
:104A00003432352046004261636B6C617368206309
:104A10006F6D70656E736174696F6E3A0A00205530
:104A2000004C0046696C616D656E74206C6F61644A
:104A30002F756E6C6F6164206C656E677468733A75
:104A40000A0020204D393030204B004C696E6561E2
:104A50007220416476616E63653A0A0020204D3809
:104A60003531205A005A2D50726F6265204F6666AC
:104A70007365740020440020490020204D333034F9
:104A800020500020440020490020204D33303120A8
:104A900050005049442073657474696E67733A0A14
:104AA0000020460020420020480020204D313435AF
:104AB0002053004D6174657269616C206865617492
:104AC000757020706172616D65746572733A0A0069
:104AD00020204D3432302053004175746F204265E0
:104AE00064204C6576656C696E673A0A0020450063
:104AF000205A002059002058002054002053002044
:104B0000204D32303520420020453C6D61785F6594
:104B10005F6A65726B3E0020583C6D61785F785F1C
:104B20006A65726B3E20593C6D61785F795F6A659A
:104B3000726B3E205A3C6D61785F7A5F6A65726B7A
:104B40003E00416476616E6365643A20423C6D6963
:104B50006E5F7365676D656E745F74696D655F75B3
:104B6000733E20533C6D696E5F6665656472617467
:104B7000653E20543C6D696E5F74726176656C5F52
:104B800066656564726174653E00205400205200C1
:104B900020204D323034205000416363656C6572D3
:104BA0006174696F6E2028756E6974732F73322972
:104BB0003A20503C7072696E745F616363656C3E4D
:104BC00020523C726574726163745F616363656CEB
:104BD0003E20543C74726176656C5F616363656C02
:104BE0003E0A00204500205A0020590020204D3266
:104BF00030312058004D6178696D756D20416363D7
:104C0000656C65726174696F6E2028756E69747366
:104C10002F7332293A0A00204500205A00205900FB
:104C200020204D3230332058004D6178696D756D0C
:104C3000206665656472617465732028756E697499
:104C4000732F73293A0A005374657073207065726C
:104C500020756E69743A0A0020204D3134392043A2
:104C6000203B20556E69747320696E2043656C7318
:104C70006975730A002020473231202020203B2014
:104C8000556E69747320696E206D6D0048617264A1
:104C9000636F6465642044656661756C7420536558
:104CA0007474696E6773204C6F616465640A0028D0
:104CB00023000028230000640000002823000000D7
:104CC00000964300009643000040400000C84100A9
:104CD00000C9420000C9420000C8440000D2434558
:104CE0004550524F4D20496E697469616C697A650F
:104CF000640A00290A002062797465733B2063729C
:104D00006320002073746F72656420736574746926
:104D10006E67732072657472696576656420280019
:104D2000202863616C63756C6174656429210A00D5
:104D300020213D2000454550524F4D2043524320F5
:104D40006D69736D61746368202D202873746F72B0
:104D500065642920002053697A653A2000496E6411
:104D600065783A2000204D61726C696E3D56363987
:104D7000290A00454550524F4D2076657273696F80
:104D80006E206D69736D61746368202845455052CB
:104D90004F4D3D004E6F20454550524F4D2E0A005D
:104DA000290A002062797465733B206372632000D6
:104DB00053657474696E67732053746F72656420F1
:104DC00028004E6F20454550524F4D2E0A00454554
:104DD00050524F4D206461746173697A6520657229
:104DE000726F722E0A004175746F6C6576656C2067
:104DF0006661696C65640A004175746F6C657665FF
:104E00006C206661696C656400205A3A2000205964
:104E10003A200042656420583A20005761726E695A
:104E20006E673A20486F6D696E672042756D70201D
:104E300044697669736F72203C20310A00020204D3
:104E4000486F6D652025732573257320466972733D
:104E500074002046697273740A00486F6D65200003
:104E600020746F6F206C6F6E672065787472757335
:104E7000696F6E2070726576656E7465640A0020D5
:104E8000636F6C6420657874727573696F6E2070DF
:104E9000726576656E7465640A0020453A00205A92
:104EA0003A0020593A00583A0000004842000048B1
:104EB0004200004040FF01FF0000A0400000A04071
:104EC000000000400000A0430080A1430000874391
:104ED0000000A0C10080964300000000000096433F
:104EE00000809643000087430000A0C10000B0C1CD
:104EF0000000000020746F6F206C6F6E6720657873
:104F000074727573696F6E2070726576656E746504
:104F1000640A0020636F6C6420657874727573692D
:104F20006F6E2070726576656E7465640A006275D6
:104F300073793A2070617573656420666F722069B9
:104F40006E7075740A00627573793A2070617573BA
:104F5000656420666F7220757365720A00627573EE
:104F6000793A2070726F63657373696E670A004DDA
:104F70003131372050726F626520737563636573DA
:104F80007366756C0020496E76616C696420657883
:104F90007472756465722000205A3A200020593AD4
:104FA000200042656420583A200050726F626520EC
:104FB0005A204F66667365743A20003F5A206F7519
:104FC00074206F662072616E676520282D32207410
:104FD0006F2035290A004D31343520533C696E6409
:104FE00065783E206F7574206F662072616E67650C
:104FF0002028302D31290A00436C69636B20746FBF
:1050000020526573756D652E2E2E00220A00556E96
:105010006B6E6F776E20636F6D6D616E643A2022E8
:1050200000454550524F4D204F4B0A004E6F204DCA
:105030006F76652E004543484F00494E464F004568
:1050400052524F52530044525952554E00434F4D05
:105050004D554E49434154494F4E006F66660035E9
:10506000503A503F5046504D5044454255473A0003
:105070004C756C7A426F742054415A2036204F464A
:10508000462E00205A00205900580020204D6178FB
:105090003A2000205A00205900580020204D696E07
:1050A0003A2000536F667420656E6473746F70737A
:1050B0003A20002569730025696D20256973002554
:1050C00069682025696D202569730025696420259C
:1050D00069682025696D2025697300256979202577
:1050E0006964202569682025696D20256973005051
:1050F00072696E742074696D653A20004D313133E8
:105100002053002F2F20004361703A004348414D47
:105110004245525F54454D50455241545552450009
:105120004D4F54494F4E5F4D4F44455300544845F1
:10513000524D414C5F50524F54454354494F4E00DD
:105140004155544F5245504F52545F53445F53544E
:10515000415455530050524F4D50545F5355505089
:105160004F525400454D455247454E43595F5041BB
:105170005253455200434153455F4C494748545FA1
:105180004252494748544E45535300544F47474CA9
:10519000455F4C494748545300534F46545741527A
:1051A000455F504F574552004255494C445F50456A
:1051B0005243454E54004C4556454C494E475F447A
:1051C000415441005A5F50524F4245004155544F9F
:1051D0004C4556454C005052494E545F4A4F420090
:1051E00050524F4752455353004155544F5245502A
:1051F0004F52545F54454D5000564F4C554D4554F9
:1052000052494300454550524F4D0042494E41528C
:10521000595F46494C455F5452414E5346455200F2
:1052200053455249414C5F584F4E5F584F464600D8
:105230004649524D574152455F4E414D453A4D61A9
:10524000726C696E20322E302E302E313638202886
:105250004769746875622920534F555243455F432F
:105260004F44455F55524C3A68747470733A2F2F0F
:10527000636F64652E616C6570686F626A656374E4
:10528000732E636F6D2F646966667573696F6E2F19
:105290004D41524C494E2050524F544F434F4C5F5A
:1052A00056455253494F4E3A312E30204D414348D6
:1052B000494E455F545950453A4C756C7A426F746B
:1052C0002054415A20362045585452554445525F87
:1052D000434F554E543A3120555549443A383435A8
:1052E00066303033632D616562642D346535332D4E
:1052F000613662392D37643039383466646536304A
:10530000390A0020284E6F7420796574206D65611C
:105310007375726564290020204176657261676546
:10532000206D65617375726564206261636B6C6189
:10533000736820286D6D293A002020536D6F6F74BB
:1053400068696E6720286D6D293A20202020202072
:105350002020202020202020202020530020204218
:1053600061636B6C6173682044697374616E63651B
:1053700020286D6D293A2020202020202020002088
:105380002846312E30203D2066756C6C2C2046302E
:105390002E30203D206E6F6E65290A002020436F5D
:1053A0007272656374696F6E20416D6F756E742FD4
:1053B000466164652D6F75743A20202020204600D8
:1053C0006163746976653A0A00696E004261636BD5
:1053D0006C61736820436F7272656374696F6E20CD
:1053E00000486F6D652058592046697273740A0031
:1053F000486F6D6520585920466972737400426584
:1054000064204C6576656C696E6720004661696C46
:10541000656420746F20656E61626C65204265640E
:10542000204C6576656C696E670A00426564204CA5
:105430006576656C20436F7272656374696F6E2068
:105440004D61747269783A000A0A426564204C65BD
:1054500076656C20436F7272656374696F6E204D60
:1054600061747269783A00202B000A436F7272658A
:1054700063746564204265642048656967687420C8
:1054800076732E2042656420546F706F6C6F67795D
:105490003A0A00202B000A42656420486569676863
:1054A0007420546F706F6772617068793A0A2020B7
:1054B000202B2D2D2D204241434B202D2D2B0A201A
:1054C00020207C20202020202020202020207C0A3A
:1054D000204C207C20202020282B29202020207CCC
:1054E00020520A2045207C2020202020202020201F
:1054F00020207C20490A2046207C20282D29204E6F
:1055000020282B29207C20470A2054207C20202082
:1055100020202020202020207C20480A2020207CC1
:1055200020202020282D29202020207C20540A20E3
:1055300020207C20202020202020202020207C0AC9
:105540002020204F2D2D2046524F4E54202D2D2B04
:105550000A2028302C30290A000A4D65616E206F20
:10556000662073616D706C656420706F696E747312
:105570003A200020643A200020623A200045716EF3
:1055800020636F656666696369656E74733A20614E
:105590003A200050726F62696E6720506F696E74B6
:1055A0002025692F2569002E0A002F0050726F6296
:1055B000696E67206D65736820706F696E74200076
:1055C000202844525952554E2900473239204175FE
:1055D000746F20426564204C6576656C696E670067
:1055E0003F20284C2C522C462C4229206F757420C9
:1055F0006F6620626F756E64732E0A003F50726F83
:10560000626520706F696E74732028592920696D56
:10561000706C61757369626C652028322D32292E99
:105620000A003F50726F626520706F696E7473205C
:1056300028582920696D706C61757369626C6520EA
:1056400028322D32292E0A003F2856296572626FB2
:105650007365206C6576656C20696D706C6175731F
:1056600069626C652028302D34292E0A004375723A
:1056700072656E742066696C653A2000456E642020
:1056800066696C65206C6973740A00426567696EAF
:105690002066696C65206C6973740A0041647661E8
:1056A0006E6365204B3D003F4B2076616C75652035
:1056B0006F7574206F662072616E67652028302DCB
:1056C0003130292E0A004D31313720486F74206562
:1056D0006E642068656174696E672E2E2E0A4D31E6
:1056E000303420533137300A473238204F310A4D99
:1056F00031313720576970696E67206E6F7A7A6C26
:10570000650A54300A473120582D31372059323537
:10571000205A31302046343030300A4D3130392073
:10572000523137300A4731205A310A4D3131340A6B
:10573000473120582D3137205932350A473120580A
:105740002D3137205939350A473120582D3137202E
:105750005932350A473120582D3137205939350A09
:10576000473120582D3137205932350A47312058DA
:105770002D3137205939350A473120582D313720FE
:105780005932350A473120582D3137205939350AD9
:10579000473120582D3137205932350A47312058AA
:1057A0002D3137205939350A473120582D313720CE
:1057B0005932350A473120582D3137205939350AA9
:1057C0004731205A31350A4D3430300A4D313036A8
:1057D00020533235350A473020582D313020592D8D
:1057E000394D31303920523136300A4D31303700A1
:1057F0004732380020466C6F773A200020643A0028
:1058000020693A0020703A00204500205A002059B3
:1058100000204D393220580043290A0061626C652E
:105820006420286D696E2074656D70200064697352
:1058300000656E00436F6C642065787472756465F2
:105840007320617265200020540020520041636380
:10585000656C65726174696F6E3A205000496E76AE
:10586000616C69642065787472756465720A0020E1
:10587000643A0020693A0020703A00536C65657004
:105880002E2E2E0047322F47332062616420706134
:1058900072616D65746572730A0050726F62652083
:1058A0005A204F66667365743A2000446F6E652017
:1058B000736176696E672066696C652E0A005344D1
:1058C0002072656164206572726F720A00446F6EA7
:1058D00065207072696E74696E672066696C650A0E
:1058E000004D32390053544F505045442E20005043
:1058F00072696E7465722073746F70706564206471
:10590000756520746F206572726F72732E20466900
:105910007820746865206572726F7220616E6420F1
:10592000757365204D39393920746F207265737431
:105930006172742E202854656D7065726174757281
:10594000652069732072657365742E205365742019
:105950006974206166746572207265737461727413
:10596000696E67290A004E6F20436865636B737523
:105970006D2077697468206C696E65206E756D6244
:1059800065722C204C617374204C696E653A20005E
:105990004E6F20436865636B73756D20776974681B
:1059A000206C696E65206E756D6265722C204C618D
:1059B0007374204C696E653A2000636865636B738D
:1059C000756D206D69736D617463682C204C617313
:1059D00074204C696E653A20004C696E65204E75E6
:1059E0006D626572206973206E6F74204C617374F0
:1059F000204C696E65204E756D6265722B312C20CE
:105A00004C617374204C696E653A20004D31313021
:105A100000526573656E643A2000204200205000F9
:105A20006F6B00220A00656E7175657565696E673A
:105A3000202200504944204175746F74756E6520B2
:105A40006661696C656421204261642065787472C6
:105A500075646572206E756D6265720A00426564D8
:105A600020436F6F6C696E672E2E2E004265642096
:105A700048656174696E672E2E2E006F6B00473289
:105A8000385859002020506C616E6E657242756600
:105A900066657242797465733A20002046726565C6
:105AA000204D656D6F72793A2000436F6D70696C9F
:105AB00065643A2053657020323720323031390A1C
:105AC00000207C20417574686F723A2028416C6513
:105AD0007068204F626A6563747320496E632E2C70
:105AE000204C756C7A426F7420476974205265703F
:105AF0006F7369746F7279290A00536570203237A9
:105B0000203230313931363A32313A313600204C98
:105B100061737420557064617465643A2000322E9C
:105B2000302E302E3136380A004D61726C696E00AD
:105B300020536F6674776172652052657365740ACD
:105B400000205761746368646F67205265736574E1
:105B50000A002042726F776E206F75742052657351
:105B600065740A002045787465726E616C20526518
:105B70007365740A00506F77657255700A0073740C
:105B80006172740A004B494C4C45442E20005072FF
:105B9000696E7465722068616C7465642E206B692F
:105BA0006C6C28292063616C6C6564210A004B4988
:105BB0004C4C2063617573656420627920746F6F4B
:105BC000206D75636820696E616374697665207401
:105BD000696D65202D2063757272656E7420636F28
:105BE0006D6D616E643A20004730205A31300A47AB
:105BF00031320A4D31303920523136300A4D34308D
:105C0000300A4D3131372050726F62696E67206201
:105C100065640070726F62655F72657769706500B8
:105C20004175746F6C6576656C206661696C65643E
:105C3000004D31313720426564206C6576656C69B2
:105C40006E67206661696C65642E0A4730205A31A0
:105C5000300A47302045300A4D333030205032353D
:105C600020533838300A4D333030205035302053EF
:105C7000300A4D3330302050323520533838300A16
:105C80004D333030205035302053300A4D333030D2
:105C90002050323520533838300A473420533100F1
:105CA00070726F62655F6661696C65640050726FE7
:105CB0007465637465642050696E0A0025301D0C9C
:105CC00018282924311C0B174527232F1B0A1E4493
:105CD0004316222B1A4142033809FF3603080602F5
:105CE00002000100074708873D91B7A8A4C4E60059
:105CF000E000E400E2005D9111241FBECFEFD1E28D
:105D0000DEBFCDBF00E00CBF13E0A0E0B2E0EAE0F0
:105D1000F6EB02E00BBF02C007900D92AE3BB1075D
:105D2000D9F726E1AEEBB3E001C01D92AC3BB20760
:105D3000E1F71EE2CBE7DEE200E006C021970109B1
:105D4000802FFE010F943B50C237D10780E0080737
:105D5000A9F70E94263B0D94F35A0C9400001F9261
:105D60000F920FB60F9211242F933F938F939F930F
:105D7000AF93BF938091BF039091C003A091C103E3
:105D8000B091C2033091BE0323E0230F2D3720F4DE
:105D90000196A11DB11D05C026E8230F0296A11D85
:105DA000B11D2093BE038093BF039093C003A093C3
:105DB000C103B093C2038091C3039091C403A09127
:105DC000C503B091C6030196A11DB11D8093C30305
:105DD0009093C403A093C503B093C603BF91AF9142
:105DE0009F918F913F912F910F900FBE0F901F9019
:105DF00018952FB7F8946091BF037091C0038091FC
:105E0000C1039091C2032FBF08953FB7F8948091CA
:105E1000C3039091C403A091C503B091C60326B5F6
:105E2000A89B05C02F3F19F00196A11DB11D3FBFD2
:105E3000BA2FA92F982F8827820F911DA11DB11D60
:105E4000BC01CD0142E0660F771F881F991F4A955C
:105E5000D1F708958F929F92AF92BF92CF92DF9227
:105E6000EF92FF926B017C01D0DF4B015C01C1140A
:105E7000D104E104F104F1F09CD3C7DFDC01CB01D4
:105E800088199909AA09BB09883E9340A105B10563
:105E900070F321E0C21AD108E108F10888EE880EFB
:105EA00083E0981EA11CB11CC114D104E104F104CB
:105EB00021F7DDCFFF90EF90DF90CF90BF90AF90B4
:105EC0009F908F9008958230910538F0880F991F28
:105ED000880F991F05970197F1F70895789484B575
:105EE000826084BD84B5816084BD85B5826085BDD6
:105EF00085B5816085BDEEE6F0E0808181608083BC
:105F0000E1E8F0E01082808182608083808181609E
:105F10008083E0E8F0E0808181608083E1EBF0E065
:105F2000808184608083E0EBF0E080818160808309
:105F3000E1E9F0E0808182608083808181608083FC
:105F4000E0E9F0E0808181608083E1EAF0E0808137
:105F500082608083808181608083E0EAF0E08081DC
:105F600081608083E1E2F1E08081826080838081D2
:105F700081608083E0E2F1E0808181608083EAE7F4
:105F8000F0E0808184608083808182608083808172
:105F9000816080838081806880831092C100089531
:105FA0001F93CF93DF93182FEB0161E016D1209759
:105FB00011F460E004C0CF3FD10531F461E0812FDE
:105FC000DF91CF911F9145C1E12FF0E0EB5FFC4FD6
:105FD000E4914E2F50E0FA013197E231F10508F0DB
:105FE0009DC08827EE58FF4F8F4F0D943B5084B5CE
:105FF000806884BDC7BD97C084B5806284BDC8BDBC
:1060000092C080918000806880938000D093890046
:10601000C093880088C08091800080628093800057
:10602000D0938B00C0938A007EC0809180008860EE
:1060300080938000D0938D00C0938C0074C08091B9
:10604000B00080688093B000C093B3006CC08091B2
:10605000B00080628093B000C093B40064C08091AF
:106060009000806880939000D0939900C09398002E
:106070005AC080919000806280939000D0939B00E2
:10608000C0939A0050C080919000886080939000E7
:10609000D0939D00C0939C0046C08091A000806872
:1060A0008093A0008091A0008F7B8093A000D0936C
:1060B000A900C093A80037C08091A000806280939F
:1060C000A000D093AB00C093AA002DC08091A00087
:1060D00088608093A000D093AD00C093AC0023C033
:1060E00080912001806880932001D0932901C09382
:1060F000280119C080912001806280932001D093F3
:106100002B01C0932A010FC08091200188608093E9
:106110002001D0932D01C0932C0105C0C038D105BA
:106120000CF04CCF46CFDF91CF911F91089590E0B6
:10613000FC013197E231F10508F04EC08827EC5799
:10614000FF4F8F4F0D943B50809180008F7703C09D
:10615000809180008F7D80938000089580918000E1
:10616000877FF9CF84B58F7702C084B58F7D84BDDA
:1061700008958091B0008F7703C08091B0008F7D2B
:106180008093B0000895809190008F7707C0809130
:1061900090008F7D03C080919000877F8093900056
:1061A00008958091A0008F7707C08091A0008F7D17
:1061B00003C08091A000877F8093A0000895809104
:1061C00020018F7707C0809120018F7D03C08091CF
:1061D0002001877F809320010895CF93DF9390E083
:1061E000FC01E55BFC4F2491FC01EF56FC4F8491D0
:1061F000882361F190E0880F991FFC01E55FFB4F58
:10620000C591D491FC01EF50FC4FA591B49161115F
:1062100009C09FB7F8948881209582238883EC91E8
:106220002E230BC0623061F49FB7F8943881822F1F
:10623000809583238883EC912E2B2C939FBF06C0DF
:106240008FB7F894E8812E2B28838FBFDF91CF91F1
:1062500008951F93CF93DF93282F30E0F901EB5F70
:10626000FC4F8491F901E55BFC4FD491F901EF56A5
:10627000FC4FC491CC23C1F0162F811158DFEC2FB5
:10628000F0E0EE0FFF1FEF50FC4FA591B4918FB7D8
:10629000F894111105C09C91ED2FE095E92302C0FF
:1062A000EC91ED2BEC938FBFDF91CF911F9108956F
:1062B000CF93DF93282F30E0F901EB5FFC4F8491FF
:1062C000F901E55BFC4FD491F901EF56FC4FC49105
:1062D000CC2389F081112BDFEC2FF0E0EE0FFF1FB4
:1062E000E952FC4FA591B491EC91ED2381E090E04F
:1062F00021F480E002C080E090E0DF91CF9108952A
:1063000008951F920F920FB60F9211240BB60F92A1
:106310002F933F934F935F936F937F938F939F93AD
:10632000AF93BF93EF93FF93E0910802F0910902BE
:106330001995FF91EF91BF91AF919F918F917F91AF
:106340006F915F914F913F912F910F900BBE0F90E6
:106350000FBE0F901F9018951F920F920FB60F92BD
:1063600011240BB60F922F933F934F935F936F932C
:106370007F938F939F93AF93BF93EF93FF93E0919E
:106380000A02F0910B021995FF91EF91BF91AF9125
:106390009F918F917F916F915F914F913F912F913D
:1063A0000F900BBE0F900FBE0F901F9018951F926D
:1063B0000F920FB60F9211240BB60F922F933F93AB
:1063C0004F935F936F937F938F939F93AF93BF93FD
:1063D000EF93FF93E0910C02F0910D021995FF915C
:1063E000EF91BF91AF919F918F917F916F915F914D
:1063F0004F913F912F910F900BBE0F900FBE0F90BA
:106400001F9018951F920F920FB60F9211240BB682
:106410000F922F933F934F935F936F937F938F933D
:106420009F93AF93BF93EF93FF93E0910E02F09190
:106430000F021995FF91EF91BF91AF919F918F91AD
:106440007F916F915F914F913F912F910F900BBE74
:106450000F900FBE0F901F9018951F920F920FB6BE
:106460000F9211240BB60F922F933F934F935F938C
:106470006F937F938F939F93AF93BF93EF93FF930C
:10648000E0910402F09105021995FF91EF91BF91FF
:10649000AF919F918F917F916F915F914F913F91BC
:1064A0002F910F900BBE0F900FBE0F901F9018955D
:1064B0001F920F920FB60F9211240BB60F922F93CB
:1064C0003F934F935F936F937F938F939F93AF937C
:1064D000BF93EF93FF93E0910602F09107021995A5
:1064E000FF91EF91BF91AF919F918F917F916F91AC
:1064F0005F914F913F912F910F900BBE0F900FBE68
:106500000F901F9018951F920F920FB60F921124A3
:106510000BB60F922F933F934F935F936F937F939D
:106520008F939F93AF93BF93EF93FF93E0911002EC
:10653000F09111021995FF91EF91BF91AF919F9149
:106540008F917F916F915F914F913F912F910F901C
:106550000BBE0F900FBE0F901F9018951F920F92B9
:106560000FB60F9211240BB60F922F933F934F93B8
:106570005F936F937F938F939F93AF93BF93EF93AB
:10658000FF93E0911202F09113021995FF91EF91A0
:10659000BF91AF919F918F917F916F915F914F913B
:1065A0003F912F910F900BBE0F900FBE0F901F9039
:1065B000189508951F93CF93DF93EC011D821C82E1
:1065C0001F821E82198681E0888782E28A871F8661
:1065D0001E86FE01B396CE01C1962FEF2193E817D8
:1065E000F907E1F711E018A3CE0122D61F8B188E10
:1065F000198E80E48A8F1B8E89EE96E39AAB89AB65
:10660000DF91CF911F910895DB01ED91FC911994D9
:10661000EF92FF921F93CF93DF931F921F92CDB7FC
:10662000DEB77C01DC01D196ED91FC91D29782E03E
:1066300069837A83199520E030E04AE069817A81A4
:10664000C701E2DF182FD701D196ED91FC91D297C7
:1066500083E01995D701D196ED91FC91D29780E016
:106660001995812F0F900F90DF91CF911F91FF907F
:10667000EF9008950F931F93CF93DF93EC018B015D
:10668000E9A9FAA982E01995E9A9FAA981E0199581
:1066900020E030E044E1B801CE01B6DF9E012D5C80
:1066A0003F4F47E1B801CE01AFDFE9A9FAA980E089
:1066B000DF91CF911F910F911994EF92FF921F9349
:1066C000CF93DF93EC017B01E9A9FAA982E0199548
:1066D000E9A9FAA981E0199520E030E045E1B70188
:1066E000CE0192DF182F882339F09E012D5C3F4F99
:1066F00047E1B701CE0188DFE9A9FAA980E0199541
:10670000812FDF91CF911F91FF90EF900895FC01B1
:10671000448F258F9C01245E3F4F42E375CFCF937A
:10672000DF931F92CDB7DEB79E012F5F3F4F46E448
:106730006BDF89810F90DF91CF910895CF93DF9325
:106740001F92CDB7DEB79E012F5F3F4F47E45CDF5E
:1067500089810F90DF91CF91089520E030E048E4E7
:1067600053CFCF93DF93EC016A817B81D8DF88839D
:106770006A817B81CE01E2DF89836A817B81CE01E0
:10678000ECDF8B879E012D5C3F4F6A817B8147E167
:10679000CE01DF91CF9138CFCF93DF93EC016A81A7
:1067A0007B8136DF882319F0CE01DBDF81E0DF91CA
:1067B000CF9108958F929F92AF92BF92CF92EF9216
:1067C0000F93CF93DF931F921F92CDB7DEB74C018B
:1067D0005B012A834983EEDEF401B382A282498100
:1067E00047A32A8120A705A3E4A2C3A2C4010F9056
:1067F0000F90DF91CF910F91EF90CF90BF90AF901E
:106800009F908F90C9CFFC016281738133CFCF936A
:10681000DF93EC01EE85FF85309709F019956A81C9
:106820007B81CE01DF91CF9148CF362F242FFC0101
:1068300062817381432F6BCF0F93FC01828193811F
:10684000648F458F278F068F9F01245E3F4F4BE358
:10685000BC01CF010F91D8CEFC0160A30895BF9277
:10686000CF92DF92EF92FF920F931F93CF93DF931C
:106870006C01D62FB42EC22F7801CC2369F0F7011A
:10688000049120E04B2D6D2FC601D6DFFFEFEF1AEC
:10689000FF0AC150D85FF1CFDF91CF911F910F91C7
:1068A000FF90EF90DF90CF90BF9008958F929F92CE
:1068B000AF92BF92CF92DF92EF92FF920F931F930E
:1068C000CF93DF935C01C62EC42FD22ED02F220F80
:1068D000220F220F1ED0882379F0DC0F8D2C912CF3
:1068E000CD1751F087012D2D4C2F6C2DC501B7DF31
:1068F000E80CF91CCF5FF4CFDF91CF911F910F917E
:10690000FF90EF90DF90CF90BF90AF909F908F90CF
:1069100008950F93FC010150040F84A996A99417C0
:1069200018F0081728F402C0081750F0041740F4B4
:106930002150260F83A995A9961720F4281720F433
:1069400080E007C0281720F481E0261710F0F8CF68
:1069500081E00F91089581E008952EE93FE00097CE
:1069600029F0F9013197F1F70197F9CF0895FC016A
:10697000128280818150838314820895FC0180817A
:106980009281980F92832181921760F494819F5F86
:1069900094839381890F821710F08FEF820F838386
:1069A00081E0089580E00895FC0191E083818617DD
:1069B00008F490E031E0461708F030E0832F892B8F
:1069C00021E05281451708F420E02823832F8923F2
:1069D000822B0895DC01FB01108212968C91129794
:1069E000818315968C9115978150828313968C9193
:1069F00083830895FB0141812381213029F02330D5
:106A000031F468EF640F04C0642F485F01C0642F45
:106A1000CBCFDC0115962C9115971696ED91FC9134
:106A20001797CF01820F911D820F911D1192E817C8
:106A3000F907E1F70895FC01A681B7818281481B1F
:106A40008581483018F0A80FB11D4770382F369552
:106A500036953695562F577080E890E002C0959590
:106A600087955A95E2F7439F402D112466956695C8
:106A70006695E62FF0E0E40FF11DEA0FFB1F308171
:106A8000222311F0832B02C08095832380830895F5
:106A9000FB014181DC0112962C911297421760F0A4
:106AA00013962C911397241738F0608115962C912A
:106AB000621710F42481BFCF0895CF92DF92FF9226
:106AC0000F931F93CF93DF936C01EB01FA809B81AF
:106AD000913051F030F0923049F0933051F41FEF83
:106AE00009C010E001E007C011E004C010E00FEFA2
:106AF00002C010E000E0F7FE03C0BE01C601C8DF1F
:106B00009881900F98839981910F9983FF0C99F741
:106B1000DF91CF911F910F91FF90DF90CF9008955B
:106B20000F931F93CF93DF938901FB01C281D38120
:106B30004233D9F058F44531E1F0473109F144319D
:106B400041F5CE0166DFCE0112DF23C04634E1F00D
:106B50004734E1F04B33E9F4B901CE014BDF882330
:106B6000C1F0B801CE01A9DF14C0B901CE0190DF98
:106B700010C0CE0103DF882369F0CE014ADF09C0CF
:106B8000B901CE0127DF05C08D8101C08981F801DF
:106B9000808381E0DF91CF911F910F910895CF9273
:106BA000DF92EF92FF920F931F93CF93DF937C01BD
:106BB000D62FD42EC22F122FC62EC20E6C2D611BC3
:106BC000183038F00FEF20E04D2DC70135DE18509A
:106BD000F5CF6C2F687F6D0F2C2F277071F097E029
:106BE00029272F5F27700FEF10E001C0000F2A95B3
:106BF000EAF720E04D2DC7011FDEDF91CF911F91F5
:106C00000F91FF90EF90DF90CF900895CF92DF9299
:106C1000EF92FF920F931F93CF93DF937C01D62EB9
:106C2000D42FC22F122FC42EC20E4C2D411B183050
:106C300038F00FEF21E06D2DC701FEDD1850F5CFC4
:106C40004C2F487F4D0F2C2F277071F097E029278C
:106C50002F5F27700FEF10E001C0000F2A95EAF7B1
:106C600021E06D2DC701E8DDDF91CF911F910F91DC
:106C7000FF90EF90DF90CF900895EF92FF920F93E7
:106C80001F93CF93DF93EC01162FF42EE22E01E039
:106C900040DE882359F02E2D4F2D612FCE01DF913C
:106CA000CF911F910F91FF90EF9079CFDF91CF910E
:106CB0001F910F91FF90EF900895EF92FF920F9325
:106CC0001F93CF93DF93EC01162FF42EE22E022FA9
:106CD00021E01FDE882359F02E2D4F2D612FCE018C
:106CE000DF91CF911F910F91FF90EF908FCFDF91A8
:106CF000CF911F910F91FF90EF900895DF92EF9247
:106D0000FF920F931F93CF93DF937C01162FC42F15
:106D1000D22ED02FFEDD8823F9F02D2D4C2F612FA0
:106D2000C7013DDF2D2F4C2F612FC7016FDF6FEFA4
:106D30006D0D610F2D2F4C2FC70168DF4FEF4D0FE9
:106D40004C0F2D2D612FC701DF91CF911F910F9116
:106D5000FF90EF90DF9023CFDF91CF911F910F91A4
:106D6000FF90EF90DF900895EF92FF920F931F93A3
:106D7000CF93DF937C01D62F122FC42F040F212F26
:106D80004C2F6D2FC7010BDFCF5F0C13F8CFDF91B6
:106D9000CF911F910F91FF90EF900895DF92EF92A6
:106DA000FF920F931F93CF93DF93EC01162FF42ED6
:106DB000E22EAFDD882329F02E2D4F2D612FCE013D
:106DC000D3DFDF91CF911F910F91FF90EF90DF9074
:106DD00008950895FC01E60FF11D849190E0982F2D
:106DE00088273196E4918E0F911D0895FC018491BE
:106DF0000895FCDF882321F0823011F083E00895AC
:106E000086E0089580E00895FC018081089566E0A1
:106E1000E1CF68E0DFCF0A96FC01849108950B96DC
:106E2000FC0184910895DC011496ED91FC91159775
:106E3000319684910895BF92CF92DF92EF92FF92A4
:106E40000F931F93CF93DF938C01E62EDC011496F2
:106E5000CD91DC911597CE01C9DFF82EF801848120
:106E60009581C7DFC82EF1E0FF1203C02FE0B22EDC
:106E700002C0BB24BA94D80114968D919C911597A9
:106E8000CADFF82EF80184819581C9DFD82ED80198
:106E900014968D919C911597BCDFB0E6BE1538F421
:106EA000009729F0C80FD91F91E6F92E0FC0F801FD
:106EB00084819581ACDFF0E4FE1538F4009729F069
:106EC000C80FD91F81E4F82E01C06196DE1490F43A
:106ED000D80150961C92509753961C9253975496F3
:106EE0001C92549751961C92519752961C9280E096
:106EF00090E066C0DF1460F38C2D90E0FE012491D9
:106F00002F3F11F4219657C0FE104CC0D8011496A3
:106F10008D919C9115976ADF9E012F5F3F4FFE0177
:106F2000882311F08230E1F48491D80153968C9338
:106F30005397F901249154962C935497FE0133965C
:106F4000E4915096EC935097FE013496E49151965B
:106F5000EC935197FE013596E4915296EC9320C044
:106F60008491982F9F709250D80152969C9352977B
:106F700082958F7051968C935197F9012491822FAD
:106F80008F7054968C93549722952F7053962C9310
:106F90005397FE013296E491E295EF705096EC9390
:106FA000CE010EC0FE013296E491EB219C012E0F22
:106FB000311DC20FD31FFD1409F48ACFF3949ECF65
:106FC000DF91CF911F910F91FF90EF90DF90CF90C5
:106FD000BF9008954F925F926F927F929F92AF926F
:106FE000BF92CF92DF92EF92FF920F931F93CF93B6
:106FF000DF931F92CDB7DEB72C01C62E942E622FE1
:107000001ADF7C01892B09F43AC0F2018481958151
:10701000F0DEB82EF201138904898189C80E8289B5
:10702000981AD92CD01A212F4D2D6C2DC20171DC4C
:10703000882311F1EB0CF11C195F16951695169526
:10704000612E712CD914C1F03C2D57018A2D8E1957
:10705000811770F4F501049120E04D2D632FC201DA
:107060003983EADBFFEFAF1ABF0A3981385FEECF11
:10707000E60CF71CD394E6CFF201808901C080E0D2
:107080000F90DF91CF911F910F91FF90EF90DF90C4
:10709000CF90BF90AF909F907F906F905F904F90F8
:1070A00008950F931F93CF93DF9300D0CDB7DEB732
:1070B0008C01DC015596ED91FC9156972B834A8308
:1070C000698319954A81480F2B816981C8010F9006
:1070D0000F900F90DF91CF911F910F917BCFAF92C7
:1070E000BF92DF92EF92FF920F931F93CF93DF93A4
:1070F0001F921F92CDB7DEB77C01D62E042FDC0184
:107100005596ED91FC91569729833A831995080F6E
:107110002981A22E3A81B32E10E0F50121915F0161
:10712000222339F0402F6D2DC70154DFD80E180FE0
:10713000F4CF812F0F900F90DF91CF911F910F917E
:10714000FF90EF90DF90BF90AF900895DF92EF92A5
:10715000FF920F931F93CF93DF937C01D62FD42EF2
:107160008901DC015596ED91FC9156971995D80E41
:10717000C0E0F8012491222349F04D2D6D2FC70165
:1071800029DFD80FC80F0F5F1F4FF3CF8C2FDF9170
:10719000CF911F910F91FF90EF90DF900895DC0148
:1071A00014962D913C9115972115310509F43FC096
:1071B00057968C915797F901811108C03596E49143
:1071C0005896EC935897F9013C9611C0813041F4E0
:1071D0003F96E4915896EC935897F901709607C042
:1071E0003D96E4915896EC935897F9013E96E491B8
:1071F0005996EC93599758968C915897082E000CF5
:10720000990B59962C915997821B910927FD9395BB
:107210005A962C915A97203441F0829FC001112434
:1072200026E0969587952A95E1F75B968C930895CD
:1072300022E037E3FC01368B258B0895CF92DF9255
:10724000EF92FF920F931F93CF93DF938C017B01FB
:107250006A01CB01FA011995D82F882311F1682F03
:10726000C801E9DDF801C189C195FFEFEF1AFF0AF6
:10727000C701F6011995F801882351F08089C80FDC
:10728000C701F6011995D82F682FC801D4DDEDCFBD
:10729000D03221F091898389890F01C080898C0FB8
:1072A00001C080E0DF91CF911F910F91FF90EF908F
:1072B000DF90CF90089544E057E3C0CFCF93DF93A2
:1072C000FC01248135812617370741F0EC017583D5
:1072D000648365DF82E097E39E8B8D8BDF91CF9196
:1072E0000895CF93DF9300D01F92CDB7DEB761151D
:1072F00071058105910579F09B01AC0169833A83A1
:107300004B835C830F94CA5029813A814B815C8105
:107310000F941F5003C060E070E0CB010F900F90FE
:107320000F900F90DF91CF910895CF92DF92EF925F
:10733000FF920F931F9362177307840795077CF4DE
:1073400089019A016B017C01C901B8016C197D09A1
:107350008E099F09C6DF6C0D7D1D8E1D9F1D1F911F
:107360000F91FF90EF90DF90CF9008954F925F9232
:107370006F927F92AF92BF92CF92DF92EF92FF9285
:107380000F931F93CF93DF93CDB7DEB729013A0157
:107390009B01AC0124193509460957098A899B8943
:1073A000AC89BD89BC01CD016A197B098C099D0995
:1073B0000F94BB4FA80197012419350946095709B5
:1073C0000F941F50CA01B9016A0D7B1D8C1D9D1DB4
:1073D000DF91CF911F910F91FF90EF90DF90CF90B1
:1073E000BF90AF907F906F905F904F90089580E036
:1073F00090E008950895CF92DF92EF92FF920F935D
:107400001F93CF93DF936C017A018B01C0E0D0E032
:10741000CE15DF0589F0D8016D918D01D601ED9172
:10742000FC910190F081E02DC6011995892B11F492
:107430007E0102C02196ECCFC701DF91CF911F9151
:107440000F91FF90EF90DF90CF9008956115710537
:1074500079F0FB0101900020E9F73197AF01461B5D
:10746000570BDC01ED91FC910280F381E02D199422
:1074700080E090E00895EACFDC01ED91FC9101906D
:10748000F081E02D19944F925F926F927F92EF926C
:10749000FF920F931F93CF93DF93CDB7DEB7A197E2
:1074A0000FB6F894DEBF0FBECDBF7C01FA01CB0151
:1074B00019A2223008F42AE08E010F5D1F4F422EE0
:1074C000512C612C712CBF01A30192010F94FD4F2F
:1074D000F901CA01015011096A3014F4605D01C05C
:1074E000695CD8016C93232B242B252B61F7B80101
:1074F000C701ACDFA1960FB6F894DEBF0FBECDBFBB
:10750000DF91CF911F910F91FF90EF907F906F903F
:107510005F904F900895CF92DF92EF92FF920F937A
:107520001F93CF93DF93EC016A017B012115310595
:1075300079F4E881F9810190F081E02D642FDF91E9
:10754000CF911F910F91FF90EF90DF90CF90199402
:107550002A303105D9F477FF18C06DE28DDF8C0138
:1075600044275527BA014C195D096E097F092AE0A5
:10757000CE0189DF800F911FDF91CF911F910F9175
:10758000FF90EF90DF90CF9008952AE0B701A60119
:10759000CE01DF91CF911F910F91FF90EF90DF907F
:1075A000CF9071CF9A01AB01770F660B770BB3CFFA
:1075B000CF93CFB7F8948091C703811127C0E6EC31
:1075C000F3E08491E0E8F3E09491E82FF0E0EE0F2F
:1075D000FF1FE55FFB4FA591B491EC91E92321F4E6
:1075E00061E085E30E94293161E085E30E94ED308E
:1075F0008CB580618CBD8CB580648CBD61E084E30A
:107600000E94ED3061E083E30E94ED308091C7037A
:107610008F5F8093C703CFBFCF910895CF92EF9232
:107620000F93FC0113AE14AE15AE0496C3D80F91A0
:10763000EF90CF9008958EBD00000DB407FEFDCFF2
:107640008EB5089580E090E0089508950E946E2F11
:10765000FCDF0F94234BC0E0D0E00F94B04B209799
:10766000E1F30E940000F9CFE9EEF3E083AF64AFED
:1076700008954AE050E0BC0189EE93E093CFEF9289
:10768000FF920F931F93CF93DF937A016F3F7105A2
:107690008105910509F040F489EE93E0EDDE8DEE71
:1076A00093E0C1DB90E014C0C0912404D091250484
:1076B0004D2F50E0EC2FF0E08B019C01BF018DEECF
:1076C00093E05CD6C80FC0932404D0932504992777
:1076D000DF91CF911F910F91FF90EF900895EF925E
:1076E000FF920F931F93CF93DF938B01C9EED3E0EB
:1076F000FBACECAC4E2D50E06F2D70E09C018DEE9C
:1077000093E094D6F80EFBAEECAE9927DF91CF91C3
:107710001F910F91FF90EF900895EF92FF920F93BA
:107720001F93CF93DF938B01C9EED3E0FBACECAC9E
:107730004E2D50E06F2D70E09C018DEE93E0C2D68F
:10774000F80EFBAEECAE9927DF91CF911F910F9110
:10775000FF90EF9008956FEF7FEFC1CFCF93DF934E
:10776000EA0182DFCE01DF91CF91F5CF4FEF5FEFDE
:1077700086CFCF93DF9300D01F92CDB7DEB729839A
:107780003A834B835C8370DF29813A814B815C8132
:10779000CA01B9010F900F900F900F90DF91CF9118
:1077A000E5CF0F931F93CF93DF931F92CDB7DEB733
:1077B000082F87E296E00E947A7F182F863168F4BE
:1077C00087E296E0C8DF153109F43DC060E270E061
:1077D00080E090E0CBDF1F5FF6CFCE0101960E94E4
:1077E0001C8360E870E07BDF8981853120F56EE2E3
:1077F00070E080E090E0BADF19811431E1F06EE2D0
:1078000070E080E090E0B2DF1331A9F089812EEFC3
:107810003FEF281B310986E0829FB001839F700DE6
:10782000112460587F4F87E296E059DF60E270E0F4
:1078300080E090E09BDF8091C803801721F00093E7
:10784000C8030E94FE820F90DF91CF911F910F918C
:1078500008954F925F926F927F928F929F92AF9214
:10786000BF92CF92DF92EF92FF920F931F93CF932D
:10787000DF93CDB7DEB72D970FB6F894DEBF0FBEFE
:10788000CDBF80911D06882309F48AC06091970CB2
:107890007091980C072E000C880B990B0F94554D86
:1078A00011E02091930C3091940C4091950C5091E3
:1078B000960C0F94B64E18160CF010E060916E0CFA
:1078C00070916F0C072E000C880B990B0F94554D7F
:1078D00020916A0C30916B0C40916C0C50916D0CA6
:1078E0000F94B64E18160CF410681093DB038090BA
:1078F0006B0290906C02A0906D02B0906E0220E03E
:1079000030E0A901C501B4010F94B34C87FD05C057
:1079100020E030E040E05FE304C020E030E040E001
:107920005FEBC501B4010F94DA4B0F94224DCB01EC
:107930000F949E40BC0186ED93E00F9445558090D6
:107940006F0290907002A0907102B090720220E0DD
:1079500030E0A901C501B4010F94B34C87FD05C007
:1079600020E030E040E05FE304C020E030E040E0B1
:107970005FEBC501B4010F94DA4B0F94224DCB019C
:107980000F949E40BC0181ED93E00F94455583E731
:1079900092E00F94AF45BC0189EC93E00F944555FC
:1079A0000E94B981182F81E055D62091DB0327FF73
:1079B00003C048E00CE002C042E102E080912104F3
:1079C00090E044977CF480912304841758F027FDBD
:1079D00036C18AE497E17C0123E060E58DEE93E017
:1079E0000E945634809121048431B8F4809123049C
:1079F000823098F0112309F425C180918D0C8823E1
:107A000009F420C18AEB96E17C0102E123E042E027
:107A100068E68DEE93E00E945634809121048C310B
:107A2000D0F59091DB038090930C9090940CA090F3
:107A3000950CB090960CC090970CD090980C843117
:107A400028F480912304883008F035C28091210405
:107A5000883008F410C2809121048C3108F412C2DD
:107A600080906A0C90906B0CA0906C0CB0906D0C98
:107A700060916E0C70916F0C80912104883008F435
:107A800007C2809121048C3108F409C2809121043D
:107A90008C3108F40AC28091010983FF27C08091CC
:107AA0003107882319F1809121048433F8F48091FF
:107AB00023048A32D8F007E028E04AE26AE28DEE39
:107AC00093E06CD905E022E04CE262E38DEE93E0B6
:107AD00065D904E02AE041E36AE28DEE93E00ED935
:107AE0004BE262E38DEE93E00E9415348091210415
:107AF000853328F480912304813308F0A6C00E94C6
:107B0000D686823048F090912104943328F49091E5
:107B10002304923308F0A1C0809121048F3208F031
:107B20005DC080912304883208F458C00F946447E4
:107B30002B013C018CE3882E912CA12CB12CC3018C
:107B4000B201A50194010F94FD4FCA01B901A5012D
:107B500094010F94FD4FCA01D62EC72E4901AE01E4
:107B60004F5F5F4F5A0150E8451651E5550651E009
:107B70006506710408F48BC0B90128E130E040E0EB
:107B800050E00F94FD4F29013A01CF92DF92C401DA
:107B900068E170E00F94D64F9F938F935F924F925E
:107BA0008CEA96E19F938F93BF92AF920F94745596
:107BB0000FB6F894DEBF0FBECDBF5AE04516510494
:107BC0006104710408F08DC098E0892F880F980F28
:107BD000892F8195A5016FE2855AC0DD809121042E
:107BE0008632A0F4809123048E3180F008E020E8F2
:107BF0004EE160E08DEE93E0D1D880912104863291
:107C000028F4809123048F3108F06DC08091210405
:107C1000823328F4809123048B3208F011C18091C3
:107C20002104813408F030C280912304873308F4A2
:107C30002BC26EE380E018DD812FB3DD25C286E222
:107C400097E1C9CE80EF96E1DFCE04E02AE441E37C
:107C500066E38DEE93E052D852CFF8E48F9FB001E7
:107C60001124072E000C880B990B0F94554D2AE018
:107C700037ED43E25CE30F94F14E0F94274D262F2E
:107C800002E042E367E38DEE93E088D845CF84E6D7
:107C90008816910498F4CF92DF923F932F9382EA53
:107CA00096E19F938F93BF92AF920F9474550FB646
:107CB000F894DEBF0FBECDBF95E087CFCF92DF92A5
:107CC0003F932F938AE996E19F938F93BF92AF9250
:107CD0000F9474550FB6F894DEBF0FBECDBF96E07B
:107CE00074CF99E072CF60E08DEE93E00E942C3467
:107CF00028E530E040E050E065E283E03ADD65E20F
:107D00008BE0B2DC112321F086ED93E024DD24C06A
:107D100080914B0D80FD17C036EDC32E33E0D32E7E
:107D2000F60161916F016623B9F06F3234F4062ECB
:107D3000000C770B880B990B04C06FE370E080E0B8
:107D400090E014DDEDCF80914A0D80FDDDCF6FEF27
:107D50007FEF8DE896E1E1DC29E530E040E050E09E
:107D600065E288E206DD65E280E37EDC112321F036
:107D700081ED93E0F0DC26C080914B0D869580FD6F
:107D800017C021EDC22E23E0D22EF60161916F01C2
:107D90006623C1F06F3234F4062E000C770B880B8B
:107DA000990B04C06FE370E080E090E0DFDCEDCF82
:107DB00080914A0D869580FDDBCF6FEF7FEF8DE8D8
:107DC00096E1ABDC2AE530E040E050E065E28DE48E
:107DD000D0DC65E285E548DC112321F089EC93E0F5
:107DE000BADC28C080914B0D8695869580FD17C022
:107DF00099ECC92E93E0D92EF60161916F016623AB
:107E0000C9F06F3234F4062E000C770B880B990BF7
:107E100004C06FE370E080E090E0A8DCEDCF8091DB
:107E20004A0D8695869580FDD9CF6FEF7FEF82E969
:107E300096E173DC61E08DEE93E00E942C34E6CE97
:107E400083E008D426E030E040E050E062E383E0E5
:107E500090DC81E0FFD380916502909166020F94DF
:107E60006840AC0162E38CE079DC65E270E080E0C0
:107E700090E07CDCD4CE8091810C11112DC0811159
:107E8000EACD2AC080912304853108F056C0E8CDA0
:107E900080915D0C11117EC08111F3CD7BC080916A
:107EA0002304853108F0A7C0F1CD809123048531EA
:107EB00008F0CEC0F0CD90FD03C080E597E102C090
:107EC00088E697E17C010CE022E048E068E08DEE76
:107ED00093E00E945634BACDB601DD0C880B990BA5
:107EE0000F94554D20E030E040E05FE30F94DA4B13
:107EF0000F94224DCB010F946840FC0180818032A9
:107F0000D1F48181803211F491E001C092E043E02C
:107F100050E0491B51094E0F5F1F892F880F980FA2
:107F2000892F819567E0815F19DC69E070E080E06E
:107F300090E01CDC90CD93E0EACF20E030E040E020
:107F40005FE3C501B4010F94DA4B0F94224DCB01CE
:107F50000F946840FC0180818032D1F481818032AD
:107F600011F491E001C092E043E050E0491B510957
:107F70004E0F5F1F892F880F980F892F81956CE115
:107F8000815FECDB69E070E080E090E0EFDB68CDE2
:107F900093E0EACF072E000C880B990B0F94554DF8
:107FA00020E030E040E05FE30F94DA4B0F94224D85
:107FB000CB010F946840FC0180818032D1F4818133
:107FC000803211F491E001C092E043E050E0491B9F
:107FD00051094E0F5F1F892F880F980F892F8195A8
:107FE00067E0865ABBDB69E070E080E090E0BEDBD2
:107FF00048CD93E0EACF20E030E040E05FE3C50108
:10800000B4010F94DA4B0F94224DCB010F946840CA
:10801000FC0180818032D1F48181803211F491E0C1
:1080200001C092E043E050E0491B51094E0F5F1F31
:10803000892F880F980F892F81956CE1865A8EDBE6
:1080400069E070E080E090E091DB20CD93E0EACF42
:1080500080918D0C882309F41ECD24E6829FC001F7
:10806000112481589F4F6FEF70E00F94EA4FCB01BE
:108070000F946840AC016CE187E670DB65E270E06C
:1080800080E090E073DB07CD2D960FB6F894DEBF4D
:108090000FBECDBFDF91CF911F910F91FF90EF9059
:1080A000DF90CF90BF90AF909F908F907F906F9018
:1080B0005F904F9008950F931F93CF93DF93CDB7A9
:1080C000DEB728970FB6F894DEBF0FBECDBF8A018A
:1080D00023E0660F771F2A95E1F7680F791F48E0C4
:1080E00050E0CE0101960F94A85429813A81F801FD
:1080F000808191812817390790F08217930760F0EB
:108100009C818281981758F081E090E03B81238127
:10811000231738F080E005C081E090E002C08FEFC7
:108120009FEF28960FB6F894DEBF0FBECDBFDF914C
:10813000CF911F910F910895EF92FF920F931F938C
:10814000CF93DF93EC018B017A018A859B8586179B
:10815000970729F088819981B1D81B870A8788857C
:108160009985019681F00E811F81B70188819981DF
:10817000A2D8080F111D888599858017910718F4DA
:1081800081E090E011C06E818A81680F97014C8177
:10819000888199810E946F382E813F81280F311D7F
:1081A0003F832E8380E090E0DF91CF911F910F916C
:1081B000FF90EF9008954F925F926F927F928F920F
:1081C0009F92AF92BF92CF92DF92EF92FF920F9366
:1081D0001F93CF93DF93CDB7DEB72D970FB6F894EB
:1081E000DEBF0FBECDBF6C012A013B014901580122
:1081F0001B861C86CE0101967C0188E0F701119256
:108200008A95E9F7DB01CA0127E0B695A79597950E
:1082100087952A95D1F79A838983F42FFF77FD8775
:108220008F2F80588B838C831A8619864F3F510578
:108230006105710509F018F460E070E026C06091F6
:10824000DE037091DF038E01075F1F4F97014BE53F
:1082500050E48091DC039091DD030E94CB7D97FD7B
:10826000EBCF69857A8583E0660F771F8A95E1F702
:108270008091DC039091DD03680F791F48E050E0A6
:10828000C7010F94A8546F8178856115710519F4A1
:108290004B86B60106C0C616D70619F08D858068D4
:1082A0008B87AE01455F5F4FC401F50119952D968F
:1082B0000FB6F894DEBF0FBECDBFDF91CF911F91F7
:1082C0000F91FF90EF90DF90CF90BF90AF909F9075
:1082D0008F907F906F905F904F9008956F927F92F4
:1082E0008F929F92AF92BF92CF92DF92EF92FF92C6
:1082F0000F931F93CF93DF9300D01F92CDB7DEB7BC
:108300006C017B013A015901480119821A821B82D2
:108310001C82AE014F5F5F4FB301C7010E942B7EED
:108320007C0149815A816B817C8141155105610530
:10833000710529F084019501C6013DDFE6CF0F905C
:108340000F900F900F90DF91CF911F910F91FF90A1
:10835000EF90DF90CF90BF90AF909F908F907F90E5
:108360006F90089521E02093E003ECEDF3E091831A
:1083700080837383628380E090E008957F92AF9260
:10838000BF92CF92DF92EF92FF920F931F93CF9302
:10839000DF93CDB7DEB72C970FB6F894DEBF0FBED4
:1083A000CDBF6C01762EF72F842FE52FB901A801E0
:1083B000D6011496AD90BC9015979091E003911161
:1083C0000AC020EC37E1482F672DC6010E94A6386D
:1083D00080E090E019C0DA82C9827B82FC838D83C1
:1083E000EE8318861F82FA86E9861C861B860CE9B6
:1083F00010E49E012F5F3F4FC501DDDEB501C601D0
:108400000E945E398F8198852C960FB6F894DEBF56
:108410000FBECDBFDF91CF911F910F91FF90EF90D5
:10842000DF90CF90BF90AF907F900895CF92DF9272
:10843000EF92FF920F931F93CF93DF93CDB7DEB7E9
:108440002C970FB6F894DEBF0FBECDBF7C01C901DB
:10845000F701C480D5802091E003211108C020EAF3
:1084600037E1C7010E94A63880E090E01CC0FA8284
:10847000E9826B837C834D835E8318861F821A8713
:1084800009871C861B860CE910E49E012F5F3F4F75
:1084900045EC5DE7BC01C60121DFB601C7010E94C2
:1084A0005E398F8198852C960FB6F894DEBF0FBE8B
:1084B000CDBFDF91CF911F910F91FF90EF90DF9093
:1084C000CF900895CF92DF92EF92FF920F931F9378
:1084D000CF93DF93CDB7DEB72C970FB6F894DEBFFE
:1084E0000FBECDBF7C01C901F701C480D5802091AA
:1084F000E003211108C020E837E1C7010E94A63837
:1085000080E090E01CC0FA82E9826B837C834D831B
:108510005E8318861F821A8709871C861B860CE9D2
:1085200010E49E012F5F3F4F48EC5DE7BC01C601A0
:10853000D5DEB601C7010E945E398F8198852C96E1
:108540000FB6F894DEBF0FBECDBFDF91CF911F9164
:108550000F91FF90EF90DF90CF900895CF93DF932E
:10856000EC01262F4CAD6BAD04960E9451382BAD1B
:10857000082E000C990B820F911D8BAF81E090E0CB
:10858000DF91CF9108950F939CE0899F802D112456
:1085900021E0280F2093E803845F8093E70390E0B5
:1085A00002964091210450E08417950714F480E06E
:1085B00033C0822F90E02091230430E0821793078C
:1085C000B4F76623A9F061E08DEE93E00E942C34AD
:1085D0004091E8034E5F0BE020E860E08DEE93E011
:1085E0000E94CE3660E08DEE93E00E942C3405C0F0
:1085F00061E08DEE93E00E942C346091E70380915E
:1086000021046817A0F29091E80380912304891750
:1086100070F280E029D881E00F910895CF93DF9325
:10862000FC0185ADEF012496811105C081E085AF85
:10863000CE010E94CC33CE01DF91CF910C94033454
:10864000CF93DF93EA0110D86FEF7FEFCE01DF9178
:10865000CF9163C8482F50E02091E603022E000C12
:10866000330B4217530781F08093E603813031F4D6
:108670006BE77EE18DEE93E00C945E3969EC78E176
:108680008DEE93E00C945E39089581E0089589EEB3
:1086900093E0C4DF80E00E9495A08DEE93E00E94FD
:1086A00007348111F7CF64EC79E080E090E00C941E
:1086B000EDA0EF92FF920F9380912604811107C0E5
:1086C00081E0809326048DEE93E00E94CC338DEE02
:1086D00093E00E94033486EFE82E8DE1F82E03E14B
:1086E00027E047E064E28DEE93E00E94563483E099
:1086F000B1DF40E158E16BE285E2A2DF4CEF57E1E8
:1087000067E387E09DDF8DEE93E00E9407348111DF
:10871000E2CF0F91FF90EF90089581E0CADF64EC03
:1087200079E080E090E00C94EDA0B1DFF6CF60E05E
:1087300070E08BE79EE116CE1F93CF93DF93C0913D
:10874000EE03C695C69589EE93E068DFDC2FDD0F5A
:108750001D2F1C0F83E07EDF6C2F80E00E94343BD6
:1087600087E296E00E94AB3B4DEE57E16D2F80E033
:1087700067DF40EE57E1612F80E062DF8DEE93E02E
:108780000E9407348111E6CFDF91CF911F910895A8
:108790000895CF93E62F6CE0869F602D112481E031
:1087A000860F8093E803645F6093E703462F50E0F1
:1087B0004E5F5F4F2091210430E0421753070CF4C5
:1087C0004CC090E02091230430E0821793070CF016
:1087D00044C0CE2F8EE30E94343B65E470E080E01D
:1087E00090E00E94B63B61E36C0F062E000C770B05
:1087F000880B990B0E94B63B60E270E080E090E04D
:108800000E94B63B6091930C7091940C8091950CF2
:108810009091960C0F94224DCB010F9468400E94CA
:10882000AB3B6FE270E080E090E00E94B63B0E94BC
:10883000B981811109C085E0C89FF0011124E35876
:10884000F34F8481811109C08091970C9091980C0D
:108850000F946840CF910C94AB3BCF910895CF9289
:10886000DF92EF92FF920F931F93CF93DF931F92AC
:108870001F92CDB7DEB77B01622F498384DE498129
:10888000882309F444C0442311F101151105F9F4BA
:10889000C7010E949B7F25E130E0281B310937FF8B
:1088A00002C02F5F3F4F3595279530E82158822F22
:1088B000830F87FD0DC060E270E080E090E02A83C6
:1088C00039830E94B63B398131502A81F0CF30E89C
:1088D000C32ED12CB601C7010E948D3B7601E81A48
:1088E000F90A0115110511F41E2D07C0FF24B70167
:1088F000C8010E946F3B1E2D181B173040F060E22C
:1089000070E080E090E00E94B63B181BF6CF0F901D
:108910000F90DF91CF911F910F91FF90EF90DF901B
:10892000CF9008950F93CF93DF93982F862FEA016E
:10893000692F29DE882331F162E770E0CE010E94C1
:108940008D3BC2E7C81BC73040F060E270E080E0BA
:1089500090E00E94B63BC81BF6CF6091E7038AE720
:108960000E94343B602F000F770B880B990B0E94FD
:10897000B63B60E270E080E090E0DF91CF910F9134
:108980000C94B63BDF91CF910F910895CF92DF9277
:10899000EF92FF920F931F93CF93DF93982F862F21
:1089A0006A017901692FEFDD882309F44BC0C70103
:1089B000002321F00E949B7F182F03C00E947A7F22
:1089C000182FC3E1D0E0C11BD1098C2F880FC80F2D
:1089D000CC0FD0E0BE01C6010E948D3BC81B6AE3EC
:1089E00070E080E090E00E94B63BC73040F060E26B
:1089F00070E080E090E00E94B63BC81BF6CF8AEFA3
:108A0000189F802D11246091E70380580E94343B09
:108A1000002369F06FEF7FEFC701DF91CF911F91C6
:108A20000F91FF90EF90DF90CF900C948D3BC7019A
:108A3000DF91CF911F910F91FF90EF90DF90CF903A
:108A40000C94AB3BDF91CF911F910F91FF90EF9072
:108A5000DF90CF900895BF92CF92DF92EF92FF9276
:108A60000F931F93CF93DF936C017B010E949B7F39
:108A7000C82FC7010E947A7F03E110E0081B11098B
:108A80008C2F90E0BB24B394081719071CF0B12C6D
:108A9000C5E201C0CFE12C2F30E0A9014E5F5F4F4E
:108AA0008091210490E04817590744F0295031097A
:108AB0006091230470E062177307BCF5D0E0E11405
:108AC000F104C9F16AE370E080E090E00E94B63BF7
:108AD000BB2081F0C45F80912104C81760F12C2F66
:108AE00030E0295031098091230490E082179307E8
:108AF0001CF421C0DD23F9F0802F880F800F6C2F2C
:108B0000880F0E94343B60E270E080E090E00E94B9
:108B1000B63BC701DF91CF911F910F91FF90EF906E
:108B2000DF90CF90BF900C94AB3BA6016C2F80E000
:108B300087DDD1E0C4CFDF91CF911F910F91FF90DE
:108B4000EF90DF90CF90BF900895CF92DF92EF9299
:108B5000FF920F931F93CF93DF931F92CDB7DEB792
:108B6000182F7A01D22ECA0169830E949B7F082F99
:108B7000812F880F810FC82ECC0C1CE06981169FB5
:108B8000100D1124DD20C1F061E08DEE93E00E9414
:108B90002C34202F220F200F220F2E5F0BE047EFE7
:108BA000410F6FEF6C0D8DEE93E00E94CE3660E0CA
:108BB0008DEE93E00E942C34A701612F8C2D40DDB7
:108BC000DD2071F061E08DEE93E00F90DF91CF91A9
:108BD0001F910F91FF90EF90DF90CF900C942C3469
:108BE0000F90DF91CF911F910F91FF90EF90DF9049
:108BF000CF900895AF92BF92DF92EF92FF920F93C2
:108C00001F93CF93DF93EC015B01D42EC901B80110
:108C1000A7010E944A8191E02D2D2927A50164E03A
:108C200081E093DFCE010E949B7F2D2DAE0164E099
:108C300094E1981B892FDF91CF911F910F91FF90A5
:108C4000EF90DF90BF90AF9080CFEF92FF920F93A5
:108C5000CF93DF93D82FC62F7901682F8C2F93DC09
:108C60008823F1F0002331F062E070E080E090E0D2
:108C70000E94B63B2D2F4C2F64E1C7010E94268035
:108C800068E770E00E946F3BC8E7C81BC73040F040
:108C900060E270E080E090E00E94B63BC81BF6CF37
:108CA000DF91CF910F91FF90EF9008958F929F9257
:108CB000AF92BF92CF92DF92EF92FF920F936B0130
:108CC0007C018090E2039090E303A090E403B090D5
:108CD000E503A50194010F94B34C882301F120E032
:108CE00030E0A901C701B6010F94B34C882351F0BD
:108CF000A5019401C701B6010F94B34C87FD04C0D0
:108D000081E003C080E001C08FEF8093E103C09257
:108D1000E203D092E303E092E403F092E503809152
:108D20002104813128F480912304833008F048C065
:108D300080912104853128F480912304843108F046
:108D40004FC0809121048F3308F057C080912304D5
:108D50008F3208F452C08091E10340E3481B8FE456
:108D6000E82E88E1F82E0DE022E06AE58DEE93E032
:108D70000E9456348091E10341E3481B95E3E92EBC
:108D800098E1F92E22E065E08DEE93E00E945634E2
:108D900029E6E22E28E1F22E00E123E04FE262E133
:108DA0008DEE93E00E94563439E9E32E38E1F32E3C
:108DB00023E04FE267E68DEE93E00E9456341DC03B
:108DC0008091E10344E0481B5AE1E52E58E1F52E7D
:108DD0000CE022E062E48DEE93E00E945634A8CFCE
:108DE00042E3E42E48E1F42E01E023E044E16CE3A9
:108DF0008DEE93E00E945634A4CF0F91FF90EF9038
:108E0000DF90CF90BF90AF909F908F900895CF92BA
:108E1000EF920F93CF93DF93C9EED3E01B821A82B8
:108E200081E393E099838883CC24CA94EE24EA9466
:108E300006E427E448E464E172E0CE010E940E3BC0
:108E40008DE393E099838883DF91CF910F91EF9029
:108E5000CF9008959091050194709093030187FD40
:108E600076C0A3989091050190959470909303011A
:108E700090910501947090930301982F990F86FDAE
:108E800072C0A3988091050180958470809303013E
:108E900080910501847080930301292F220F96FD94
:108EA00060C0A39880910501809584708093030130
:108EB00080910501847080930301922F990F26FD04
:108EC0004EC0A39880910501809584708093030122
:108ED00080910501847080930301292F220F96FD54
:108EE0003CC0A39880910501809584708093030114
:108EF00080910501847080930301922F990F26FDC4
:108F00002AC0A39880910501809584708093030105
:108F100080910501847080930301292F220F96FD13
:108F200018C0A398809105018095847080930301F7
:108F30008091050184708093030126FD16C0A398DB
:108F40008091050180958470809303010895A39A10
:108F500089CFA39AE7CFA39AD5CFA39AC3CFA39AD9
:108F6000B1CFA39A9FCFA39A8DCFA39A80910501E9
:108F7000809584708093030108952F923F925F92B1
:108F80007F929F92AF92BF92CF92DF92EF92FF9229
:108F90000F931F93CF93DF937C011B01942E6901E4
:108FA0008AE0481709F47BC0A5E14A134EC0DB01F3
:108FB0001296ED91FC9113971281C681D781A49AE4
:108FC00088E28A950000E9F700EE010F80E1582E53
:108FD000510E98E2792E88EF3DDF872D8A950000AB
:108FE000E9F7103208F046C0812F8077806832DFC1
:108FF000812F8295807F2EDF872D8A950000E9F7EB
:1090000080E828DF80E026DF872D8A950000E9F7D9
:109010008AEF20DF872D8A950000E9F75E01B0E135
:10902000AB0EB11C8881807F15DF89918295807F8E
:1090300011DFCA15DB05B1F7872D8A950000E9F726
:109040001F5F0F5F1511C7CFA4989601492DB1017D
:10905000C701DF91CF911F910F91FF90EF90DF90AB
:10906000CF90BF90AF909F907F905F903F902F9058
:109070000C949035802F80778068ECDE802F82956D
:10908000807FE8DE872D8A950000E9F780E8E2DE40
:1090900080E8E0DE872D8A950000E9F7B9CF9C9A39
:1090A000A4989B9AA3988091040184608093040102
:1090B000809105018095847080930301A49AC8E291
:1090C0008C2F8A950000E9F788E790E00E94AD3484
:1090D00088EFC0DE8C2F8A950000E9F780E2BADEC7
:1090E00080E0B8DE8C2F8A950000E9F780E0B2DEE0
:1090F00080E8B0DE8C2F8A950000E9F780E0AADED8
:1091000080E1A8DE8C2F8A950000E9F78FE090E0DF
:109110000E94AD3480E29EDE80E49CDE8C2F8A9536
:109120000000E9F780E296DE80E694DECA95000052
:10913000E9F710E0D8E208E2812F807780688ADEC4
:10914000812F8295807F86DE8D2F8A950000E9F73A
:1091500080E880DE80E07EDE8D2F8A950000E9F7D2
:109160008AEF78DE8D2F8A950000E9F7C0E280E073
:1091700071DE80E06FDE9D2F9A950000E9F7C15007
:10918000B1F788EF67DE802F8A950000E9F71F5F4F
:10919000103209F0D1CF80E05DDE80EC5BDE88E24A
:1091A0008A950000E9F7A49850CFCF93DF931F92E0
:1091B0001F92CDB7DEB789839A830E94917A20E00F
:1091C00040E060E070E089819A810F900F90DF911C
:1091D000CF910C94447B0F93CF93DF9361E081E0B8
:1091E0000E945D7CD091F505C0E0D11117C080913F
:1091F000F405811104C00E947080811165C08091C6
:109200002202882309F457C081E09091F40591115E
:1092100080E004E024E04FE857E24BC0D130C1F4D5
:109220008091F405813021F40E947080811155C035
:1092300080912202882309F43EC081E09091F405D8
:10924000913009F080E003E02EE346E857E231C0B8
:10925000D230B9F48091F405823021F40E947080FC
:10926000811144C080912202882329F181E09091EC
:10927000F405923009F080E003E02EE34DE757E279
:1092800018C0D330C1F48091F405833021F40E94DA
:109290007080811134C080912202882361F081E0C6
:1092A0009091F405933009F080E003E02EE347E766
:1092B00057E26C2F37DBCF5FDF5FC53009F095CF0A
:1092C00084E08093F30522C081E00E94777B809147
:1092D000C105882309F493CF19C084E690E765DFC0
:1092E0008091C105882309F4A3CF10C086E895E7D3
:1092F0005CDF8091C105882309F4B4CF07C08EE9F3
:1093000099E753DF8091C105882329F2DF91CF913E
:109310000F910895CF93DF93EC01CB01BA010F9425
:10932000554D23E333E343E250E40F94F14E0F94A1
:10933000274D6883DF91CF910895CF93DF93EC01A0
:10934000CB01BA010F94554D2FE632E143E85AE3C1
:109350000F94F14E688379838A839B83DF91CF9149
:1093600008956AE879E48DEB99E40C949B7B6DE9B0
:1093700079E480EE99E40C949B7B0F94554D23E3A4
:1093800033E343E250E40F94F14E0F94274D862FC0
:109390000D94BD3FCF93DF9300D01F92CDB7DEB7C2
:1093A00069837A838B839C8360E2CE0101960F945C
:1093B000E1420F900F900F900F90DF91CF910895A1
:1093C0000F94554D2FE632E143E85AE30F94F14EE6
:1093D000E1CF2F923F924F925F926F927F928F9246
:1093E0009F92AF92BF92CF92DF92EF92FF920F9334
:1093F0001F93CF93DF93CDB7DEB729970FB6F894BD
:10940000DEBF0FBECDBF1C0179876887CA01B901D5
:10941000E982FA820B831C83DE82CD82AF8220E058
:1094200030E04AE754E40F94F14E6B017C0120E0F8
:1094300030E040E057EC0F94B64E18162CF0C12CDB
:10944000D12CE12C27ECF22EC701B6010F94224D4E
:109450002B013C0120E030E04AE754E469817A8145
:109460008B819C810F94F14E4B015C0120E03EEF1B
:109470004FEF56E40F94B34C87FD07C0812C9EEF4D
:10948000992EAA24AA9496E4B92E20E030E04AE767
:1094900054E4E885F98560817181828193810F941C
:1094A000F14E6B017C01C301B2010F94554D9B013C
:1094B000AC01C701B6010F94D94B0F94274D6983B6
:1094C0007A838B839C83C501B4010F94224D7B0169
:1094D0008C01E418F50806091709FF81FF938D80B8
:1094E0009E8087EBA82E89E4B82EC980DA80A3017C
:1094F000920168857985C1010E94B87A0F902996FA
:109500000FB6F894DEBF0FBECDBFDF91CF911F9194
:109510000F91FF90EF90DF90CF90BF90AF909F9012
:109520008F907F906F905F904F903F902F90089515
:109530008F929F92AF92BF92CF92DF92EF92FF9263
:109540000F931F93CF93DF9361E081E00E945D7CD6
:10955000D091F505C0E0D11119C08091F4058111B9
:1095600004C00E9470808111C4C0809122028823AF
:1095700009F4B6C081E09091F405911180E004E017
:1095800024E04AEC57E26C2FCDD9AAC0D130E1F4E7
:109590008091F405813021F40E9470808111B2C065
:1095A00080912202882309F49BC011E08091F40588
:1095B000813009F010E08091050C0F94BD3F00E070
:1095C0009C0144EB57E289C0D23009F58091F40543
:1095D000823021F40E9470808111C3C080912202E8
:1095E000882309F47DC011E08091F405823009F0F0
:1095F00010E06091060C7091070C8091080C90911E
:10960000090CC8DE00E09C0140EB57E266C0D33095
:1096100009F58091F405833021F40E947080811156
:10962000B9C080912202882309F45AC011E08091C8
:10963000F405833009F010E060910A0C70910B0C76
:1096400080910C0C90910D0CA5DE00E09C014CEA81
:1096500057E243C0D43001F58091F405843021F401
:109660000E9470808111AFC0809122028823C1F1D5
:1096700011E08091F405843009F010E060910E0C47
:1096800070910F0C8091100C9091110C83DE00E012
:109690009C0148EA57E221C0D53011F58091F405CC
:1096A000853021F40E9470808111A6C08091220231
:1096B0008823B1F011E08091F405853009F010E0C5
:1096C000609128027091290280912A0290912B02C8
:1096D00061DE00E09C0144E957E26C2F812F56D9EE
:1096E000CF5FDF5FC53009F036CF86E08093F305AA
:1096F0009BC081E00E94777B8091C105882309F49B
:1097000034CF92C081E00E9465806091050C70E0CA
:1097100080E090E00F94534D29EC38EC48EC5EE388
:109720000F94F14E0F94274D1F92812C912C41EBF9
:10973000A42E49E4B42E6B0114E6E12EF12C00E0D6
:1097400010E020E030E0A90165E07CE08FEB97E2DB
:109750000E94B87A0F908091C105882309F420CF28
:1097600063C081E00E946580A12CC12CD12C16E63B
:10977000E12EFE2C0EE111E420E030E0A90166E0CC
:109780007CE082EB97E225DE8091C105882309F415
:1097900025CF4AC081E00E946580A12CC12CD12C2C
:1097A00016E6E12EFE2C0EE111E420E030E0A901E6
:1097B0006AE07CE08EEA97E20CDE8091C1058823A6
:1097C00009F42FCF31C081E00E946580A12CC12C0B
:1097D000D12C16E6E12EFE2C0EE111E420E030E063
:1097E000A9016EE07CE08AEA97E2F3DD8091C10591
:1097F000882309F439CF18C081E00E946580A12C2C
:10980000C12CD12C16E6E12EFE2C0EE111E420E055
:1098100030E0A90168E272E08EE997E2DADD80913A
:10982000C105882309F442CFDF91CF911F910F9199
:10983000FF90EF90DF90CF90BF90AF909F908F9070
:109840000895CF93DF93EC01CB01BA010F94554DEE
:109850002AE037ED43E25CE30F94F14E68837983AD
:109860008A839B83DF91CF910895CF93DF93EC019F
:10987000CB01BA010F94554D688379838A839B830A
:10988000DF91CF910895CF93DF93EC01CB01BA0123
:109890000F94554D20E030E048EC51E40F94F14E28
:1098A000688379838A839B83DF91CF910895CF93D7
:1098B000DF93EC01CB01BA010F94554D6883798396
:1098C0008A839B83DF91CF910895CF93DF93EC013F
:1098D000CB01BA010F94554D20E030E048EC51E443
:1098E0000F94F14E0F94274D688379838A839B836D
:1098F000DF91CF910895CF93DF93EC01CB01BA01B3
:109900000F94554D20E030E048EC52E40F94F14EB6
:109910000F94274D688379838A839B83DF91CF914E
:109920000895CF93DF93EC01CB01BA010F94554D0D
:109930002AE037ED43E25CE30F94F14E68837983CC
:109940008A839B83DF91CF910895CF93DF93EC01BE
:10995000CB01BA010F94554D2DEC3CEC4CEC5DE382
:109960000F94F14E688379838A839B83DF91CF9133
:10997000089561E27CE48EE39DE40C949B7B65E3B7
:109980007CE48CEB9DE40C949B7B67E57CE48DEEA2
:109990009CE40C949B7B63E47CE48BE59DE40C9459
:1099A0009B7B65E67CE488ED9DE40C949B7B6BE7F8
:1099B0007CE488E79DE40C949B7B61E97CE484E093
:1099C0009DE40C949B7B65EA7CE481E29DE40C942D
:1099D0009B7B0D94CF030D941604CF93DF9300D09F
:1099E0001F92CDB7DEB70F94554D69837A838B8371
:1099F0009C83CE0101960F942A440F900F900F90F4
:109A00000F90DF91CF910895CF93DF9300D01F92F5
:109A1000CDB7DEB70F94554D2AE037ED43E25CE356
:109A20000F94F14E69837A838B839C83CE010196D8
:109A30000F945F440F900F900F900F90DF91CF9194
:109A40000895CF93DF9300D01F92CDB7DEB70F9468
:109A5000554D2DEC3CEC4CEC5DE30F94F14E6983DD
:109A60007A838B839C83CE0101960F94FF440F90E1
:109A70000F900F900F90DF91CF910895CF93DF93C8
:109A800000D01F92CDB7DEB70F94554D2AE037EDC9
:109A900043E25CE30F94F14E69837A838B839C836A
:109AA000CE0101960F94A3410F900F900F900F904D
:109AB000DF91CF910895CF93DF9300D01F92CDB760
:109AC000DEB70F94554D20E030E048EC51E40F94A0
:109AD000F14E69837A838B839C83CE0101960F9428
:109AE0002A440F900F900F900F90DF91CF9108951F
:109AF000CF93DF9300D01F92CDB7DEB70F94554DB3
:109B000020E030E048EC52E40F94F14E0F94274DE2
:109B10000F94534D69837A838B839C83CE01019686
:109B20000F942A440F900F900F900F90DF91CF91D8
:109B30000895CF92DF92EF92FF926B017C0120E0BB
:109B400030E0A9010F94B34C87FD05C020E030E060
:109B500040E05FE304C020E030E040E05FEBC7019D
:109B6000B6010F94DA4B0F94224DCB01FF90EF908A
:109B7000DF90CF900D9468400F94554DDACFCF937E
:109B8000DF9300D01F92CDB7DEB70F94274D0F940F
:109B9000534D69837A838B839C83CE0101960F9406
:109BA0002A440F900F900F900F90DF91CF9108955E
:109BB0000F94554D20E030E048EC51E40F94F14E05
:109BC000DECF81E00C94777B6F927F928F929F9291
:109BD000AF92BF92CF92DF92EF92FF920F931F93BB
:109BE000CF93DF9300D01F92CDB7DEB761E081E065
:109BF0000E945D7C6090F505712C61101AC0809107
:109C0000F405811104C00E947080811159C18091B6
:109C10002202882309F44BC181E09091F40591114F
:109C200080E004E024E04DE359E2672D0E94924475
:109C30003EC181E068122CC08091F405813021F48E
:109C40000E947080811143C180912202882309F40F
:109C50002EC111E08091F405813009F010E080916F
:109C6000330E9091340EA091350EB091360E89834B
:109C70009A83AB83BC83CE0101960F942A4400E003
:109C80009C0141E359E2672D812F0E94C6440FC118
:109C900082E068122CC08091F405823021F40E9489
:109CA000708081114CC180912202882309F4FFC089
:109CB00011E08091F405823009F010E08091370EB8
:109CC0009091380EA091390EB0913A0E89839A8303
:109CD000AB83BC83CE0101960F942A4400E09C0123
:109CE0004DE159E2672D812F0E94C644E0C083E018
:109CF00068122CC08091F405833021F40E9470809A
:109D000081114FC180912202882309F4D0C011E053
:109D10008091F405833009F010E080913B0E909122
:109D20003C0EA0913D0EB0913E0E89839A83AB8389
:109D3000BC83CE0101960F942A4400E09C014BE0C5
:109D400059E2672D812F0E94C644B1C084E0681299
:109D500027C08091F405843021F40E947080811125
:109D600058C180912202882309F4A1C011E080919A
:109D7000F405843009F010E06091FF0D7091000E41
:109D80008091010E9091020E0F94534DF8DE00E089
:109D90009C014DEF58E2672D812F0E94C64487C079
:109DA00085E0681227C08091F405853021F40E9477
:109DB000708081116AC180912202882309F477C0E2
:109DC00011E08091F405853009F010E06091030EF8
:109DD0007091040E8091050E9091060E0F94534DD4
:109DE000CEDE00E09C014FEE58E2672D812F0E94ED
:109DF000C6445DC086E0681227C08091F4058630B5
:109E000021F40E94708081117CC1809122028823FC
:109E100009F44DC011E08091F405863009F010E09E
:109E20006091070E7091080E8091090E90910A0EB4
:109E30000F94534DA4DE00E09C0141EE58E2672DE3
:109E4000812F0E94C64433C087E0681230C08091E1
:109E5000F405873021F40E947080811187C18091C0
:109E60002202882321F111E08091F405873009F066
:109E700010E060910B0E70910C0E80910D0E909180
:109E80000E0E0F94534D0F94274D0F94534D69832D
:109E90007A838B839C83CE0101960F942A4400E041
:109EA0009C0143ED58E2672D812F0E94C6447394B4
:109EB000639485E07812A1CE88E08093F30591C188
:109EC00080DE8091C105882309F4A1CE8AC181E09A
:109ED0000E9465802AE037ED43E25DE36091330E36
:109EE0007091340E8091350E9091360E0F94F14E94
:109EF00020E030E040E85FE30F94D94B0F94274D0A
:109F00001F92812C912C5BECA52E5CE4B52E6B018D
:109F100017E7E12E1FE0F12E00E010E021E030E035
:109F200040E050E063E37EE087E399E20E94B87A84
:109F30000F908091C105882309F486CE52C181E03B
:109F40000E94658020E030E048EC52E46091370EDA
:109F50007091380E8091390E90913A0E0F94D94B32
:109F60000F94274D1F92812C912C35ECA32E3CE4AD
:109F7000B32E6B011BE9E12E1FE7F12E00E010E08C
:109F800024E630E040E050E067E37EE087E299E2DB
:109F90000E94B87A0F908091C105882309F483CE7E
:109FA00020C181E00E9465802AE037ED43E25DE355
:109FB00060913B0E70913C0E80913D0E90913E0E53
:109FC0000F94F14E20E030E040E85FE30F94D94B6E
:109FD0000F94274D1F92812C912C9BECA92E9CE471
:109FE000B92E6B0117E7E12E1FE0F12E00E010E023
:109FF00021E030E040E050E06BE37EE084E199E274
:10A000000E94B87A0F908091C105882309F47ACE16
:10A01000E8C081E00E9465806091FF0D7091000EA4
:10A020008091010E9091020E0F94534D2AE037ED6E
:10A0300043E25DE30F94F14E20E030E040E850E46D
:10A040000F94D94B0F94274D1F92B9EE8B2EBCE481
:10A050009B2E11EDA12E1CE4B12E6B0114E7E12E15
:10A060001FE0F12E00E010E024E030E040E050E09E
:10A070006FEF7DE084E099E20E94B87A0F908091C2
:10A08000C105882309F46DCEACC081E00E946580D3
:10A090006091030E7091040E8091050E9091060E52
:10A0A0000F94534D2AE037ED43E25DE30F94F14EF8
:10A0B00020E030E040E850E40F94D94B0F94274D56
:10A0C0001F92E9EE8E2EECE49E2EF1EDAF2EFCE415
:10A0D000BF2E6B0114E7E12E1FE0F12E00E010E02F
:10A0E00024E030E040E050E063E07EE086EF98E27C
:10A0F0000E94B87A0F908091C105882309F45BCE45
:10A1000070C081E00E9465806091070E7091080E1A
:10A110008091090E90910A0E0F94534D2AE037ED6D
:10A1200043E25DE30F94F14E0F94274D1F9239EEF9
:10A13000832E3CE4932E41EDA42E4CE4B42E6B010F
:10A1400018E7E12E1FE0F12E00E010E020E030E003
:10A15000A90167E07EE088EE98E20E94B87A0F904D
:10A160008091C105882309F450CE3BC081E00E9454
:10A17000658060910B0E70910C0E80910D0E909188
:10A180000E0E0F94534D2AE037ED43E25CE30F943B
:10A19000F14E20E030E040E85FE30F94D94B0F949C
:10A1A000274D1F9289EE882E8CE4982E97EDA92ECC
:10A1B0009CE4B92E6B011DEDE12E13E0F12E00E0C1
:10A1C00010E021E030E040E050E06BE07EE08AED1E
:10A1D00098E20E94B87A0F908091C105882309F413
:10A1E0003ECE0F900F900F900F90DF91CF911F9167
:10A1F0000F91FF90EF90DF90CF90BF90AF909F9026
:10A200008F907F906F9008950F931F93CF93DF935C
:10A2100061E081E00E945D7CC091F505D0E0C11154
:10A220001AC08091F405811104C00E9470808111D0
:10A23000E8C080912202882309F461C081E09091F6
:10A24000F405911180E004E024E041E158E26D2F33
:10A250000E94924454C0C130D9F48091F4058130F9
:10A2600021F40E9470808111D3C080912202882342
:10A2700009F445C081E09091F405913009F080E047
:10A2800003E02EE348E058E26D2F0E94924437C06D
:10A29000C230D1F48091F405823021F40E947080A4
:10A2A0008111C0C080912202882349F181E0909100
:10A2B000F405923009F080E003E02EE34BEF57E223
:10A2C0006D2F0E9492441BC0C330C9F48091F405E5
:10A2D000833021F40E9470808111AEC080912202EF
:10A2E000882369F081E09091F405933009F080E0D3
:10A2F00003E02EE346EF57E26D2F0E9492440E9446
:10A300002D7B81111DC0C430E9F48091F4058430A7
:10A3100021F40E947080811199C0809122028823CB
:10A3200009F49EC081E09091F405943009F080E03A
:10A3300003E02EE34DEE57E26D2F0E94924490C051
:10A3400014E001C015E0C1131BC08091F4058C130B
:10A3500004C00E947080811185C0809122028823F0
:10A3600071F081E09091F4059C1380E003E02EE30E
:10A3700044EE57E26D2F0E9492441C2F01C01C2F07
:10A3800081E0810FC81318C08091F4058C1304C0BC
:10A390000E947080811170C080912202882361F038
:10A3A00081E09091F4059C1380E003E02EE348EDFA
:10A3B00057E26D2F0E94924482E0810FC81318C0AB
:10A3C0008091F4058C1304C00E94708081115EC0DE
:10A3D00080912202882361F081E09091F4059C1322
:10A3E00080E003E02EE34FEC57E26D2F0E94924491
:10A3F000DF5FCF5FD53009F012CF1D5F1093F305FB
:10A400004EC0DFDB8091C105882309F412CF47C01D
:10A4100080E795E50E94D5488091C105882309F41D
:10A4200024CF3DC084EE9DE40E94D5488091C105B3
:10A43000882309F437CF33C08EE397E50E94D548CF
:10A440008091C105882309F449CF29C082E799E5A5
:10A450000E94D5488091C105882309F45ECF1FC0B2
:10A4600015E08ECF88E99AE40E94D5488091C10515
:10A47000882309F472CF13C081E194E50E94D54886
:10A480008091C105882309F487CF09C08FED92E53B
:10A490000E94D5488091C105882309F499CFDF91A6
:10A4A000CF911F910F9108952F923F924F925F92FB
:10A4B0006F927F928F929F92AF92BF92CF92DF92D4
:10A4C000EF92FF920F931F93CF93DF9300D000D0B2
:10A4D000CDB7DEB71C017E836D8329013A014601A9
:10A4E00020E030E040E057ECB201C3010F94B64EDB
:10A4F00018162CF0412C512C612C27EC01C0272D73
:10A50000B201862D922F0F94224D2B013C0120E0A9
:10A510003EEF4FEF56E4B701C8010F94B34C87FDEF
:10A5200006C0B12C9EEFF92E0FEF16E401C0BE2C31
:10A53000C301B2010F94554D9B01AC01ED81FE8129
:10A5400060817181828193810F94D94B0F94274D43
:10A5500069837A838B839C836B2D7F2DC8010F9435
:10A56000224D7B018C01E418F50806091709AF920A
:10A570008FEBA82E8CE4B82EC980DA80A30192015B
:10A580006D817E81C1010E94B87A0F9026960FB628
:10A59000F894DEBF0FBECDBFDF91CF911F910F9119
:10A5A000FF90EF90DF90CF90BF90AF909F908F90F3
:10A5B0007F906F905F904F903F902F9008956F9293
:10A5C0007F928F929F92AF92BF92CF92DF92EF9243
:10A5D000FF920F931F93CF93DF9300D01F92CDB7BD
:10A5E000DEB761E081E00E945D7C6090F505712C32
:10A5F00061101AC08091F405811104C00E9470801E
:10A60000811198C080912202882309F48AC081E0D8
:10A610009091F405911180E004E024E046E45AE2D0
:10A62000672D0E9492447DC081E068122CC0809109
:10A63000F405813021F40E947080811182C08091E4
:10A640002202882309F46DC011E08091F405813065
:10A6500009F010E08091700D9091710DA091720D34
:10A66000B091730D89839A83AB83BC83CE0101962D
:10A670000F94A34100E09C0142E35AE2672D812F31
:10A680000E94C6444EC082E0681225C08091F40545
:10A69000823021F40E947080811181C08091220259
:10A6A000882309F43EC011E08091F405823009F05E
:10A6B00010E06091CF0B7091D00B8091D10B9091F5
:10A6C000D20B37DA00E09C014EE15AE2672D812F70
:10A6D0000E94C64426C083E0681223C08091F4051E
:10A6E000833021F40E947080811171C08091220218
:10A6F0008823B9F011E08091F405833009F010E06F
:10A700006091D30B7091D40B8091D50B9091D60BA7
:10A7100010DA00E09C014EE05AE2672D812F0E9482
:10A72000C6447394639485E0781262CF84E080938A
:10A73000F30564C046DA8091C105882309F462CF2D
:10A740005DC020E030E048EC52E46091700D709103
:10A75000710D8091720D9091730D0F94F14E0F94C5
:10A76000274D1F92812C912C29EBA22E2CE4B22E86
:10A770006B01EE24EA941FE7F12E00E010E020E0E8
:10A7800030E0A90160E77DE08CE39AE20E94B87AAC
:10A790000F908091C105882309F451CF2FC081E02B
:10A7A0000E946580A12CC12CD12CE12CF12C08E455
:10A7B00013E420E030E0A9016FEC7BE088E29AE24C
:10A7C00073DE8091C105882309F468CF17C081E04A
:10A7D0000E946580A12CC12CD12CE12CF12C08E425
:10A7E00013E420E030E0A90163ED7BE086E19AE22A
:10A7F0005BDE8091C105882309F478CF0F900F901C
:10A800000F900F90DF91CF911F910F91FF90EF90DC
:10A81000DF90CF90BF90AF909F908F907F906F9080
:10A8200008956F927F928F929F92AF92BF92CF9234
:10A83000DF92EF92FF920F931F93CF93DF9300D09D
:10A840001F92CDB7DEB761E081E00E945D7C609031
:10A85000F505712C61101AC08091F405811104C0B6
:10A860000E9470808111BDC080912202882309F46A
:10A87000B0C081E09091F405911180E004E024E003
:10A880004CEF59E2672D0E949244A3C081E0681208
:10A8900023C08091F405813021F40E9470808111E1
:10A8A000A7C080912202882309F493C080919D0D56
:10A8B000811103C02CEE39E202C020EF39E281E0C1
:10A8C0009091F405913009F080E001E043EE59E207
:10A8D000672D0E94C6447DC082E0681225C0809129
:10A8E000F405823021F40E94708081118FC0809124
:10A8F0002202882309F46DC011E08091F4058230B2
:10A9000009F010E060917F027091800280918102D5
:10A91000909182020ED900E09C0145ED59E2672D2D
:10A92000812F0E94C64455C083E0681225C08091E3
:10A93000F405833021F40E94708081117CC08091E5
:10A940002202882309F445C011E08091F405833088
:10A9500009F010E060918302709184028091850279
:10A9600090918602E6D800E09C0147EC59E2672D01
:10A97000812F0E94C6442DC084E068122AC08091B5
:10A98000F405843021F40E947080811169C08091A7
:10A9900022028823F1F011E08091F405843009F05F
:10A9A00010E080917B0290917C02A0917D02B09199
:10A9B0007E0289839A83AB83BC83CE0101960F9478
:10A9C000A34100E09C0147EB59E2672D812F0E94D3
:10A9D000C6447394639485E078123CCF7092F3057B
:10A9E0006CC0EFD88091C105882309F43DCF65C0C4
:10A9F00040E050E06DE97DE083EF99E20E941F7B2B
:10AA00008091C105882309F44CCF57C0A12CC12CDB
:10AA1000D12CE12CF12C01E913E420E030E0A90174
:10AA20006FE772E08CED99E23FDD8091C1058823EC
:10AA300009F45DCF42C0A12CC12CD12CE12CF12C0A
:10AA400001E913E420E030E0A90163E872E08EEC54
:10AA500099E22ADD8091C105882309F470CF2DC0C9
:10AA600020E030E048EC52E460917B0270917C027F
:10AA700080917D0290917E020F94F14E0F94274DAC
:10AA80001F92812C912C89EBA82E8CE4B82E6B019F
:10AA900018EEE12E13E0F12E00E010E020E030E0AF
:10AAA000A9016BE772E08FEB99E20E94B87A0F90F0
:10AAB0008091C105882309F46ACF0F900F900F9001
:10AAC0000F90DF91CF911F910F91FF90EF90DF904A
:10AAD000CF90BF90AF909F908F907F906F90089590
:10AAE000AF92CF92DF92EF92FF920F931F93CF938B
:10AAF000DF9361E081E00E945D7CD091F505C0E0CC
:10AB0000D1111AC08091F405811104C00E94708097
:10AB1000811109C180912202882309F4FBC081E0E0
:10AB20009091F405911180E004E024E045EA59E2B7
:10AB30006C2F0E949244EEC0D13031F58091F40523
:10AB4000813021F40E9470808111F5C08091220231
:10AB5000882309F4DFC011E08091F405813009F009
:10AB600010E06091230E7091240E8091250E90913B
:10AB7000260E0E94994D00E09C0147E959E26C2F96
:10AB8000812F0E94C644C6C0D23031F58091F405B1
:10AB9000823021F40E9470808111E7C080912202EE
:10ABA000882309F4B7C011E08091F405823009F0E0
:10ABB00010E06091270E7091280E8091290E9091DF
:10ABC0002A0E0E94994D00E09C0149E859E26C2F41
:10ABD000812F0E94C6449EC0D33031F58091F40588
:10ABE000833021F40E9470808111D9C080912202AB
:10ABF000882309F48FC011E08091F405833009F0B7
:10AC000010E060912B0E70912C0E80912D0E909182
:10AC10002E0E0E94994D00E09C014BE759E26C2FEB
:10AC2000812F0E94C64476C0D43031F58091F4055E
:10AC3000843021F40E9470808111CBC08091220267
:10AC4000882309F467C011E08091F405843009F08D
:10AC500010E060912F0E7091300E8091310E909126
:10AC6000320E0E94994D00E09C014DE659E26C2F96
:10AC7000812F0E94C6444EC0D53031F58091F40535
:10AC8000853021F40E9470808111BDC08091220224
:10AC9000882309F43FC011E08091F405853009F064
:10ACA00010E060913F0E7091400E8091410E9091A6
:10ACB000420E0E94994D00E09C0143E659E26C2F40
:10ACC000812F0E94C64426C0D63021F58091F4051C
:10ACD000863021F40E9470808111AEC080912202E2
:10ACE0008823C1F011E08091F405863009F010E06E
:10ACF0006091430E7091440E8091450E9091460EE6
:10AD00000E94994D00E09C014FE459E26C2F812F85
:10AD10000E94C644CF5FDF5FC53009F0F1CE87E007
:10AD20008093F305A1C00E94E14D8091C105882365
:10AD300009F4F0CE99C081E00E946580A12CC12C5D
:10AD4000D12CE12C10ECF12E09E714E420E030E0E6
:10AD500040E85FE363E27EE08EE999E2A5DB809163
:10AD6000C105882309F4F2CE7FC081E00E9465808E
:10AD7000A12CC12CD12CE12C10ECF12E09E714E40C
:10AD800020E030E040E85FE367E27EE080E999E2BE
:10AD90008BDB8091C105882309F400CF65C081E079
:10ADA0000E946580A12CC12CD12CE12C10ECF12E3D
:10ADB00009E714E420E030E040E85FE36BE27EE086
:10ADC00082E899E271DB8091C105882309F40ECFF6
:10ADD0004BC081E00E946580A12CC12CD12CE12CBC
:10ADE00010ECF12E09E714E420E030E040E85FE3E6
:10ADF0006FE27EE084E799E257DB8091C10588230A
:10AE000009F41CCF31C081E00E946580A12CC12CC7
:10AE1000D12CE12C10ECF12E09E714E420E030E015
:10AE2000A9016FE37EE088E699E23EDB8091C105EF
:10AE3000882309F42BCF18C081E00E946580A12CE3
:10AE4000C12CD12CE12C10ECF12E09E714E420E008
:10AE500030E0A90163E47EE089E599E225DB809199
:10AE6000C105882309F43ACFDF91CF911F910F914B
:10AE7000FF90EF90DF90CF90AF9008956F927F9208
:10AE80008F929F92AF92BF92CF92DF92EF92FF92FA
:10AE90000F931F93CF93DF9300D01F92CDB7DEB7F0
:10AEA00061E081E00E945D7C6090F505712C61108D
:10AEB0001AC08091F405811104C00E947080811134
:10AEC000C2C080912202882309F4B5C081E090912C
:10AED000F405911180E004E024E041EC58E2672D94
:10AEE0000E949244A8C081E0681226C08091F405B7
:10AEF000813021F40E9470808111ADC080912202C6
:10AF0000882309F498C011E08091F405813009F09C
:10AF100010E06091CF0D7091D00D8091D10D909186
:10AF2000D20D0E94994D00E09C0141EB58E2672D43
:10AF3000812F0E94C6447FC082E0681226C08091A3
:10AF4000F405823021F40E94708081119EC08091AE
:10AF50002202882309F46FC011E08091F405823049
:10AF600009F010E06091D30D7091D40D8091D50D52
:10AF70009091D60D0E94994D00E09C0141EA58E263
:10AF8000672D812F0E94C64456C083E068122CC0F2
:10AF90008091F405833021F40E94708081118FC06C
:10AFA00080912202882309F446C011E08091F405C3
:10AFB000833009F010E08091D70D9091D80DA091C9
:10AFC000D90DB091DA0D89839A83AB83BC83CE010E
:10AFD00001960F945F4400E09C0141E958E2672D1F
:10AFE000812F0E94C64427C084E0681224C080914B
:10AFF000F405843021F40E947080811198C0809102
:10B0000022028823C1F011E08091F405843009F018
:10B0100010E06091DB0D7091DC0D8091DD0D909161
:10B02000DE0D0E94994D00E09C0141E858E2672D39
:10B03000812F0E94C6447394639485E0781237CFC1
:10B040007092F3058DC00E94E14D8091C105882367
:10B0500009F437CF85C081E00E946580A12CC12C06
:10B06000D12CE12C10E8F12E07E714E420E030E0C9
:10B0700040E85FE36FEC7DE089EB98E215DA8091C0
:10B08000C105882309F43ACF6BC081E00E94658036
:10B09000A12CC12CD12CE12C10E8F12E07E714E4EF
:10B0A00020E030E040E85FE363ED7DE089EA98E28C
:10B0B000FBD98091C105882309F449CF51C081E0B3
:10B0C0000E94658020E030E048EC52E46091D70DAA
:10B0D0007091D80D8091D90D9091DA0D0F94F14EA9
:10B0E00020E030E040E251E40F94D94B0F94274D1B
:10B0F0001F92812C912C9DEDA92E9CE4B92E6B0101
:10B1000015EFE12E1FE7F12E00E010E02AE030E01D
:10B1100040E050E067ED7DE089E998E20E94B87A6E
:10B120000F908091C105882309F43ACF19C081E0BE
:10B130000E946580A12CC12CD12CE12C10E8F12EAD
:10B1400007E714E420E030E040E85FE36BED7DE0EA
:10B1500089E898E2A9D98091C105882309F44FCFE5
:10B160000F900F900F900F90DF91CF911F910F9143
:10B17000FF90EF90DF90CF90BF90AF909F908F9017
:10B180007F906F9008952F923F924F925F926F92AF
:10B190007F928F929F92AF92BF92CF92DF92EF9267
:10B1A000FF920F931F93CF93DF93CDB7DEB729970D
:10B1B0000FB6F894DEBF0FBECDBF1C01798768873C
:10B1C000CA01B901E982FA820B831C83DE82CD8237
:10B1D000AF8220E030E040E251E40F94F14E6B0189
:10B1E0007C0120E030E040E057EC0F94B64E18169A
:10B1F0002CF0C12CD12CE12C27ECF22EC701B6018A
:10B200000F94224D2B013C0120E030E040E251E45C
:10B2100069817A818B819C810F94F14E4B015C0195
:10B2200020E03EEF4FEF56E40F94B34C87FD07C08C
:10B23000812C9EEF992EAA24AA9496E4B92E20E0A0
:10B2400030E040E251E4E885F985608171818281D6
:10B2500093810F94F14E6B017C01C301B2010F94F5
:10B26000554D9B01AC01C701B6010F94D94B0F940A
:10B27000274D69837A838B839C83C501B4010F9426
:10B28000224D7B018C01E418F50806091709FF819E
:10B29000FF938D809E8083EEA82E8CE4B82EC9800B
:10B2A000DA80A301920168857985C1010E94B87A8C
:10B2B0000F9029960FB6F894DEBF0FBECDBFDF9179
:10B2C000CF911F910F91FF90EF90DF90CF90BF90A3
:10B2D000AF909F908F907F906F905F904F903F9036
:10B2E0002F9008959F92AF92BF92CF92DF92EF92EC
:10B2F000FF920F931F93CF93DF9300D01F92CDB790
:10B30000DEB761E081E00E945D7C9090F505B12C94
:10B3100091101AC08091F405811104C00E947080C0
:10B320008111D4C080912202882309F4C7C081E032
:10B330009091F405911180E004E024E04FE658E29A
:10B340006B2D0E949244BAC081E098122CC080916B
:10B35000F405813021F40E9470808111BFC080917A
:10B360002202882309F4AAC011E08091F4058130FB
:10B3700009F010E08091130E9091140EA091150E1B
:10B38000B091160E89839A83AB83BC83CE0101965C
:10B390000F94FF4400E09C014BE558E26B2D812F98
:10B3A0000E94C6448BC082E098122CC08091F405A4
:10B3B000823021F40E9470808111ACC08091220201
:10B3C000882309F47BC011E08091F405823009F0F4
:10B3D00010E08091170E9091180EA091190EB09167
:10B3E0001A0E89839A83AB83BC83CE0101960F9496
:10B3F000FF4400E09C0147E458E26B2D812F0E943E
:10B40000C6445CC083E098122CC08091F405833060
:10B4100021F40E947080811199C0809122028823BA
:10B4200009F44CC011E08091F405833009F010E07C
:10B4300080911B0E90911C0EA0911D0EB0911E0EBE
:10B4400089839A83AB83BC83CE0101960F94FF441A
:10B4500000E09C0143E358E26B2D812F0E94C6441B
:10B460002DC084E098122AC08091F405843021F424
:10B470000E947080811186C0809122028823F1F0A1
:10B4800011E08091F405843009F010E080911F0EE6
:10B490009091200EA091210EB091220E89839A8363
:10B4A000AB83BC83CE0101960F94FF4400E09C0166
:10B4B0004FE158E26B2D812F0E94C644B3949394C0
:10B4C00085E0B81225CFB092F30577C00E94E14D18
:10B4D0008091C105882309F425CF6FC081E00E94C7
:10B4E0006580A12C6BEEC62E6CE4D62EE12C1CE3FD
:10B4F000F12E0CE116E420E030E040EA50E463E194
:10B500007EE085E698E23FDE8091C105882309F45C
:10B5100026CF53C081E00E946580A12C4BEEC42E43
:10B520004CE4D42EE12C1CE3F12E0CE116E420E0D7
:10B5300030E040EA50E467E17EE081E598E223DE16
:10B540008091C105882309F439CF37C081E00E947A
:10B550006580A12C2BEEC22E2CE4D22EE12C1CE314
:10B56000F12E0CE116E420E030E040EA50E46BE11B
:10B570007EE08DE398E207DE8091C105882309F41F
:10B580004CCF1BC081E00E946580A12C8BEEC82EA1
:10B590008CE4D82EE12C1CE3F12E0CE116E420E023
:10B5A00030E040EA50E46FE17EE089E298E2EBDDD2
:10B5B0008091C105882309F45FCF0F900F900F9001
:10B5C0000F90DF91CF911F910F91FF90EF90DF903F
:10B5D000CF90BF90AF909F9008950F93CF93DF933C
:10B5E00061E081E00E945D7CC091F505D0E0C11171
:10B5F00018C08091F405811104C00E9470808111EF
:10B60000B5C080912202882361F081E09091F40519
:10B61000911180E004E024E047EB5AE26D2F0E9494
:10B62000924480914B0D8770873009F058C0C1302B
:10B63000D9F48091F405813021F40E947080811149
:10B640009EC080912202882309F4C1C081E09091BC
:10B65000F405913009F080E003E02EE340EB5AE27C
:10B660006D2F0E949244B3C0C230D9F48091F4058A
:10B67000823021F40E94708081118BC0809122025F
:10B68000882309F4A4C081E09091F405923009F078
:10B6900080E003E02EE349EA5AE26D2F0E949244D3
:10B6A00096C0C330D1F58091F405833021F40E9417
:10B6B0007080811178C080912202882309F487C0AC
:10B6C00081E09091F405933009F080E003E02EE3EF
:10B6D00042EA5AE26D2F0E94924484E03EC0C1309B
:10B6E000F1F48091F405813021F40E947080811181
:10B6F00064C080912202882309F46BC081E090919C
:10B70000F405913009F080E000E22EE344E95AE2CA
:10B710006D2F0E94924482E020C084E001C082E04C
:10B72000C8131BC08091F4058C1304C00E94708064
:10B73000811151C080912202882371F081E09091A3
:10B74000F4059C1380E003E02EE34AE85AE26D2FF3
:10B750000E9492448C2F01C08C2FDF5FCF5FD530C9
:10B7600009F045CF8F5F8093F3053EC081E00E94D2
:10B77000777B8091C105882309F443CF35C08AE1E6
:10B7800090E60E94D5488091C105882309F459CFDD
:10B790002BC08FE190E60E94D5488091C105882397
:10B7A00009F46CCF21C084E290E60E94D5488091D4
:10B7B000C105882309F47FCF17C08EE99AE20E9461
:10B7C000B67A8091C105882309F493CF0DC084E037
:10B7D000C4CF82E0C2CF89E290E60E94D548809132
:10B7E000C105882309F4A6CFDF91CF910F91089569
:10B7F000CF92DF92EF92FF92CF93C82F0E94F92E43
:10B800006B017C0124EA30E74DE75FE360910C06B1
:10B8100070910D0680910E0690910F060F94B34C17
:10B8200087FD05C04AEF50E060E070E003C040E0F3
:10B8300050E0BA01C40ED51EE61EF71EC0920806DF
:10B84000D0920906E0920A06F0920B06C0932302FA
:10B85000CF91FF90EF90DF90CF9008952F923F927D
:10B860004F925F926F927F928F929F92AF92BF9210
:10B87000CF92DF92EF92FF921F93CF93DF93CDB7DA
:10B88000DEB728970FB6F894DEBF0FBECDBF1C0100
:10B89000162F0E947080882331F01092230680E0DA
:10B8A0000E94777BDDC020911B0630911C063E83F1
:10B8B0002D83232B09F4A0C0E4E01E9FC0011124B6
:10B8C00098878F83FC01E559FD4F80809180A2808D
:10B8D000B38020E030E04AE754E4C501B4010F949E
:10B8E000D94B2B013C0120E030E04AE754E4C5018C
:10B8F000B4010F94DA4B6B017C01809160028823C4
:10B90000B9F1113029F198F0123091F540905802B8
:10B910005090590260905A0270905B02C0905C0295
:10B92000D0905D02E0905E02F0905F0221C04090F6
:10B9300048025090490260904A0270904B02C090B9
:10B940004C02D0904D02E0904E02F0904F0210C099
:10B9500040905002509051026090520270905302F9
:10B96000C0905402D0905502E0905602F0905702D9
:10B970002D813E81B901330F880B990B0F94554DE2
:10B9800020910C0630910D0640910E0650910F0645
:10B990000F94F14E9B01AC01C501B4010F94DA4B39
:10B9A0009B01AC018F81988585599D4F5C01FC01FD
:10B9B00020833183428353838D819E8197FF0CC006
:10B9C000C301B2010F94B64E18168CF4F5014082F3
:10B9D0005182628273820BC0C701B6010F94B34CCF
:10B9E00087FF05C0F501C082D182E282F382812FF8
:10B9F000FFDE81E08093220210921C0610921B064B
:10BA000080912202882361F124E0129FF001112429
:10BA1000E559FD4F80819181A281B38189839A8309
:10BA2000AB83BC832DEC3CEC4CEC5DE360910C06ED
:10BA300070910D0680910E0690910F060F94B64EF0
:10BA400087FD05C0CE0101960F94694205C060E2F2
:10BA5000CE0101960F94E142BC01C1010E942B4529
:10BA600028960FB6F894DEBF0FBECDBFDF91CF9101
:10BA70001F91FF90EF90DF90CF90BF90AF909F907D
:10BA80008F907F906F905F904F903F902F90089590
:10BA900060E088E39BE2E2CE61E081E39BE2DECE00
:10BAA00062E08AE29BE2DACECF93DF9300D01F926E
:10BAB000CDB7DEB70E947080882331F01092230644
:10BAC00080E00E94777B57C060911B0670911C0636
:10BAD0006115710569F1072E000C880B990B0F9405
:10BAE000554D20910C0630910D0640910E06509157
:10BAF0000F060F94F14E9B01AC016091770270919B
:10BB000078028091790290917A020F94DA4B6093D7
:10BB10007702709378028093790290937A0283E09F
:10BB200067DE81E08093220210921C0610921B06B1
:10BB3000809122028823F9F02091290530912A056D
:10BB400040912B0550912C056091770270917802FD
:10BB50008091790290917A020F94D94B69837A830C
:10BB60008B839C83CE0101960F946942BC018EEBBE
:10BB70009AE20E942B450F900F900F900F90DF914B
:10BB8000CF91089521E02093230660930C067093D3
:10BB90000D0680930E0690930F0620E040E060E0D3
:10BBA00070E080912705909128050C94447B60E01B
:10BBB00070E080E291E4E6CF60E070E080E89FE32F
:10BBC000E1CF6DEC7CEC8CEC9DE3DCCF6DEC7CECA0
:10BBD0008CEC9CE3D7CF8F929F92AF92BF92CF9283
:10BBE000DF92EF92FF920F931F93CF93DF93CDB726
:10BBF000DEB76E970FB6F894DEBF0FBECDBFD82E5E
:10BC0000709328056093270561E081E00E945D7CC8
:10BC1000F090F5058CE0C82EE12C91E028ECA22EE6
:10BC20002AE2B22E9E012F5F3F4F490131E0D31629
:10BC300059F1D31628F082E0D81609F449C06CC037
:10BC4000F110D2C0992389F08091F40518166CF098
:10BC500020911B0630911C062F5F3F4F30931C062E
:10BC600020931B068F5F8093F40580912202882326
:10BC700009F432C100E010E021E041E063E27BE240
:10BC80008E2D0E942F4428C1F110AEC0992389F057
:10BC90008091F40518166CF020911B0630911C065B
:10BCA0002F5F3F4F30931C0620931B068F5F8093BE
:10BCB000F40580912202882309F411C100E010E00C
:10BCC00021E041E06CE17BE28E2D0E942F4407C110
:10BCD000F1108AC0992389F08091F40518166CF050
:10BCE00020911B0630911C062F5F3F4F30931C069E
:10BCF00020931B068F5F8093F40580912202882396
:10BD000009F40BC100E010E021E041E065E17BE2D5
:10BD10008E2D0E942F4401C14091770250917802EC
:10BD20006091790270917A024093290550932A0517
:10BD300060932B0570932C05F11020C0992389F096
:10BD40008091F40518166CF020911B0630911C06AA
:10BD50002F5F3F4F30931C0620931B068F5F80930D
:10BD6000F40580912202882349F000E010E021E0F0
:10BD700041E06BE07BE28E2D0E942F4493E0D912CC
:10BD800033C06091930C7091940C8091950C9091BC
:10BD9000960C2091580C211127C00F94224D209110
:10BDA00038023091390262177307F4F421E0F2127D
:10BDB00019C08091F405813021F40E9470808111B6
:10BDC000C0C080912202882369F081E09091F4053F
:10BDD000913009F080E004E024E04BEF5AE26E2D50
:10BDE0000E94924482E0A2C031E0F3121BC0809115
:10BDF000F405813021F40E9470808111ABC08091E4
:10BE00002202882309F468C081E09091F405913002
:10BE100009F080E004E024E041EF5AE26E2D0E9438
:10BE200092445AC082E0F8121BC08091F40582301F
:10BE300021F40E947080811196C080912202882393
:10BE400009F49BC081E09091F405923009F080E004
:10BE500003E02EE347EE5AE26E2D0E9492448DC01D
:10BE600093E0F9121BC08091F405833021F40E9405
:10BE70007080811186C080912202882309F4C3C09A
:10BE800081E09091F405933009F080E003E02EE327
:10BE90004EED5AE26E2D0E949244B5C024E0F2129B
:10BEA0001BC08091F405843021F40E9470808111C0
:10BEB00072C080912202882309F4A5C081E090918C
:10BEC000F405943009F080E003E02EE343ED5AE2FC
:10BED0006E2D0E94924497C032E0D31611F085E097
:10BEE00025C085E0F81219C08091F405853021F451
:10BEF0000E947080811159C080912202882369F0CC
:10BF000081E09091F405953009F080E003E02EE3A4
:10BF100042ED5AE26E2D0E949244809122028823C3
:10BF200021F095E0F91609F44AC086E0E394F39411
:10BF30002CE0C20E90E035E0E31278CE8093F3055A
:10BF400066C081E00E94777B8091C105882309F457
:10BF500038CF5DC081E00E94777B8091C105882346
:10BF600009F44DCF54C087ED9DE50E94D5488091DE
:10BF7000C105882309F461CF4AC082E0D812AFCF4F
:10BF8000CCCF8CED9DE50E94D5488091C1058823DA
:10BF900009F471CF3CC081EE9DE50E94D5488091A7
:10BFA000C105882309F485CF32C086EE9DE50E9445
:10BFB000D5488091C105882309F49ECF28C06C2DF7
:10BFC00086E00E94343B8E010B5E1F4F23E041E070
:10BFD0006DEC7CEC8CEC9CE30F9462509F938F9300
:10BFE000BF92AF929F928F920F947455B40189EED5
:10BFF00093E00E943B3A0F900F900F900F900F909C
:10C000000F9086E093CF92E0D91269CF86CF6E96DB
:10C010000FB6F894DEBF0FBECDBFDF91CF911F9159
:10C020000F91FF90EF90DF90CF90BF90AF909F90D7
:10C030008F9008954FEF68E47DE580E0CCCD4FEF21
:10C040006CE47DE581E0C7CD4FEF60E57DE582E002
:10C05000C2CD4FEF64E57DE583E0BDCD0F93CF9377
:10C06000DF9361E081E00E945D7CD091F505C0E046
:10C07000D1111AC08091F405811104C00E94708012
:10C0800081116FC080912202882309F461C081E090
:10C090009091F405911180E004E024E045E85AE233
:10C0A0006C2F0E94924454C0D130D9F48091F40591
:10C0B000813021F40E94708081115CC08091220245
:10C0C000882309F445C081E09091F405913009F08E
:10C0D00080E003E02EE34BE75AE26C2F0E9492448B
:10C0E00037C0D230D1F48091F405823021F40E941F
:10C0F0007080811149C080912202882349F181E03A
:10C100009091F405923009F080E000E22EE34DE6D4
:10C110005AE26C2F0E9492441BC0D330C9F4809124
:10C12000F405833021F40E947080811137C0809122
:10C130002202882369F081E09091F405933009F0A0
:10C1400080E000E22EE348E55AE26C2F0E94924420
:10C15000CF5FDF5FC53009F08BCF84E08093F305BC
:10C1600025C081E00E94777B8091C105882309F476
:10C1700089CF1CC08DEE9AE50E94D5488091C105FB
:10C18000882309F49BCF12C087E79AE20E94B67A0F
:10C190008091C105882309F4AECF08C089E69AE2F0
:10C1A0000E94B67A8091C105882309F2DF91CF9170
:10C1B0000F910895CF92DF92EF92FF920F931F930A
:10C1C0008091B208811103C084EF98E002C082EB35
:10C1D00098E024E8C22E2BE2D22E7C0107E71BE276
:10C1E00021E031E644E051E660E77BE28AE69BE24B
:10C1F0000E946B7D1F910F91FF90EF90DF90CF9089
:10C20000089580E00C94777B84EF98E00E94448B43
:10C210000E94707B0C947C860E94E68F21E030E0C7
:10C22000811102C020E030E030931C0620931B06F1
:10C230001092F50581E08093C10583E0809322028E
:10C240000895EF92FF920F931F93CF93DF93809106
:10C250001D06882331F00E94F69090932E0580935E
:10C260002D0561E081E00E945D7CC091F505D0E084
:10C27000C11118C08091F405811104C00E94708022
:10C28000811197C080912202882361F081E0909112
:10C29000F405911180E004E024E045E65BE26D2FB7
:10C2A0000E9492448091010985FD1FC083FF1DC03B
:10C2B000C130C9F48091F405813021F40E9470806E
:10C2C000811180C080912202882369F081E09091E1
:10C2D000F405913009F080E000E22EE341E65BE2F4
:10C2E0006D2F0E94924492E001C091E08091220261
:10C2F000882309F456C0E12CF12C11E01C0F209189
:10C300002D0530912E05E216F30608F04AC0C91338
:10C3100043C0C901019760E070E08E199F090E9437
:10C32000B98C909101098091F40594FF1CC08C1385
:10C3300050C00E947080882309F44BC084EF98E0BD
:10C340000E948B8F1092F50582E090E090931C067E
:10C3500080931B0681E08093C10510921E0683E046
:10C360008093220254C08C1304C00E9470808111FB
:10C370003FC080912202882369F081E09091F4050A
:10C380009C1380E000E025EB36E14FE35BE26D2F8C
:10C390000E942546912F01C09F5F8FEFE81AF80A8F
:10C3A000AECFDF5FCF5FD53009F062CF9093F3055A
:10C3B0002EC081E00E94777B8091C105882309F41B
:10C3C00061CF25C029DF8091C105882309F47ACF88
:10C3D0001EC0809122028823E9F281E09091F40549
:10C3E0009C1380E001E025EB36E140E55BE2CFCF36
:10C3F0000E94917A20E040E060E070E08AED90E6F3
:10C400000E94447B8091C105882309F4B2CFDF915B
:10C41000CF911F910F91FF90EF900895CF93DF93ED
:10C42000EC01CB01BA010F94554D0F94224D798345
:10C430006883DF91CF9108956EE072E685EA92E617
:10C440000C949B7B0F931F93CF93DF9361E081E06C
:10C450000E945D7CC091F505D0E081E0C11122C051
:10C46000882389F08091F40518166CF020911B0642
:10C4700030911C062F5F3F4F30931C0620931B0604
:10C480008F5F8093F40580912202882309F441C0D4
:10C4900000E010E020E041E069EE7CE28D2F0E9498
:10C4A0002F4437C0C130D1F48091F405813021F49C
:10C4B0000E947080811137C080912202882349F147
:10C4C00081E09091F405913009F080E000E22EE3E4
:10C4D0004EED5CE26D2F0E9492441BC0C230C9F445
:10C4E0008091F405823021F40E947080811122C075
:10C4F00080912202882369F081E09091F4059230C6
:10C5000009F080E000E22EE34AEC5CE26D2F0E942D
:10C510009244DF5FCF5F80E0D53009F09FCF83E0AA
:10C520008093F3050DC0C093D70B8091C10588237C
:10C5300019F206C0C093D70B8091C1058823C1F2C0
:10C54000DF91CF911F910F9108950F94554D0F9446
:10C55000224DCB010D946840EF92FF920F931F93F1
:10C56000CF93DF93CDB7DEB72B970FB6F894DEBF2E
:10C570000FBECDBF7C0140913005842F042E000CEE
:10C58000990B20913105223051F0233019F028E128
:10C590003DE20AC047FF06C024E23DE205C026E3B3
:10C5A0003DE202C02DE23DE29F934F933F932F93D4
:10C5B0008E010F5F1F4F1F930F930F94745540917F
:10C5C0003602509137024F50510997010F900F904A
:10C5D0000F900F900F900F904E155F050CF49A017D
:10C5E0003093980C2093970C80E00E94D1B5C8013D
:10C5F0000E94487D2B960FB6F894DEBF0FBECDBFCC
:10C60000DF91CF911F910F91FF90EF900895E091EE
:10C61000300587E1E802F0011124E157F34F8085EE
:10C6200091859ACF7F928F929F92AF92BF92CF9235
:10C63000DF92EF92FF920F931F93CF93DF93782EA9
:10C64000809331056093300561E081E00E945D7C5C
:10C65000D091F505C0E081E0D1112EC0882389F08A
:10C660008091F40518166CF020911B0630911C0681
:10C670002F5F3F4F30931C0620931B068F5F8093E4
:10C68000F40580912202882309F494C022E07216F6
:10C6900049F033E0731203C06AEF7CE205C06AEE32
:10C6A0007CE202C06AE07DE200E010E021E041E0CF
:10C6B0008C2F0E942F447EC0D130D9F48091F40594
:10C6C000813021F40E94708081117DC0809122020E
:10C6D000882309F46FC081E09091F405913009F04E
:10C6E00080E004E024E045E75DE26C2F0E94924484
:10C6F00061C0D230D9F48091F405823021F40E94D7
:10C700007080811169C080912202882309F452C08F
:10C7100081E09091F405923009F080E000E22EE390
:10C7200049E65DE26C2F0E94924444C0D330D1F4BC
:10C730008091F405833021F40E947080811157C0EC
:10C74000809122028823B1F181E09091F405933029
:10C7500009F080E000E22EE34DE55DE26C2F0E94DF
:10C76000924428C0D43031F58091F405843021F40E
:10C770000E947080811146C0809122028823D1F0EE
:10C7800011E08091F405843009F010E0209130052B
:10C7900037E12303F0011124E157F34F80859185A0
:10C7A0000F94684000E09C014FE35DE26C2F812F05
:10C7B0000E94C644CF5FDF5F80E0C53009F04CCFF8
:10C7C000C093F3055CC081E00E94777B8091C10536
:10C7D000882309F47BCF53C08091380590913905A7
:10C7E000BBDE8091C105882309F48DCF48C08091BC
:10C7F0003A0590913B05B0DE8091C105882309F48C
:10C800009FCF3DC081E00E9465800091300527E107
:10C81000020380011124F801E157F34F608571850F
:10C82000072E000C880B990B0F94554D20E030E03B
:10C8300040EF52E40F94D94B0F94274DF801E9567D
:10C84000F34F1F9287E0882E83E6982E9CE1A92E55
:10C8500092E6B92E6B011AEAE12EF12C00E010E00D
:10C8600028E730E040E050E0BF018EE49DE20E9406
:10C87000B87A0F908091C105882309F47DCFDF91AC
:10C88000CF911F910F91FF90EF90DF90CF90BF90CD
:10C89000AF909F908F907F90089560E081E0C2CE2E
:10C8A0008F929F92AF92BF92CF92DF92EF92FF92C0
:10C8B0000F931F93CF93DF934C015B016A0160E0FC
:10C8C00085E00E945D7CD091F505F12C82E0E82E98
:10C8D000D1111AC080912202882321F18091270270
:10C8E000823041F0833019F46FE97CE205C06DE8D5
:10C8F0007CE202C06FEA7CE200E010E021E041E06F
:10C900008F2D0E942F440EC0D13061F480912202FD
:10C91000882341F000E010E020E041E0B4018F2DD9
:10C920000E942F44A114B10481F0D23081F480918F
:10C930002202882309F46EC000E010E020E041E00C
:10C94000B5018F2D0E942F4465C0C2E001C0C3E035
:10C95000C114D10491F0DC130FC08091220288230E
:10C9600051F000E010E020E041E0B6018F2D0E9480
:10C970002F44CD2F01C0CD2FCF5F21E030E0A11497
:10C98000B10411F420E030E081E090E0C114D10462
:10C9900011F480E090E0820F931F029781F0DC1386
:10C9A0000DC080912202882349F000E010E020E0D1
:10C9B00041E068EC7CE28F2D0E942F44CF5FDC13B6
:10C9C00014C080912202882371F000E010E021E081
:10C9D00040E06DEB7CE28F2D0E942F4460912F058B
:10C9E0008F2D0E94C943E0922202F394DF5F85E01D
:10C9F000F8126ECFCF5FC093F305DF91CF911F91F7
:10CA00000F91FF90EF90DF90CF90BF90AF909F90ED
:10CA10008F900895C3E0C114D10409F0ADCFADCF1C
:10CA200040E050E060E070E082E89CE239CF49E706
:10CA30005CE269E67CE280E69CE232CF40E050E0D6
:10CA400060E57CE287E49CE22BCF40E050E068E3C5
:10CA50007CE289E29CE224CF40E050E06AE17CE2A3
:10CA60008DE09CE21DCF41E05CE260EF7BE280EE76
:10CA70009BE216CF40E050E062ED7BE289EC9BE266
:10CA80000FCF40E050E069EB7BE28CEA9BE208CFFD
:10CA900040E050E06FE97BE28EE99BE201CF40E0AD
:10CAA00050E06FE87BE286E89BE2FACE611160938A
:10CAB000270240932F05082E000C990BAA0BBB0BE5
:10CAC0008C309105A0F5FC018827EA56FF4F8F4F67
:10CAD0000D943B5087E195E61FC08EE195E61CC0A2
:10CAE00081E495E619C083E395E616C08AE395E6EE
:10CAF00013C08FE495E610C088E495E60DC08CE283
:10CB000095E60AC085E295E607C01092D70B82E24F
:10CB100092E602C080E195E6009749F021E020937B
:10CB2000230620E040E060E070E00C94447B0C942D
:10CB3000707BCF92DF92EF92FF920F931F9386E468
:10CB4000C82E8EE2D82EE12CF12C0BE31EE221E060
:10CB500031E64CE956E866E37EE281E39EE20E941C
:10CB60006B7D1F910F91FF90EF90DF90CF90089514
:10CB70009091010993FB882780F993FF06C081E01B
:10CB800090913107911101C080E00895EF92FF92DA
:10CB90000F931F93CF93DF9361E081E00E945D7C50
:10CBA000C091F50510E0C11118C08091F405811104
:10CBB00004C00E9470808111C8C180912202882324
:10CBC00061F081E09091F405911180E004E024E0AF
:10CBD00045E25EE2612F0E9492448091010982FB4E
:10CBE000002700F982FD07C0D1E09091A91691308D
:10CBF00019F0D0E001C0D02F83FBEE24E0F883FFD2
:10CC000003C0B6DFF82E01C0F12CDD2309F458C0B3
:10CC1000C130D9F48091F405813021F40E947080F4
:10CC200081119CC180912202882309F4A9C181E06D
:10CC30009091F405913009F080E000E22EE349E1A3
:10CC40005EE2612F0E9492449BC1C230D9F4809170
:10CC5000F405823021F40E947080811187C1809197
:10CC60002202882309F48CC181E09091F40592306E
:10CC700009F080E003E02EE34EE05EE2612F0E94C7
:10CC800092447EC1C33009F063C08091F4058330C3
:10CC900021F40E947080811175C180912202882345
:10CCA00009F46EC181E09091F405933009F080E0C1
:10CCB00003E02EE349E05EE2612F0E94924460C1EE
:10CCC0008091A916823029F053DF8823F9F00111F1
:10CCD0001DC0C130E9F48091F405813021F40E9437
:10CCE0007080811159C180912202882309F45CC1AE
:10CCF00081E09091F405913009F080E000E22EE3AC
:10CD00004CEF5DE2612F0E9492444EC1D1E001C020
:10CD1000D2E0CD131BC08091F4058C1304C00E9497
:10CD20007080811143C180912202882371F081E0DB
:10CD30009091F4059C1380E003E02EE345EF5DE263
:10CD4000612F0E949244DC2F01C0DC2FDF5F01C005
:10CD5000D4E0CD131BC08091F4058C1304C00E9455
:10CD6000708081112DC180912202882371F081E0B1
:10CD70009091F4059C1380E003E02EE349EE5DE220
:10CD8000612F0E949244DC2F01C0DC2F81E08D0FC7
:10CD9000C81318C08091F4058C1304C00E947080E1
:10CDA000811118C180912202882361F081E0909165
:10CDB000F4059C1380E003E02EE34BED5DE2612F70
:10CDC0000E94924482E08D0F4091970C5091980CF4
:10CDD0009091580C911107C020913802309139027E
:10CDE00042175307DCF0C81333C08091F4058C134D
:10CDF00004C00E9470808111F7C0809122028823B4
:10CE000039F181E09091F4059C1380E000E22EE37B
:10CE100043EC5DE2612F0E9492441AC0C81318C00F
:10CE20008091F4058C1304C00E9470808111E6C0CB
:10CE300080912202882361F081E09091F4059C1397
:10CE400080E003E02EE343EB5DE2612F0E94924419
:10CE5000DD5FCD1318C08091F4058C1304C00E94CF
:10CE600070808111D5C080912202882361F081E019
:10CE70009091F4059C1380E003E02EE345EA5DE227
:10CE8000612F0E94924491E09D0FEE2009F43BC077
:10CE9000F11053C0C91318C08091F4058C1304C05D
:10CEA0000E9470808111BEC080912202882361F0AF
:10CEB00081E09091F4059C1380E000E22EE344E9C8
:10CEC0005DE2612F0E94924482E08D0FC81318C06A
:10CED0008091F4058C1304C00E9470808111ACC055
:10CEE00080912202882361F081E09091F4059C13E7
:10CEF00080E003E02EE343E85DE2612F0E9492446C
:10CF000093E09D0F1AC0C91316C08091F4058C13CD
:10CF100002C00E94708080912202882361F081E02B
:10CF20009091F4059C1380E000E22EE34AE75DE275
:10CF3000612F0E94924492E09D0F1F5FCF5F1530DA
:10CF400009F031CE9093F30580C081E00E94777B99
:10CF50008091C105882309F430CE77C00E94AF8646
:10CF60008091C105882309F45DCE6FC089E995E6FB
:10CF70000E94D5488091C105882309F470CE65C010
:10CF8000D4E004CF84E899E60E94D5488091C10599
:10CF9000882309F482CE59C00E94C0868091C105C1
:10CFA000882309F4A0CE51C0D2E0D0CE8EE290E624
:10CFB0000E94D5488091C105882309F4B4CE45C0AC
:10CFC0008EE09CE60E94D5488091C105882309F433
:10CFD000CACE3BC084EA99E70E94D5488091C1053A
:10CFE000882309F4DFCE31C083ED9DE20E94B67A3A
:10CFF0008091C105882309F400CF27C08DE494E611
:10D000000E94D5488091C105882309F411CF1DC025
:10D0100081E89BE60E94D5488091C105882309F4E8
:10D0200022CF13C081EA9DE20E94B67A8091C105A9
:10D03000882309F439CF09C081E291E60E94D548DE
:10D040008091C105882309F44BCFDF91CF911F91C7
:10D050000F91FF90EF9008956091880C70E080E050
:10D060000C9486B060918B0270918C02072E000C9C
:10D07000880B990B0F94554D2AE037ED43E25CE3A2
:10D080000F94F14E60938702709388028093890217
:10D0900090938A020895CF93DF93EC01CB01BA01FC
:10D0A0000F94554D0F94274D6883DF91CF910895CC
:10D0B00080E00C94D1B56BE478E681E698E60C94B8
:10D0C0009B7B0F94554D0F94274D862F0D94EC3F6D
:10D0D000EF92FF920F931F93CF93DF9300D01F9295
:10D0E000CDB7DEB7082F7B010E947080882331F016
:10D0F0001092230680E00E94777B3BC060911B0664
:10D1000070911C066115710551F010921C06109269
:10D110001B0681E080932202802F0E94E7A8809165
:10D120002202882331F184E0089F800111240152FA
:10D13000124F6091C10B7091C20B072E000C880B2F
:10D14000990B0F94554D9B01AC01F80160817181E1
:10D15000828193810F94F14E69837A838B839C83C0
:10D1600060E2CE0101960F947943BC01C7010E9491
:10D170002B450F900F900F900F90DF91CF911F9143
:10D180000F91FF90EF90089561EC7EE280E0A0CFD8
:10D1900066EB7EE281E09CCF20E040E060E070E062
:10D1A0000E94447B81E0809323061092C20B109270
:10D1B000C10B089584EC98E6EFCF88EC98E6ECCFAD
:10D1C0002F923F924F925F926F927F928F929F9297
:10D1D000AF92BF92CF92DF92EF92FF920F931F9385
:10D1E000CF93DF93CDB7DEB729970FB6F894DEBFA4
:10D1F0000FBECDBF1C017987688769011A83098337
:10D20000EB82BA01550F880B990B0F94554D4B01CA
:10D210005C0120E030E040E057EC0F94B64E181669
:10D220002CF0812C912CA12C27ECB22EC501B4013D
:10D230000F94224D2B013C01B601DD0C880B990B9C
:10D240000F94554D4B015C0120E03EEF4FEF56E44B
:10D250000F94B34C87FD07C0812C9EEF992EAA2412
:10D26000AA9496E4B92EE885F98560817181072E2C
:10D27000000C880B990B0F94554D6B017C01C30179
:10D28000B2010F94554D9B01AC01C701B6010F943B
:10D29000D94B0F94274D6C837D838E839F83C5016B
:10D2A000B4010F94224D7B018C01E418F5080609A6
:10D2B0001709FB81FF9389809A808CE1A82E82E672
:10D2C000B82ECC80DD80A301920168857985C101EB
:10D2D0000E94B87A0F9029960FB6F894DEBF0FBE61
:10D2E000CDBFDF91CF911F910F91FF90EF90DF9015
:10D2F000CF90BF90AF909F908F907F906F905F90F6
:10D300004F903F902F9008958F929F92AF92BF922F
:10D31000CF92DF92EF92FF920F931F93CF93DF9301
:10D3200061E081E00E945D7CD091F505C0E0D11103
:10D330001AC08091F405811104C00E94708081118F
:10D3400021C180912202882309F413C181E09091C8
:10D35000F405911180E004E024E041EB5EE26C2FE3
:10D360000E94924406C1D13011F58091F4058130BC
:10D3700021F40E94708081110EC1809122028823C5
:10D3800009F4F7C011E08091F405813009F010E054
:10D3900080916502909166020F94684000E09C01C4
:10D3A00045EA5EE26C2F812F0E94C644E2C0D23073
:10D3B00011F58091F405823021F40E947080811172
:10D3C000FCC080912202882309F4D3C011E080912F
:10D3D000F405823009F010E08091970C9091980C40
:10D3E0000F94684000E09C0147E95EE26C2F812FBA
:10D3F0000E94C644BEC0D33011F58091F40583303D
:10D4000021F40E9470808111EDC080912202882356
:10D4100009F4AFC011E08091F405833009F010E009
:10D4200080916E0C90916F0C0F94684000E09C010D
:10D430004FE85EE26C2F812F0E94C6449AC0D43020
:10D4400001F58091F405843021F40E9470808111EF
:10D45000DEC080912202882309F48BC011E0809104
:10D46000F405843009F010E08091880C0F94EC3FB3
:10D4700000E09C0147E75EE26C2F812F0E94C644CA
:10D4800078C0D53011F58091F405853021F40E94E3
:10D4900070808111DFC080912202882309F469C065
:10D4A00011E08091F405853009F010E080918B0245
:10D4B00090918C020F94684000E09C014DE65EE282
:10D4C0006C2F812F0E94C64454C0D630D9F480916D
:10D4D000F405863021F40E9470808111CDC08091C6
:10D4E0002202882309F445C081E09091F40596302A
:10D4F00009F080E003E02EE342E65EE26C2F0E943A
:10D50000924437C0D730D1F48091F405873021F4AC
:10D510000E9470808111BAC080912202882349F153
:10D5200081E09091F405973009F080E003E02EE36C
:10D5300047E55EE26C2F0E9492441BC0D830C9F4CC
:10D540008091F405883021F40E9470808111A8C078
:10D5500080912202882369F081E09091F40598304F
:10D5600009F080E003E02EE348E45EE26C2F0E94C5
:10D570009244CF5FDF5FC53009F0D9CE89E0809358
:10D58000F30597C081E00E94777B8091C1058823D5
:10D5900009F4D7CE8EC0E12C00E010E027EE33E096
:10D5A0004AE050E065E672E08BEA9EE209DE809197
:10D5B000C105882309F4E1CE7CC081E00E9465802A
:10D5C000E12C08E518E622E231E040E050E067E9AE
:10D5D0007CE08EE99EE2F4DD8091C105882309F4A8
:10D5E000F0CE67C081E00E946580E12C0EE116EB71
:10D5F0002CE830E040E050E06EE67CE083E99EE21B
:10D60000DFDD8091C105882309F4FFCE52C081E09F
:10D610000E946580C090880CD12C1F928CE2882ECD
:10D6200088E6982E9BE5A92E98E6B92EE12CF12CE0
:10D630008701EA9420E030E0A90168E87CE083E813
:10D640009EE20E94B87A0F908091C105882309F468
:10D6500000CF2FC0E12C02E318E627EE33E04AE0CA
:10D6600050E06BE872E082E79EE2AADD8091C1059E
:10D67000882309F410CF1DC08AED98E60E94D54892
:10D680008091C105882309F42ACF13C08DED98E657
:10D690000E94D5488091C105882309F43DCF09C077
:10D6A00083EC9CE70E94D5488091C105882309F44A
:10D6B0004FCFDF91CF911F910F91FF90EF90DF90AF
:10D6C000CF90BF90AF909F908F9008950E947080F0
:10D6D000882329F01092230680E00E94777B80E067
:10D6E0000C9459430E947080882341F020E040E070
:10D6F00060E070E086E69BE60E94447B80E00C944C
:10D7000095A00F93CF93DF9361E081E00E945D7C51
:10D71000D091F505C0E0D11117C08091F4058111B9
:10D7200004C00E94708081114CC080912202882325
:10D7300009F43EC081E09091F405911180E004E08D
:10D7400024E043EE5EE231C0D130B9F48091F405BB
:10D75000813021F40E94708081113CC080912202AE
:10D76000882331F181E09091F405913009F080E057
:10D7700003E02EE342ED5EE218C0D530C9F480919B
:10D78000F405853021F40E94708081112DC08091B4
:10D790002202882369F081E09091F405953009F028
:10D7A00080E003E02EE34CEC5EE26C2F0E9492449A
:10D7B000CF5FDF5FC53009F0AECF86E08093F30521
:10D7C0001BC081E00E94777B8091C105882309F40A
:10D7D000ACCF12C082E79BE60E94D5488091C1057C
:10D7E000882309F4BBCF08C08BEE98E40E94D5488B
:10D7F0008091C105882359F2DF91CF910F9108954F
:10D8000060E070E080E00E9486B060E070E081E05F
:10D810000E9486B00E946BB60C94707B8F929F9290
:10D82000AF92BF92CF92DF92EF92FF920F931F932E
:10D83000CF93DF9361E081E00E945D7CD091F5059C
:10D84000C0E0D1111AC08091F405811104C00E947A
:10D8500070808111ABC080912202882309F474C0CA
:10D8600081E09091F405911180E004E024E04FE123
:10D870005FE26C2F0E94924467C0D13011F5809115
:10D88000F405813021F40E947080811198C080914C
:10D890002202882309F458C011E08091F4058130F8
:10D8A00009F010E08091970C9091980C0F946840CB
:10D8B00000E09C0141E15FE26C2F812F0E94C64491
:10D8C00043C0D23009F58091F405823021F40E94E2
:10D8D000708081119AC0809122028823A9F111E001
:10D8E0008091F405823009F010E080916E0C9091E7
:10D8F0006F0C0F94684000E09C0149E05FE26C2FE0
:10D90000812F0E94C64420C0D330F1F48091F405E9
:10D91000833021F40E94708081119CC0809122028A
:10D92000882391F011E08091F405833009F010E034
:10D930008091880C0F94BD3F00E09C0141EF5EE2B6
:10D940006C2F812F0E94C6448091970C9091980C67
:10D9500020916E0C30916F0C232B11F4892BE9F080
:10D96000D430C9F48091F405843021F40E94708091
:10D970008111A1C080912202882369F081E09091F9
:10D98000F405943009F080E000E22EE348EE5EE218
:10D990006C2F0E94924485E001C084E0CF5FDF5F7E
:10D9A000C53009F04ECF8093F3058BC081E00E9413
:10D9B000777B8091C105882309F44DCF82C081E037
:10D9C0000E946580C090970CD090980C1F9268E5DB
:10D9D000862E68E6962E7CE1A72E72E6B72E12E21E
:10D9E000E12EFF24F39400E010E020E030E0A901F4
:10D9F00067E97CE088E19FE20E94B87A0F9080910D
:10DA0000C105882309F443CF5CC081E00E94658092
:10DA1000C0906E0CD0906F0C1F923EE1832E36EBBF
:10DA2000932E4CE1A42E42E6B42E1CE8E12EF12CFC
:10DA300000E010E020E030E0A9016EE67CE08DE03F
:10DA40009FE20E94B87A0F908091C105882309F463
:10DA500042CF37C081E00E9465806091880C70E001
:10DA600080E090E00F94534D29EC38EC48EC5EE3F5
:10DA70000F94F14E0F94274D1F928CE2882E88E66A
:10DA8000982E91EBA92E99E4B92E6B0114E6E12EA4
:10DA9000F12C00E010E020E030E0A90168E87CE033
:10DAA0008DEF9EE20E94B87A0F908091C105882385
:10DAB00009F434CF06C0A4DE8091C105882309F49F
:10DAC00059CFDF91CF911F910F91FF90EF90DF9091
:10DAD000CF90BF90AF909F908F90089580E095E297
:10DAE00090934C0580934B058CE491E09093500506
:10DAF00080934F0580EC9EEF90934E0580934D05EB
:10DB00009091470580E2890F863740F080EF890FBA
:10DB100020E431E030934E0520934D0510924905E5
:10DB200080934A058FEF8093480508958F929F92C6
:10DB3000BF92CF92DF92EF92FF920F931F93CF93FA
:10DB4000DF931F92CDB7DEB7F7D7882309F4D6C18C
:10DB500080911B06863214F085E202C087FD80E0CA
:10DB6000282F082E000C330B30931C0620931B0625
:10DB7000982F990F890F809347058091AB058823D3
:10DB800009F4BCC120914D0530914E050091490525
:10DB900010914A05020F131FE0904B05F0904C05C1
:10DBA00080914F0590915005E80EF91E01304FE726
:10DBB000140768F031952195310930934E05209373
:10DBC0004D056CED70E085E090E00F94E046F7FEC7
:10DBD00015C080914F0590915005919581959109BF
:10DBE0009093500580934F0568E171E085E090E0E7
:10DBF0000F94E04681E08093480517C081E0E81665
:10DC000080E4F80694F06BE470E084EF91E00F9408
:10DC1000E04680913D05815080933D05882311F0B9
:10DC20005DDF6CC11092AB0569C120914F05309149
:10DC30005005C7019A508130934108F098C08F2D4C
:10DC4000992787FD9A950A9765E070E00F94EA4F4F
:10DC5000812F17FF02C087E0810F482F459545951A
:10DC6000459581E090E0A0E0B0E004C0880F991FE6
:10DC7000AA1FBB1F4A95D2F7FB01EE0FFF1FE15C05
:10DC8000FA4F408151818A0108231923012B09F49D
:10DC900019C180959095842395239183808384E096
:10DCA00090E0861B970B4091AC055091AD05840F19
:10DCB000951F9093AD058093AC0580913E058150F2
:10DCC00080933E05811103C082E08093AB05932FC2
:10DCD0009095991F9927991F80914805881F88273B
:10DCE000881F9817F1F0319521953109309350052F
:10DCF00020934F0520E130E040E050E060EF7FEFFF
:10DD00008FEF9FEF0E94953920914D0530914E0580
:10DD1000620F731F70934E0560934D0560E773E0CB
:10DD200021C080914D0590914E0591958195910965
:10DD300090934E0580934D0520E130E040E050E0A7
:10DD400060EF7FEF8FEF9FEF0E94953920914F0595
:10DD500030915005620F731F7093500560934F050B
:10DD600060E872E085E090E00F94E046ABC01216E8
:10DD700013060CF0A7C0FDE3FF1A41E0E41642E0F1
:10DD8000F40608F09FC080914705181B103108F079
:10DD900099C03195219531093093500520934F0555
:10DDA00060E773E083E090E00F94E0468FEF8093AC
:10DDB000480521E012300CF020E08EEF810F8C300E
:10DDC000A0F080914D0590914E0541E050E018166D
:10DDD000190614F040E050E030E04217530709F014
:10DDE00055C091958195910927C0143050F520E0D8
:10DDF00030E0A90160EC7FEF8FEF9FEF0E94953933
:10DE000020914D0530914E05620F731F70934E05A2
:10DE100060934D0561157E4F34F480E09EEF909342
:10DE20004E0580934D0580914D0590914E058130B2
:10DE3000924064F180E092E090934E0580934D050E
:10DE400025C01C301CF120E430E040E050E060E0F0
:10DE500070E0CB010E94953920914D0530914E051F
:10DE6000620F731F70934E0560934D0561157E4FD1
:10DE700034F480E09EEF90934E0580934D058091A1
:10DE80004D0590914E0581309240A4F68091AB05EE
:10DE90008230C1F480E480933E058FEF9FEF909332
:10DEA000400580933F0590934205809341059093F0
:10DEB000440580934305909346058093450581E092
:10DEC0008093AB052091490530914A0580914D051D
:10DED00090914E05820F931F90934A0580934905B8
:10DEE00020914B0530914C0580914F059091500544
:10DEF000820F931F90934C0580934B0561E08DEE4C
:10DF000093E00E942C34809121048E3130F0809176
:10DF100021048E3308F456C05AC0809123048A30FD
:10DF2000B0F38DE3E82E85E0F82E9AE0892E912C4F
:10DF3000B82C8091210490E094012C5F3F4F28176A
:10DF400039075CF442E0E40EF11C85E0880E911C78
:10DF5000EEE18E16910461F7DACF809123048815E3
:10DF600088F330E0C12CD12CF70182819381A0E0AD
:10DF7000B0E00C2C04C0B695A795979587950A94A8
:10DF8000D2F780FD07C0FFEFCF1ADF0A385F3038C5
:10DF900059F7D8CF00E010E0A801480D591D809135
:10DFA000210490E0481759073CF08091230490E049
:10DFB000841795070CF056C00F5F1F4F04301105F2
:10DFC00059F7E1CF809123048C3308F056C080913B
:10DFD000AB058823B1F080914C05482F582F550F81
:10DFE000550B9A0133272F5F3F4F8091210490E01A
:10DFF000281739073CF080912304841708F04EC09D
:10E0000001C0B3D5809121048B30D8F40091AC05C8
:10E010001091AD0569E080E00E94343BC8010E9488
:10E02000393B69E08EE60E94343B20913D0583E058
:10E0300090E0821B91096FEF7FEF8C5D904D0E9405
:10E040008D3B0E947080882391F10F90DF91CF91DA
:10E050001F910F91FF90EF90DF90CF90BF909F9016
:10E060008F90C0C527E04B2D400F632F8DEE93E0BE
:10E0700039830E943D3639819FCF20E14DE3609185
:10E0800047058DEE93E00E943D3620E14CE3609120
:10E0900047058DEE93E00E943D3699CF60914A0589
:10E0A00002E022E08DEE93E00E947E36ABCF0F902F
:10E0B000DF91CF911F910F91FF90EF90DF90CF9064
:10E0C000BF909F908F90089566E97DE682E079D5B4
:10E0D000EDE3F5E088E3828783E0808380E4818359
:10E0E000138212821582148217821682118610867C
:10E0F000F5DC82E190E090931C0680931B06089566
:10E100008F929F92AF92BF92CF92DF92EF92FF9247
:10E110006091680520E030E090E080E0F901E35C88
:10E12000FA4FC7A4CC2011F061E0620F8C29722F46
:10E130007295707F40E050E0D12CE12CF12C46012B
:10E140005701042E04C0B694A794979487940A9418
:10E15000D2F780FE08C0E92FF0E0E35CFA4FA72F6A
:10E16000A42BA2AB9F5F4F5F5F4F4530510539F73E
:10E170002F5F3F4F2330310589F66093680540E0FB
:10E1800050E020E090E0A0E0B0E06C017D01042EC2
:10E1900004C0F694E794D794C7940A94D2F7C0FECB
:10E1A00005C0209366052AE335E007C02E504F5F77
:10E1B0005F4F4530510549F7F4CF422F3150A0F061
:10E1C000225F6C017D01032E04C0F694E794D7947E
:10E1D000C7940A94D2F7C0FEF0CF409367058091B0
:10E1E0006905823069F403C020936705F8CF8091F8
:10E1F0006505181614F08CEF01C084E08093650566
:10E20000FF90EF90DF90CF90BF90AF909F908F9056
:10E21000089580E090E0FC01E35CFA4F16820396DB
:10E220008E319105C1F70895EDE3F5E010828AE0A3
:10E23000818383E080A78FE084A78FE187A780ABED
:10E2400081AB5EDFE6CF1F93CF93DF93EC01162FF8
:10E25000E0DF809140058093620587E3809363054A
:10E2600086E0809364056AE070E088EE93E00F94A6
:10E27000E04690913F05915090933F05992351F0CE
:10E280001092610518831092400510921C0610929E
:10E290001B0601C01882DF91CF911F9108952F9224
:10E2A0003F925F926F927F928F929F92AF92BF92B6
:10E2B000CF92DF92EF92FF920F931F93CF93DF9352
:10E2C0001F92CDB7DEB784E08093220280911D06B5
:10E2D000882309F470C280911B0690911C068E3130
:10E2E000910514F08DE190E097FF02C080E090E08E
:10E2F00090931C0680931B06880F991F880F991F07
:10E3000020914005422F022E000C550B481759074B
:10E3100074F42D5FAC01421B510927FD5395423027
:10E3200051051CF02093400502C0809340052091C8
:10E330004005422F022E000C550B841795077CF4E4
:10E340002350422F022E000C550B481B590B423014
:10E3500051051CF02093400502C080934005809138
:10E36000AB05882309F427C220917F05222349F0B9
:10E3700090917E05920F90937E05933F14F4109236
:10E380007F05823070F081508093AB05823011F4AC
:10E390004BDF11C2843609F00EC281E08093AB05D9
:10E3A0000AC280916B058F5F80936B054091690570
:10E3B00090E0242F30E035952795281739070CF089
:10E3C000B3C09091800581E08927809380051092E9
:10E3D0006B05442309F4A8C09091650580913D0523
:10E3E000890F20916605821724F020916705281770
:10E3F000D4F491959093650520913E052B5F209371
:10E400003E0580933D05809168053AE08302C00196
:10E410001124820F911D27FD9A95C99724F064E17C
:10E420008BEA95E010DF9091650580913D05890F9D
:10E4300080933D0580916905882309F475C024E126
:10E4400030E040E050E060E070E0CB010E949539A0
:10E45000672B682B692B09F067C0E3E4F5E080E0E7
:10E4600090E0208121115AC09C01220F331F8901A5
:10E47000080F191FC8018F5B9A4F892B09F454C0EC
:10E480002091690530E02F5F3F4F032E000C440BB5
:10E49000550B60E070E0CB010E949539FB01E35C15
:10E4A000FA4F42A9242F30E0B4E035952795BA956C
:10E4B000E1F7F901E55BFC4F808190E0035C1A4FC6
:10E4C0004F7050913D056EE0469F500D1124452F31
:10E4D000FC01E85BFC4F5081450FFC01EB5BFC4FFE
:10E4E00090819695842F890FF801848380913E0551
:10E4F00082502F5F3F4FFAE02F9F800D1124F801CB
:10E50000858322E030E040E050E060E070E0CB0145
:10E510000E9495396E5FF801668306C001963396B6
:10E520008A30910509F09DCF90916105992341F0C2
:10E5300080916005890F8093600587FD10926105C9
:10E5400080916105882309F4A2C020916005E091C3
:10E550003E052E170CF49BC0022E000C330B0E2E22
:10E56000000CFF0BCF014D96821793070CF48FC060
:10E5700010913D05E0905F05CE2C0E2C000CDD08BF
:10E58000C601811B910917FD93956EE070E00F9411
:10E59000EA4FF62E653008F07AC02E1B3F0BC901FA
:10E5A00002966AE070E00F94EA4F062F633008F09D
:10E5B0006EC0812C912C540183940F2C04C0880CC4
:10E5C000991CAA1CBB1C0A94D2F7A62F660FBB0B82
:10E5D000BD01635C7A4FFB0197A5892F882109F45F
:10E5E00056C0FD01E55BFC4FE0814E2F50E0812FCE
:10E5F000FEE0FF9E800D11249A01285B3C4FF9013B
:10E60000F080F80EEF140CF442C0FA01EB5BFC4F03
:10E610001081412F50E04F0D511DF7FC5A95C41643
:10E62000D506ACF510926105282D20952923FB0114
:10E6300027A723E030E02A1B3B0B8091AC0590918B
:10E64000AD05280F391F3093AD052093AC056AE066
:10E6500070E088E290E00F94E04620913E05FAE0F9
:10E660000F9F200D1124912F96958F2D890F855086
:10E67000809362052093630584E080936405809114
:10E680006905815080936905882321F039DD03E411
:10E6900015E012C084E18093AB05BBDDF8CF829119
:10E6A000890F808380346CF0F80110820D5F1F4F5A
:10E6B000F5E001361F07E9F0F80190819923B1F3E5
:10E6C000EECF87339CF3F80132972081809140058B
:10E6D000281764F3022E000C330B082E000C990B44
:10E6E0000A968217930714F368E78BEA95E0ABDD8F
:10E6F000DDCF80917F05811124C024EF31E040E01F
:10E7000050E060E070E0CB010E949539672B682BE8
:10E71000692BB9F422E030E040E050E060E070E0C6
:10E72000CB010E949539672B682B692B09F099C1A1
:10E730008FEF80937F05813009F495C18FE7809337
:10E740007E05809161058823B1F180917F05882342
:10E7500091F180916005873074F520915F0580917B
:10E760007E05281744F1022E000C330B082E000CF6
:10E77000990B0C9682179307F4F010927F05109274
:10E7800061058091AC059091AD050A969093AD0519
:10E790008093AC056AE070E088E290E00F94E04678
:10E7A00080917E058F5F8093620581E08093630591
:10E7B00084E0809364058091250682FF04C08091E7
:10E7C0006A05815001C08AE080936A050E947080CA
:10E7D0008823C1F08091AB05811103C010926A05B6
:10E7E00011C0813079F48091610581110BC0809155
:10E7F00040058B5F80935F0584E3809360058CEF19
:10E800008093610580916A05811101C0EBD161E0BF
:10E810008DEE93E00E942C3430913E05632F032E41
:10E82000000C770B80916805AB012AE08202400D55
:10E83000511D1124425051098091210490E0841708
:10E8400095072CF080917F0581116BC06FC080917E
:10E85000230490E086179707ACF3FBE46F2EF3E0F8
:10E860007F2EC12CD12CF30121913F01432F032E88
:10E87000000C550BBA01695F7F4F8091210490E035
:10E88000681779074CF4365FFFEFCF1ADF0A23E0F1
:10E89000C216D10441F7D6CF8091230490E08417AB
:10E8A00095078CF310913D0546E4542E510EA12C92
:10E8B000B12CC601835C9A4F4C01822F90E01C0161
:10E8C000220C331CF40187A590E0A0E0B0E00A2CF4
:10E8D00004C0B695A795979587950A94D2F780FFBF
:10E8E00019C0809180057101E80EF11CC701E4E0B8
:10E8F000880F991FEA95E1F7AC01495A504D7A010A
:10E9000008E022E0432F612F8DEE93E039830E94CF
:10E9100056343981125F5FEFA51AB50A1511D2CFAF
:10E92000B2CF80912104883008F49FC08091AB055C
:10E93000882369F0909121049F3348F49091230437
:10E94000973328F0823008F49EC081FD9CC08091EE
:10E9500061058823B1F040916005242F042E000C3E
:10E96000330BB9016D5F7F4F8091210490E06817F0
:10E9700079073CF08091230490E0821793070CF014
:10E9800090C000E010E0F801E35CFA4F8681882334
:10E9900099F04581842F042E000C990B20912104BD
:10E9A00030E08217930744F002972091230430E06F
:10E9B000281739070CF07DC00D5F1F4F0E31110570
:10E9C00011F7809164058823B1F040916305242FED
:10E9D000042E000C330BB9016A5F7F4F8091210434
:10E9E00090E0681779073CF08091230490E082174B
:10E9F00093070CF066C08091AB05811101C0B5D0C2
:10EA0000809121048A3008F06EC00091AC0510910D
:10EA1000AD0569E080E00E94343BC8010E94393BAB
:10EA200080913F05882309F45EC011E060E1C62EA5
:10EA3000D12C80913F05811708F455C0B601611BA8
:10EA40007109660F660F660F72E4E72E7FE2F72EFC
:10EA500005E021E041E08DEE93E00E9456341F5F17
:10EA6000E8CF81E066CE83EF6ACE2AE2E22E2FE283
:10EA7000F22E05E022E042E060917E058DEE93E00B
:10EA80000E94563453CF97E4E92E9FE2F92E08E016
:10EA900022E047E3609140058DEE93E00E945634FA
:10EAA00056CF24E060915F058DEE93E00E945D36C5
:10EAB00068CF425023E064818DEE93E00E945D3682
:10EAC0007BCF84E3E82E8FE2F82E07E022E060910E
:10EAD00062058DEE93E00E9456348091640581506A
:10EAE0008093640588CF0F90DF91CF911F910F9194
:10EAF000FF90EF90DF90CF90BF90AF909F908F905E
:10EB00007F906F905F903F902F900895CF93DF9309
:10EB10006FE471E784E155D0CDE3D5E083E08A83EB
:10EB20008AE08DA71CA280DB1B8210921C0610922B
:10EB30001B06DF91CF91089580911D06882319F05F
:10EB400082E080933C0584E0809322028091AB05B3
:10EB5000882349F090913C058FEF890F80933C0505
:10EB600081E019160CF080E008950F938091210444
:10EB7000853228F5809123048B3108F160E08DEE19
:10EB800093E00E942C3409E028E34BE164E28DEE2F
:10EB900093E00E94CE3661E08DEE93E00E942C342B
:10EBA0000E94B981882359F063E285E20E94343BD8
:10EBB0006FEF7FEF87EB9FE20F910C948D3B0F91EE
:10EBC0000895FB011092AD051092AC058093AB0542
:10EBD00020E040E060E070E0CF0156D581E0809316
:10EBE000230608951092230680E081C58091420596
:10EBF0009091440589130DC080914305909145057E
:10EC0000891714F02FEF01C021E0820F8093430594
:10EC100008C0891714F02FEF01C021E0820F809304
:10EC2000420589131BC02091AA0521502093AA05F3
:10EC300030E0832F90E0DC01AA0FBB1FA35CBA4F2A
:10EC4000880F991FFC01E15CFA4F85819681169629
:10EC50009C938E9315973F5F231758F70895EF9273
:10EC6000FF921F93CF93DF931091AA0520913F0548
:10EC7000E22E022E000CFF0830913E05C32F032E1A
:10EC8000000CDD0BE5E4F5E040E0411709F446C077
:10EC9000CF010397DC019C91BF0161507109DB0139
:10ECA0008C9198131DC0692F092E000C770B6150B1
:10ECB0007109C617D70711F039132DC09081BF0114
:10ECC00062507109DB018C91582F98170CF4592F61
:10ECD00025170CF189170CF4892F8217E4F020C056
:10ECE000BF0162507109DB015C91652F052E000C9C
:10ECF000770B61507109E616F70611F025130BC06A
:10ED0000582F98170CF4592F35172CF089170CF43D
:10ED1000892F83172CF44F5F3296B7CF80E001C064
:10ED200081E0DF91CF911F91FF90EF90089528E14E
:10ED300030E040E050E060E070E0CB010E949539A7
:10ED400060933E052AE030E040E050E060E070E093
:10ED5000CB010E94953960933F0581DF8111E7CF98
:10ED6000089590913D05811102C08FEF01C081E0AF
:10ED7000980F937090933D058091AA058F5F8093C3
:10ED8000AA0590E0FC01EE0FFF1FE35CFA4F209113
:10ED9000A7052583880F991FFC01ED5BFA4F809131
:10EDA000A905808308951F93CF93DF93CDE3D5E02A
:10EDB00080E091E09093A7058093A60580E095E020
:10EDC0009093A9058093A80518821092AA051D8228
:10EDD00015E01E8381E0C5DF1B8310921C06109294
:10EDE0001B061C82DF91CF911F910895EF92FF9235
:10EDF0000F931F93CF93DF938091AA05843008F47B
:10EE0000DEC090E0FC01EE0FFF1FE55CFA4F35819C
:10EE1000FC01EE0FFF1FE35CFA4F6581AC0142502D
:10EE20005109361739F0C0E0880F991FFC01EF5BDC
:10EE3000FA4F82C0F12CDC01AA0FBB1FAD5BBA4FA9
:10EE4000880F991FFC01EF5BFA4F8F2D90E084171C
:10EE500095070CF0B4C0BC01660F771F635C7A4F56
:10EE6000EB016D818C01000F111F015C1A4FE8014D
:10EE70002D816217F1F0722F62170CF4762F37177D
:10EE8000ECF126170CF4262F2317C4F1880F991FD5
:10EE90008D5B9A4FEC01288191E0808128170CF05E
:10EEA00090E081E06C9162170CF480E0981731F1EA
:10EEB00088C0361323C07C9120818C01000F111F64
:10EEC0000B5B1A4FE8016881880F991F8D5B9A4F81
:10EED000EC018881122F72170CF4172F982F8617C8
:10EEE0000CF4962F911754F0922F27170CF4972FAC
:10EEF00068170CF4862F98170CF063C0F394A5CF15
:10EF00007C01DFEFED1AFD0A8C01000F111F0D5B74
:10EF10001A4FD8017C918C01000F111F0B5B1A4F07
:10EF2000D8012C91721729F1A081B22F72170CF41D
:10EF3000B72FAB173CF4CF5F8C2F90E08417950769
:10EF4000FCF23DC027170CF4272F2A17A4F3880FD3
:10EF5000991FDC01A35CBA4F15962C9191E0231701
:10EF60000CF090E081E062170CF480E0981719F340
:10EF700028C020812713DFCFD701AA0FBB1FA35CB6
:10EF8000BA4F15962C91880F991FDC01A35CBA4FDC
:10EF900015968C91762F36170CF4732F982F8217B5
:10EFA0000CF4922F97173CF2962F63170CF4932FC3
:10EFB00028170CF4822F98170CF4BDCF02C080E004
:10EFC00001C081E0DF91CF911F910F91FF90EF90F1
:10EFD0000895BF92CF92DF92EF92FF920F931F930B
:10EFE000CF93DF931F92CDB7DEB7A6DD882309F458
:10EFF00086C08091A6059091A705392F4091A8055C
:10F000005091A90520913D05213061F02CF421118A
:10F0100016C0CA01C3970AC0223031F0233079F4F8
:10F02000C39709C0C39607C0CA01C3969093A905A8
:10F030008093A80504C09093A7058093A60510911E
:10F04000A7050091A905311303C0051709F457C09E
:10F05000183110F40A3048F01092AB0568E270E005
:10F0600080E991E00F94E0464AC08091AA0590E0C3
:10F07000FC01EE0FFF1FE35CFA4F1583880F991F09
:10F08000FC01ED5BFA4F008380911B0690914105D6
:10F09000282F291B39F08093410581E012160CF0CE
:10F0A00080E05FDE80914005882321F081508093CD
:10F0B000400501C09BDD9ADE8111CECF80913E05D7
:10F0C00018131DC080913F05081319C06CED70E046
:10F0D00085E090E00F94E04668E171E085E090E023
:10F0E0000F94E0468091AC059091AD050196909308
:10F0F000AD058093AC0582E08093400518DE61E0A9
:10F100008DEE93E00E942C3480912104893058F4D4
:10F11000E090AC05F090AD0567E080E00E94343BE4
:10F12000C7010E94393B06E32CE749E062E08DEE1F
:10F1300093E00E947E3610E08091AA053091210470
:10F14000181708F084C0412F50E0BA01660F771FEE
:10F15000FB01E35CFA4FA581FB01E15CFA4F2581DD
:10F16000CA010396A21351C0FB01EB5BFA4F208149
:10F17000880F991FFC01E35CFA4FC080DC2CC2169B
:10F180000CF4D22E8D2D95E08902A0011124425F4E
:10F190005F4F832F90E0481759070CF456C02C1589
:10F1A0000CF4C22EEC2DF5E0EF0290011124265F45
:10F1B0003F4F8091230490E0281739070CF045C099
:10F1C0008C2D880F880F8C0DEBE0BE2EB80ECB0176
:10F1D0008E5B9A4F7C01DC14C4F12B2D0B2C000CA0
:10F1E000330BA9014D5F5F4F8091210490E04817D8
:10F1F00059073CF08091230490E0821793070CF0AC
:10F2000053C0C39495E0B90EE6CF880F991FFC0157
:10F21000E35CFA4F8081982F990F990F890F5BE07B
:10F22000E52EE80E4E2D0E2C000C550BBA016D5F2D
:10F230007F4F832F90E0681779073CF0609123049B
:10F2400070E0641775070CF03EC01F5F75CF4091EA
:10F250003F05842F880F880F480F455F642F042EC9
:10F26000000C770BFB013396832F90E0E817F9072A
:10F270003CF08091230490E0861797070CF045C07E
:10F280008091AB05811101C070DC2AD7882309F475
:10F290004AC00F90DF91CF911F910F91FF90EF9097
:10F2A000DF90CF90BF909ECCF7016081862F880FB2
:10F2B000880F680F6C5F04E024E04B2D8DEE93E027
:10F2C0000E94CE369ECFD22EA2170CF4DA2EC22E7A
:10F2D0002A170CF4CA2EFD2CFF0CFF0C8F2D8D0D60
:10F2E00030E094E0F92EF80ECD140CF4AECF6F2D73
:10F2F000630F04E024E04E2D8DEE93E039830E94ED
:10F30000CE36D39439813B5FEFCF60913E05862F97
:10F31000880F880F680F6C5F04E024E08DEE93E0A7
:10F320000E947E36ADCF0F90DF91CF911F910F914C
:10F33000FF90EF90DF90CF90BF90089569EE77E750
:10F3400081E03FDC30DDF3CC0F931F93CF93DF934D
:10F3500061E081E0B2D2D091F505C0E0D11116C0D4
:10F360008091F405811103C0BBD681119AC08091B0
:10F370002202882309F43CC081E09091F4059111A8
:10F3800080E004E024E040E150E32FC0D130B1F44C
:10F390008091F405813019F4A3D681118AC080913F
:10F3A0002202882329F181E09091F405913009F03F
:10F3B00080E003E02EE34EEF5FE217C0D230C1F4ED
:10F3C0008091F405823019F48BD681117CC0809134
:10F3D0002202882369F081E09091F405923009F0CF
:10F3E00080E003E02EE34FEE5FE26C2F0E94924438
:10F3F00034D1182FD330D1F48091F405833019F42F
:10F400006FD681116AC080912202882309F477C0E7
:10F4100081E09091F405933009F080E000E22EE362
:10F4200040EE5FE26C2F0E94924469C0811169C076
:10F43000D430B1F48091F405843019F451D681119F
:10F4400053C080912202882319F181E09091F40544
:10F45000943009F080E000E22EE342ED5FE215C057
:10F46000D530B1F48091F405853009F444C0809121
:10F470002202882369F081E09091F405953009F02B
:10F4800080E000E22EE341EC5FE26C2F0E949244A8
:10F4900086E0CF5FDF5FC53009F060CF8093F30572
:10F4A0003BC081E024D18091C105882309F45FCF5E
:10F4B00033C084E091E50E94D5488091C10588233E
:10F4C00009F46DCF29C083EC9CE70E94D548809158
:10F4D000C105882309F47BCF1FC0E2D28091C1050A
:10F4E000882309F490CF18C0DED28091C10588230B
:10F4F00009F4A7CF11C0F4D5811105C0B8CF1123ED
:10F5000039F284E0C6CF0E949BD781E028D2809157
:10F51000C105882309F4ABCFDF91CF911F910F91E3
:10F520000895E091C205E63000F581E08E0F8093EA
:10F53000C20580911B0690911C06A0E0B0E03091BE
:10F54000F5052091F30548E0E49FF0011124ED5307
:10F55000FA4F4091160650911706518340838283DB
:10F560009383A483B5833683278308950D948134D0
:10F570002F923F924F925F926F927F928F929F92C3
:10F58000AF92BF92CF92DF92EF92FF920F931F93B1
:10F59000CF93DF9300D000D0CDB7DEB71C012B8313
:10F5A0003C834D835E8369837A83BBDF83E08093F2
:10F5B00022023092C0052092BF0569817A81709342
:10F5C000BE056093BD052B813C814D815E812093FA
:10F5D000B9053093BA054093BB055093BC05E09242
:10F5E000B505F092B6050093B7051093B805D09213
:10F5F0001C06C0921B06B0921706A09216069092A7
:10F60000B4058092B3058C8D8093B20526960FB613
:10F61000F894DEBF0FBECDBFDF91CF911F910F9148
:10F62000FF90EF90DF90CF90BF90AF909F908F9022
:10F630007F906F905F904F903F902F900895FB01C7
:10F64000908181E08927808383E0809322024115A5
:10F65000510511F0FA011994089580914D0E909181
:10F660004A0E891B8F7071F49091010992FB8827D3
:10F6700080F992FD08C081E09091A916913019F0AF
:10F6800080E0089581E00895E0911606F091170654
:10F69000E817F90721F13091260637FD109226066A
:10F6A000909317068093160670931C0660931B06B2
:10F6B0004093F5052093F305805D9F4721F4109258
:10F6C00023061092C2050E94C84382E08093220262
:10F6D00081E08093C10510921E061092AE05089538
:10F6E00020E040E060E070E080ED9FE7CDCFE0916A
:10F6F000C205EE23F9F0E150E093C20598E0E99FDE
:10F70000F0011124DF01AD53BA4F17962C911797D2
:10F71000811108C016964C91169712966D917C91A6
:10F72000139703C040E060E070E0ED53FA4F808132
:10F730009181AACFD5CFCF93DF93FC01EB018091CC
:10F740001B0690911C0697FF04C010921C06109295
:10F750001B064091B5055091B6056091B7057091B3
:10F76000B80580911B0690911C06092E000CAA0B6F
:10F77000BB0B481759076A077B0724F450931C06F4
:10F7800040931B06809122028823D1F020911B0612
:10F7900030911C068091B9059091BA05A091BB05E6
:10F7A000B091BC05BC01CD01620F731F811D911D7D
:10F7B0001995BC018091BF059091C0050E942B4511
:10F7C00080911006811108C08091B205882389F1CB
:10F7D00080912202882369F18091BD059091BE0538
:10F7E000009791F020911B0630911C064091B905BD
:10F7F0005091BA056091BB057091BC05420F531F33
:10F80000611D711DFE011995E091B305F091B405DC
:10F81000309741F08091B205811103C080911006AC
:10F82000811119955DD4882321F080E0DF91CF917B
:10F830005ECFDF91CF9108950F931F93CF93DF9306
:10F8400080912202882359F06091AF057091B00534
:10F8500000E010E020E041E081E00E942F44809130
:10F86000B10581111CC081E08093B105C0911606DD
:10F87000D091170620E040E060E070E08CE19CE76A
:10F8800003DF0E9478F41092B10520E040E060E0D0
:10F8900070E0CE01DF91CF911F910F91F5CEDF91F6
:10F8A000CF911F910F910895009711F484E290E396
:10F8B0009093B0058093AF05BFCF282F1092150607
:10F8C00080911B0690911C068130904820F0109288
:10F8D0001C0610921B0680911D06882331F0809132
:10F8E0001B068093F4051092C1058091F30518164C
:10F8F000BCF4082E000C990B821B91092091F40591
:10F90000022E000C330B2817390754F097FF02C062
:10F9100080E090E08093F40590931C0680931B0692
:10F920008091F4056623C1F09091F505891714F4D0
:10F930008093F5052091F505022E000C330B2C5F0A
:10F940003F4F482F082E000C550B2417350734F471
:10F9500084508093F50508958093F50508958823D4
:10F9600061F063E972E084E690E00F94E0466AEBB0
:10F9700072E084E690E00D94E04668EB71E084E18B
:10F9800090E00D94E046CF92DF92EF92FF92CF93FA
:10F99000DF93A6D3882361F00E9463A01092230610
:10F9A00080E0DF91CF91FF90EF90DF90CF909FCEDE
:10F9B00081E080932306C0911B06D0911C062097FE
:10F9C00009F442C010921C0610921B06BE010D2EB7
:10F9D000000C880B990B0F94554D2091E70D309139
:10F9E000E80D4091E90D5091EA0D0F94F14E2091F0
:10F9F000240D3091250D4091260D5091270D0F9427
:10FA0000DA4B6B017C0120E030E040E050EC0F94D9
:10FA1000B64E87FD19C020E030E040EA50E4C7014F
:10FA2000B6010F94B34C18167CF0BE0182E00E9420
:10FA3000E7A8C092240DD092250DE092260DF092F9
:10FA4000270D82E080932202809122028823C9F050
:10FA500084E29DE00F940541BC0185E190E30E94A2
:10FA60002B456091240D7091250D8091260D90916C
:10FA7000270DDF91CF91FF90EF90DF90CF900C9406
:10FA80005646DF91CF91FF90EF90DF90CF90089591
:10FA900021E02093B1050F9486341092B1050895AA
:10FAA0000E94D5D35CCF0E942CE259CF20911B0637
:10FAB00030911C062115310559F081E0121613060C
:10FAC0000CF080E08093AE0510921C0610921B068D
:10FAD0008091AE0508954F925F926F927F928F92C0
:10FAE0009F92AF92BF92CF92DF92EF92FF920F93CD
:10FAF0001F93CF93DF931F921F92CDB7DEB75C01A8
:10FB00004A01390128018701760169837A83CEDFB2
:10FB1000D82EE6D2C82E69817A81811104C08091E5
:10FB200022028823F9F092014D2DC5010E94FA4569
:10FB3000CC20C1F0DD2011F0F40101C0F3010F90E1
:10FB40000F90DF91CF911F910F91FF90EF90DF9079
:10FB5000CF90BF90AF909F908F907F906F905F906D
:10FB60004F9019940F900F90DF91CF911F910F91AB
:10FB7000FF90EF90DF90CF90BF90AF909F908F90CD
:10FB80007F906F905F904F900895FC018081089561
:10FB9000FC01849108954F925F926F927F928F92B1
:10FBA0009F92AF92BF92CF92DF92EF92FF920F930C
:10FBB0001F93CF93DF936C017B015A012901672BBF
:10FBC00031F088248394912CC0E0D0E019C0F80172
:10FBD0001182108227C03701680C791C76946794D3
:10FBE000E3012197A201BE01C601F501199518167E
:10FBF000190654F0892BC9F04301FFEF8F1A9F0AB1
:10FC0000E814F90440F702C07E01FACFCE15DF05F3
:10FC100030F4CE0102968816990620F02196F8015C
:10FC2000D183C0838FEF9FEF05C0F801D183C083DC
:10FC300080E090E0DF91CF911F910F91FF90EF90C6
:10FC4000DF90CF90BF90AF909F908F907F906F90FC
:10FC50005F904F9008958F929F92AF92BF92CF92F4
:10FC6000DF92EF92FF920F931F93CF93DF93EC01FC
:10FC70006B017A01FB01199587FD06C0082F10E082
:10FC800020E030E0219620C1982F907E903CC1F476
:10FC9000082F0F7110E020E030E04801590186E0A4
:10FCA000880C991CAA1CBB1C8A95D1F7CE01019621
:10FCB000F60119958F7395018401082B229604C1D2
:10FCC000982F907F903E19F58F70882E912CA12C43
:10FCD000B12C16E0880C991CAA1CBB1C1A95D1F7F4
:10FCE000CE010196F60119958F73882A06E0880CDB
:10FCF000991CAA1CBB1C0A95D1F7CE010296F601ED
:10FD000019958F7395018401082B2396DDC0982FD8
:10FD1000987F903F81F58770882E912CA12CB12C73
:10FD2000F6E0880C991CAA1CBB1CFA95D1F7CE01F1
:10FD30000196F60119958F73882AA6E0880C991C04
:10FD4000AA1CBB1CAA95D1F7CE010296F601199503
:10FD50008F73882AB6E0880C991CAA1CBB1CBA9524
:10FD6000D1F7CE010396F60119958F7395018401A1
:10FD7000082B2496A9C0982F9C7F983FE9F58370A3
:10FD8000882E912CA12CB12C56E0880C991CAA1C11
:10FD9000BB1C5A95D1F7CE010196F60119958F73C8
:10FDA000882A66E0880C991CAA1CBB1C6A95D1F7AE
:10FDB000CE010296F60119958F73882A76E0880C99
:10FDC000991CAA1CBB1C7A95D1F7CE010396F601AB
:10FDD00019958F73882AE6E0880C991CAA1CBB1C15
:10FDE000EA95D1F7CE010496F60119958F73950126
:10FDF0008401082B259668C0982F9E7F9C3F09F0B0
:10FE00004AC08170882E912CA12CB12C86E0880CE0
:10FE1000991CAA1CBB1C8A95D1F7CE010196F6014C
:10FE200019958F73882A96E0880C991CAA1CBB1C14
:10FE30009A95D1F7CE010296F60119958F73882A0B
:10FE400026E0880C991CAA1CBB1C2A95D1F7CE0170
:10FE50000396F60119958F73882A36E0880C991C51
:10FE6000AA1CBB1C3A95D1F7CE010496F601199550
:10FE70008F73882A46E0880C991CAA1CBB1C4A95E3
:10FE8000D1F7CE010596F60119958F73950184017E
:10FE9000082B269619C0982F907C903849F4082F8B
:10FEA000007C003871F42196CE01F6011995F7CF48
:10FEB000082F0E7F0D3F28F02196CE01F6011995EF
:10FEC000F7CF00E010E09801E114F10429F0F70108
:10FED0000083118322833383CE01DF91CF911F9161
:10FEE0000F91FF90EF90DF90CF90BF90AF909F90D9
:10FEF0008F9008951F93CF93DF9300D01F92CDB7BB
:10FF0000DEB710E0AE014F5F5F4F65EC7DE7A3DE2B
:10FF100049815A816B817C81452B462B472B11F0FF
:10FF20001F5FF0CF812F0F900F900F900F90DF91F8
:10FF3000CF911F9108951F93CF93DF9300D01F920D
:10FF4000CDB7DEB710E0AE014F5F5F4F68EC7DE7E5
:10FF500082DE49815A816B817C81452B462B472B60
:10FF600011F01F5FF0CF812F0F900F900F900F9027
:10FF7000DF91CF911F910895FC01A081B1811C9266
:10FF8000A281B3818C918F5F8C930280F381E02DED
:10FF900080816CE0689F600D112480E00C94343BFC
:10FFA000109215068091100610921006882349F0D1
:10FFB00020E040E060E070E086EC95E665DB0C94C4
:10FFC0009743209165023091660240911B06509143
:10FFD0001C06C901840F951F2436310551F44730A2
:10FFE000510514F0069720C04A3F5F4F64F506960E
:10FFF0001BC02436310524F48536910524F504C050
:020000021000EC
:100000008436910524F41FC08A3091053CF0883E67
:1000100043E094072CF087EE93E002C08AE090E082
:100020002817390731F40DC08A30910584F78AE02A
:1000300090E0909366028093650210921C061092E5
:100040001B060C94293C84E690E0E1CFCF93DF932C
:100050001F92CDB7DEB78091B208811103C084EF43
:1000600098E02FC0211103C082EB98E02AC08DE0F8
:10007000815048F0440F411DE82FF0E0EC50F74F5D
:1000800090814927F5CF809107068417A9F0409306
:10009000070682EB98E069832DDF90E06981861B7B
:1000A000910997FF02C080E090E0809318061092BB
:1000B000190688E0809324028091190690E08E54FE
:1000C000974F0F90DF91CF9108958093150610926E
:1000D000110610921206109213061092140608953B
:1000E000809110061092100608957F928F929F9231
:1000F000AF92BF92CF92DF92EF92FF920F931F9336
:10010000CF93DF93CDB7DEB728970FB6F894DEBF55
:100110000FBECDBF7C014B016A015901FB018081FB
:100120006CE0689F600D1124F7018081982F990F72
:10013000890F880F0E94343BC114D10409F496C082
:10014000FE82ED8298868F82011103C01C2D0D2D39
:1001500074C09D2C0C2D1D2DD12C88248394AE01B0
:100160004F5F5F4FB5018C2D992D75DDC82E992EEF
:1001700089819A81AB81BC81772473940097A10512
:10018000B105C9F0712C80329105A105B10581F04E
:10019000AC01BD014D52510961097109423051054F
:1001A0006105710540F08B97A105B10589F503C084
:1001B000DD2009F455C0F70120818D2D90E0820FDC
:1001C000911D46972CF0253018F0CE010596D4DE0F
:1001D000372D3825D30EF70180818D0D8083DD20EA
:1001E00089F0DA94AE014F5F5F4FB501C80133DD8E
:1001F0008C0169817A818B819C814FEF5FEF0E9436
:100200003F3BEDCF711032C00C2D192DD12CA7CF53
:10021000D3940115110509F0A2CF0C2D192D9FCFF4
:100220004FEF5FEF0E943F3BF70120812F5F20835C
:10023000253118F0CE0105969FDEAE014F5F5F4F6E
:10024000B501812F902F07DD182F092F69817A8141
:100250008B819C81611571058105910509F706C0A7
:100260000115110589F20F5F1F4FD3CF28960FB6E6
:10027000F894DEBF0FBECDBFDF91CF911F910F91DC
:10028000FF90EF90DF90CF90BF90AF909F908F90B6
:100290007F900895AF92BF92CF92DF92EF92FF923C
:1002A0000F931F93CF93DF931F921F92CDB7DEB7AB
:1002B0005C016B017A013FDE182FE114F10419F0A3
:1002C000C70139DE01C080E01A821982C114D1044D
:1002D000C1F4412F50E090E09A01280F391F2631D8
:1002E00031057CF425E130E0241B350B281B390B4C
:1002F00037FF02C02F5F3F4F359527952A8381E056
:10030000898301E028EC3DE7A501BE016F5F7F4FC7
:10031000CE010296EADEC114D10489F08A818823D5
:1003200021F01A8289818F5F898300E025EC3DE707
:10033000A601BE016F5F7F4FCE010296D6DEE114AB
:10034000F10451F000E028EC3DE7A701BE016F5F2A
:100350007F4FCE010296C9DE0F900F90DF91CF91B3
:100360001F910F91FF90EF90DF90CF90BF90AF90D3
:100370000895CF92DF92EF92FF920F931F930E9406
:10038000F92E009103061091040620910506309184
:1003900006066B017C01C01AD10AE20AF30AF7FCD7
:1003A00013C020910206209520930206DC01CB01A8
:1003B0008A549C4FAF4FBF4F80930306909304061F
:1003C000A0930506B093060681E090910206911174
:1003D00001C080E01F910F91FF90EF90DF90CF90D0
:1003E0000895CF9393E090932202811110922506F5
:1003F0000E94F92EDC01CB018C509E4FAF4FBF4FB6
:1004000080931F0690932006A0932106B0932206A6
:1004100068E873E182E090E00F94E046C6E0C150E6
:1004200049F00F947F4662E070E080E090E00E9427
:100430002A2FF5CFCF910895AF92BF92CF92DF923E
:10044000EF920F931F93CF93DF9300D01F92CDB7FE
:10045000DEB7809123028F3F09F444C00E94F92E39
:10046000009108061091090620910A0630910B06AA
:10047000DC01CB01801B910BA20BB30BB7FD32C08B
:1004800090914A0E80914D0E8F5F8F70981751F1A9
:10049000E091230284E0E802F0011124E25BFC4FCA
:1004A00020E030E040E752E46081718182819381F5
:1004B0000F94BA4C69837A838B839C83A12CB12CD3
:1004C0006501E12C8E010F5F1F4F27E732E043E704
:1004D00052E06FE672E08BE692E00F94EA018FEF54
:1004E000809323020F900F900F900F90DF91CF9188
:1004F0001F910F91EF90DF90CF90BF90AF90089534
:100500000F931F930E94F92E00911F061091200651
:100510002091210630912206DC01CB01801B910B3A
:10052000A20BB30BB7FD0FC08091030185FB992788
:1005300090F981E089279091030196FF8260629B88
:100540008460809325068091250681709091250610
:1005500091FD82609091F605891741F18130A9F0F3
:1005600028F0823041F0833059F01EC0913089F07C
:100570009230A9F019C0992361F0933081F014C032
:10058000913069F0923081F404C0992341F09330A6
:1005900059F490911A069F5F90931A0605C09091A6
:1005A0001A06915090931A068093F6051F910F91A9
:1005B0000895CF93DF930E949743E4E0F1E08081B8
:1005C0008F7D8083C5E0D1E0888180958072A3E033
:1005D000B1E08C9380818F7B80838881809580744B
:1005E0008C936A98729A54985C9A82E0809324065D
:1005F00087DF10921A06DF91CF910895CF93C091B3
:100600006B0687E296E076DCC81790F480916B0663
:100610008F5F21E0280FE82FF0E0E95DF94F90812E
:10062000907C903811F4822FF4CF80936B0602C037
:1006300010926B06CF9108950F931F93CF93DF9382
:100640008C01C0916B06D0E0C95DD94FCE0152DC60
:10065000F8018083CE01DF91CF911F910F91089512
:1006600081E090912706911101C080E00895CF9319
:10067000DF9320916A06211120C0FC010190002027
:10068000E9F73197EF01C81BD90BC334D10534F01A
:1006900031972081207C2038D9F3F4CFBC01DD27AD
:1006A000AE0187E296E00F945A55C95DD94F188282
:1006B00010926B0683E080932202DF91CF91089520
:1006C000CF93DF93CDB7DEB78E8190916A068917FD
:1006D00090F080936A069E01275F3F4F4F815885B7
:1006E00062E470E087E296E00F94A35510926B06E7
:1006F00083E080932202DF91CF9108950F931F939F
:10070000CF93DF938C0167FF03C010926A0660E00D
:1007100080916A0690E0262F062E000C330B2817D6
:1007200039071CF160936A06C8010F94BC54F801A4
:10073000E80FF91FEF01C01BD10BC334D10534F012
:1007400031978491807C8038D9F3F4CFDD27AE01D6
:10075000B80187E296E00F94DD54C95DD94F188245
:1007600010926B0683E080932202DF91CF911F915C
:100770000F9108954F925F926F927F928F929F9206
:10078000AF92BF92CF92DF92EF92FF920F931F939F
:10079000CF930E94F92E6B017C014EDEB1DE809179
:1007A000250682FF15C080910106811113C091E0DA
:1007B000909301062091B416211103C08091B105D8
:1007C0008927809310061092B41681E00ADE02C0D9
:1007D00010920106C9B1C295C17081E0C82780910D
:1007E0002406C81779F10E944543882359F11091D6
:1007F0002406C0932406CC2309F4CAC164EF71E037
:1008000080E090E00E94EDA00E941C90123009F060
:10081000BAC10E94F3900E94974383E08093220222
:100820000E94F92E6B017C01DC01CB018C599F4F9A
:10083000AF4FBF4F8093FD059093FE05A093FF053A
:10084000B09300068091FD059091FE05A091FF05F3
:10085000B0910006A7019601281B390B4A0B5B0BD0
:1008600057FF05C080911E06882309F41FC2D701D7
:10087000C6018C599F4FAF4FBF4F8093FD0590939A
:10088000FE05A093FF05B093000660911A06062EA0
:10089000000C770B77FF03C0719561957109062EE7
:1008A000000C770B880B990B0F94554D2B013C01D5
:1008B00020E030E040E050E40F94B64E87FF05C0E2
:1008C0008091100681117DC08DC08091150688230E
:1008D00009F456C08090110690901206A09013065D
:1008E000B090140681149104A104B104E1F120E058
:1008F00030E040E05FE3C301B2010F94F14E2B0101
:100900003C01C701B601681979098A099B090F944E
:10091000534D9B01AC01C301B2010F94BA4C20E0CE
:1009200030E04AE754E40F94F14E4B015C0120E0C3
:1009300030E040EA52E40F94B64E87FF0FC020E04B
:1009400030E040EF51E4C501B4010F94B64E87FD8D
:100950000AC02AE030E040E050E009C024E630E080
:1009600040E050E004C021E030E040E050E0C092C0
:100970001106D0921206E0921306F092140604C0FB
:1009800021E030E040E050E0A0911A0600911B0603
:1009900010911C060A2E000CBB0B0F945C5022E039
:1009A00030E040E050E00F941F50DA01C901800FA1
:1009B000911FA11DB11D90931C0680931B061092E0
:1009C0001A06D701C6018856954CAF4FBF4F80938A
:1009D000F9059093FA05A093FB05B093FC0581E01F
:1009E0008093220220911606309117064FE7203D92
:1009F000340741F480912402882309F4D4C0815043
:100A0000809324022152314651F58091240288239B
:100A100021F081508093240222C084E0809324023C
:100A2000809119068F5F8093190690911806981788
:100A300028F4109219068CE08093240281E08093C0
:100A40002202D701C6018856954CAF4FBF4F809305
:100A5000F9059093FA05A093FB05B093FC058091EE
:100A60006F0081FB222720F981FF05C080916F0074
:100A70008D7F80936F0080915C0D90915D0DA091B2
:100A80005E0DB0915F0D222329F020916F0022604E
:100A900020936F003AE0B695A795979587953A957C
:100AA000D1F7009721E0A207B10520F08FEF9FEF6B
:100AB000A0E0B0E09695879520912202211105C013
:100AC00030911E063111EEC051C0009741F04091A7
:100AD000F7055091F8054817590708F047C080916D
:100AE0001E06811117C0223008F06DC080912604C7
:100AF000811107C081E0809326048DEE93E00E946F
:100B0000CC338DEE93E00E94033481E080931D0688
:100B100080931E0683E00E942A4361E08DEE93E0FD
:100B20000E942C34E0911606F09117061995109248
:100B30001D0680911E06811152C0109210060E945F
:100B4000F92EDC01CB018C199D09AE09BF0900917A
:100B5000F7051091F80520E030E0081719072A077B
:100B60003B0720F49093F8058093F70580911606D3
:100B700090911706805D9F4709F457C08091230626
:100B8000811153C07EC060E08FE990E3B7DD43CEB2
:100B9000ECD5123009F43FCE60E081E990E3AEDDA0
:100BA0000E94707B38CE8CE0809324028091F70500
:100BB0009091F80501979093F8058093F70581E0EF
:100BC000809322021FCF243030F0243009F08ECFE2
:100BD000109222028BCF81E08093220287CF8DEE8C
:100BE00093E00E94073491E0811101C090E090935E
:100BF0001E06992309F4A1CF0E94F92EDC01CB0136
:100C00008C199D09AE09BF09C090F705D090F80571
:100C1000E12CF12CC816D906EA06FB0608F046C0FE
:100C20009093F8058093F70541C048E9C40E4AE364
:100C3000D41EE11CF11CC092F905D092FA05E09295
:100C4000FB05F092FC0580911E0681112FC080915A
:100C50002202813099F0833049F5CF911F910F9195
:100C6000FF90EF90DF90CF90BF90AF909F908F90CC
:100C70007F906F905F904F900C94C8431092220227
:100C800015C08091F9059091FA05A091FB05B091EE
:100C9000FC05C81AD90AEA0AFB0AF7FCD4CF0E945D
:100CA000707BD1CF009709F435CF11CFCF911F9131
:100CB0000F91FF90EF90DF90CF90BF90AF909F90FB
:100CC0008F907F906F905F904F90089561E016DD58
:100CD0000C94707BCF93DF931F921F92CDB7DEB73A
:100CE00089839A8366DC89819A81F0DF0F900F9067
:100CF000DF91CF910C949C438091010982FD05C046
:100D00008091A916823061F410C08091B2088111DF
:100D100003C084EF98E002C082EB98E061E0A7CCCA
:100D2000813031F083E690E305C084E890E302C0AF
:100D300088E790E36FEFE2CC1092B4161092920223
:100D4000809101098064809301090E9444B00F944E
:100D50001F4760E085E590E3D1DC0C94707B89E46B
:100D600090E30E94547C60E08CE390E3C7DC40E0B9
:100D700061E080E00E94566582E390E30D94813447
:100D8000BBDF1092B416109292020E94B8658823BD
:100D900021F08091010982FF04C00E943CB00D94B3
:100DA00098478EE290E30F948134F7CF8091010948
:100DB00082FF2AC00E94B865882319F18091BC0681
:100DC0009091BD06A091BE06B091BF060097A10507
:100DD000B105B9F0BC01CD016D597F4F8F4F9F4FC9
:100DE00024E630E040E050E00F94FD4F6091B806FB
:100DF0007091B9068091BA069091BB060F94FD4F91
:100E000001C020E020932606809126068F77089562
:100E100080ED9FE79093170680931606089561E092
:100E2000FC0180810E9429318FEF0C94DFA1CF93C8
:100E3000DF93EC018A810E94A1A160E08881DF91AB
:100E4000CF910C9429318F929F92AF92BF92EF92E3
:100E5000FF920F931F93CF93DF93EC018B017A01E5
:100E60000E94F92E4B015C012CE2820E21E0921EC1
:100E7000A11CB11C0E94B9A18B838F3F61F40E9419
:100E8000F92EDC01CB0188199909AA09BB09B7FD24
:100E9000F1CF81E10DC08E3F51F4B701C8010E942E
:100EA000C0A10E94B9A10E94B9A111E003C08FE0C6
:100EB000898310E0CE01B3DF812FDF91CF911F91A5
:100EC0000F91FF90EF90BF90AF909F908F900895FB
:100ED000CF92DF92EF92FF926A017B010E94F92E7E
:100EE000C60ED71EE81EF91E0E94B9A18F3F61F001
:100EF0000E94F92EDC01CB018C199D09AE09BF09B6
:100F0000B7FDF2CF80E001C081E0FF90EF90DF906D
:100F1000CF900895EF92FF921F93CF93DF9300D06D
:100F20001F92CDB7DEB77C01162F29833A834B83FE
:100F30005C837DDF48E552E060E070E0C701C8DF18
:100F4000812F80640E94DFA18C810E94DFA18B81B0
:100F50000E94DFA18A810E94DFA189810E94DFA116
:100F6000112311F087E801C085E90E94DFA11C3040
:100F700011F40E94B9A110E00E94B9A1F701838386
:100F800087FF04C01F3F11F01F5FF6CF0F900F9037
:100F90000F900F90DF91CF911F91FF90EF900895E8
:100FA0008F929F92AF92BF92CF92DF92EF92FF9279
:100FB0000F931F93CF93DF93EC01162F1C8219829E
:100FC00048830E94F92E6B017C0120EDC20E27E0C0
:100FD000D21EE11CF11CA89561E088810E94293194
:100FE00061E088810E94ED300E94B2A185E08A8391
:100FF0000E94A1A10AE08FEF0E94DFA10150D9F762
:10100000A89520E030E0A90160E0CE0183DF8B836A
:10101000813061F00E94F92EDC01CB018C199D0911
:10102000AE09BF09B7FDEDCF81E055C0A8952AEA0A
:1010300031E040E050E068E0CE016CDF853011F433
:1010400081E009C004E00E94B9A18B830150D9F767
:101050008A3A51F482E08C83A8958C81823081F0A9
:10106000812C912C540111C00E94F92EDC01CB017E
:101070008C199D09AE09BF09B7FDD9CF82E02BC0FD
:10108000812C912CA12C80E4B82E20E030E0A90125
:1010900067E3CE013FDFA501940169E2CE013ADFAB
:1010A0008B83882361F00E94F92EDC01CB018C191F
:1010B0009D09AE09BF09B7FDE8CF8AE00CC08C815D
:1010C0008230D1F420E030E0A9016AE3CE0122DFD2
:1010D000882329F088E08983CE01A1DE16C00E9412
:1010E000B9A1807C803C11F483E08C830E94B9A17B
:1010F0000E94B9A10E94B9A1CE0191DE173018F467
:101100001A8381E003C088E1898380E0DF91CF9179
:101110001F910F91FF90EF90DF90CF90BF90AF9015
:101120009F908F9008950F931F93CF93DF93EC01BF
:1011300089018C81833039F089E0440F551F661F87
:10114000771F8A95D1F79A01AB0161E1CE01E2DE0A
:10115000811109C040E052E0B801CE01DF91CF918A
:101160001F910F9170CE84E08983CE0158DE80E01C
:10117000DF91CF911F910F910895CF93DF93EC01F1
:10118000862FBA010E94E4A18FEF0E94DFA18FEFAA
:101190000E94DFA10E94B9A18B83982F9F71953087
:1011A00031F083E18983CE013ADE80E001C081E045
:1011B000DF91CF9108950F931F93CF93DF93EC01AD
:1011C00089018C81833039F089E0440F551F661FF7
:1011D000771F8A95D1F79A01AB0168E1CE019ADEBB
:1011E00081111EC0A8016EEFCE01C7DF8823E1F098
:1011F00048E552E060E070E0CE016ADE882371F0DD
:1012000020E030E0A9016DE0CE0184DE81110AC04A
:101210000E94B9A1811106C011E007C087E103C097
:1012200086E001C086E1898310E0CE01F8DD812FE0
:10123000DF91CF911F910F910895CF93DF931F926C
:10124000CDB7DEB72091B6163091B716CE01019614
:101250002115310519F0821B930B02C08C5B96415E
:101260000F90DF91CF910895FC01238121110C94FF
:101270005D9A08958CE696E0F7CF87E896E0F4CF84
:101280008091A206811107C00E942CE2882319F0E8
:1012900081E08093A206089580910109847F8B7F6D
:1012A000809301091092B8061092B9061092BA06FE
:1012B0001092BB061092BC061092BD061092BE069C
:1012C0001092BF0610922D0710926C078EE091E0ED
:1012D000EDE6F7E0DF019C011D9221503040E1F77F
:1012E0008FEF8093B1080895FC0120E03EE2DB011E
:1012F0004C91403241F0283011F430833196DB01BB
:101300004C91408331962F5F6F5F7F4F2B3079F781
:10131000108208952F923F924F925F926F927F9228
:101320008F929F92AF92BF92CF92DF92EF92FF92F5
:101330000F931F93CF93DF93CDB7DEB7C356D10979
:101340000FB6F894DEBF0FBECDBF8C015B014A0122
:101350004DB65EB6312C7E0187E5E80EF11C9BE1AF
:10136000292E42EB58E0BE016F5F7F4FC5010E94FE
:10137000CD9818160CF005C18C85282F28712031C6
:1013800009F074C09091B7069150923008F46EC085
:101390006DB67EB6BE016F5F7F4FC701A5DF011539
:1013A000110521F0F8018081811173C021E081E0F5
:1013B00090E0F70101900020E9F73197EE19FF095D
:1013C000E80FF91F32968DB79EB78E1B9F0B0FB695
:1013D000F8949EBF0FBE8DBFEDB7FEB731966F017B
:1013E000211102C0B80102C06EE573E0C6010F947E
:1013F0004555B701C6010F942F556EE573E0C60140
:101400000F942F551CAE1FAE21E0A701B501CE01F0
:10141000CC960E94599C81110DC08091B706811114
:1014200009C00E941FA181EA92E30E9411A1C70195
:101430000E9417A7FE01FC96DE019196822D019075
:101440000D928A95E1F740E050E0BE016F5D7F4F5D
:10145000C60160DFCE01819607DFCE01CC9604DFA6
:101460000FB6F8947EBE0FBE6DBE7BCF99819923D7
:1014700009F487C0953E09F474CF9E3209F471CF08
:101480009091B2089E3209F46CCF8A7009F069CF4E
:101490000AC0F80101900020E9F73197CF01801BC5
:1014A000910B20E086CF81E0203109F080E090911F
:1014B000010980FB94F990930109811108C0898585
:1014C000873409F04ECF8A858E3709F44ACF809150
:1014D000B706813021F068F08230B9F142CF8091B7
:1014E000B5069091B60601969093B6068093B50620
:1014F00038CFBE016F5F7F4F84EF98E0F5DE0115B6
:10150000110511F0680105C084EFC82E88E0D82EBF
:1015100008C0F60181916F018823B1F30E94C0A633
:10152000F8CFF60181916F01882319F00E94C0A6BF
:10153000F8CF80E20E94C0A66D8D7E8D8F8D98A120
:101540004AE050E00E94CDA70CCFBE016F5F7F4FF5
:1015500084EF98E0C9DE8114910441F064EF78E0F3
:10156000C4010F941C55892B51F40BC0832D90E0BE
:101570002091B3063091B4068217930711F033948B
:10158000F0CE0FB6F8945EBE0FBE4DBECD59DF4F04
:101590000FB6F894DEBF0FBECDBFDF91CF911F9184
:1015A0000F91FF90EF90DF90CF90BF90AF909F9002
:1015B0008F907F906F905F904F903F902F90089505
:1015C000CF93DF93CDB7DEB76B970FB6F894DEBF3E
:1015D0000FBECDBF1092B70640E050E0BA0186E9D9
:1015E00098E00E947C998BE1E6E9F8E0DE01119633
:1015F00001900D928A95E1F740E050E0BE016F5FE7
:101600007F4F80E090E086DECE0101962DDE6B9666
:101610000FB6F894DEBF0FBECDBFDF91CF91089516
:101620000F931F93CF93DF93CDB7DEB72D970FB6F0
:10163000F894DEBF0FBECDBF80913107882391F0B3
:10164000BE016F5F7F4F8EE297E00E94EF968E01A2
:101650000F5F1F4FF80181918F01882339F00E949D
:10166000C0A6F8CF87E992E30E9411A18AE00E9408
:10167000C0A62D960FB6F894DEBF0FBECDBFDF918A
:10168000CF911F910F910895CF92DF92EF92FF9229
:101690000F931F93CF93DF93CDB7DEB7EDB6FEB6B2
:1016A000DC010D900020E9F79D01281B390B2C5F10
:1016B0003F4F4DB75EB7421B530B0FB6F8945EBF5A
:1016C0000FBE4DBF0DB71EB70F5F1F4F9F938F9378
:1016D00081E592E39F938F931F930F930F9474551B
:1016E000680154E0C50ED11C0F900F900F900F9021
:1016F0000F900F90F6018081882349F0082E000C8E
:10170000990B0F94A054F60181936F01F3CFC80198
:101710000F9486348DE492E30F9494340FB6F894CA
:10172000FEBE0FBEEDBEDF91CF911F910F91FF90D6
:10173000EF90DF90CF9008958091010983FF03C05F
:1017400084608093010908951092CE0B8091010965
:101750008F7B8B7F809301090E94B865882321F0DD
:101760008EE297E00C945D9A0895EEDF8091010976
:10177000877F8093010908950F931F93CF93DF9381
:101780008B01EA01DB016D917C910E94EF96D801FB
:10179000ED91FC919081888191110EC08936B0F451
:1017A0008FE28083F801808191810196918380830B
:1017B00088818F5F88830AC0893680F73196D80187
:1017C000ED93FC9388818F5F8883E1CFDF91CF9188
:1017D0001F910F9108950F931F93CF93DF9300D024
:1017E000CDB7DEB79C012F5F3F4F3B832A832FE2AB
:1017F000FC01208381E0898310E00BE180916C077C
:10180000181770F4019FC0011124AE014F5F5F4FA4
:10181000BE016E5F7F4F8359984FAEDF1F5FEECFE3
:1018200089818B3570F4AE014F5F5F4FBE016E5FF3
:101830007F4F8EE297E0A0DF8A819B8101979B8397
:101840008A83EA81FB8110820F900F900F90DF91C5
:10185000CF911F910F9108958091010982FF1FC0C0
:1018600085E191E30E9411A16091B8067091B906DB
:101870008091BA069091BB064AE050E00E94C2A750
:101880008FE20E94C0A66091BC067091BD06809157
:10189000BE069091BF064AE050E00C94CDA784E0CC
:1018A00091E30C9411A1EF92FF920F931F93CF93AA
:1018B000DF938C01FC0101900020E9F73197EF01E3
:1018C000C81BD90B10922E076EE470E00F943A55A6
:1018D0007C01009729F4FE013197E00FF11F0EC043
:1018E00060E270E00F943A558C010F5F1F4F6AE27F
:1018F00070E0C7010F943A55FC0131978DE0818368
:101900008AE082831382B8018EE297E00E94EC9E07
:1019100080912E07882361F00E9422A18DEE90E332
:10192000DF91CF911F910F91FF90EF900C9411A137
:10193000DF91CF911F910F91FF90EF9008958EE26C
:1019400097E00E94129A8EE297E00E945D9A809141
:1019500001098D7F8E7F809301091092B806109245
:10196000B9061092BA061092BB0681E08093BF0BB5
:1019700008950F931F93CF93DF93CDB7DEB76B9787
:101980000FB6F894DEBF0FBECDBF8B0122E02093CF
:10199000B7069093B4068093B30640E050E0BA01D6
:1019A0008BE798E00E947C998BE1EBE7F8E0DE01A1
:1019B000119601900D928A95E1F7A801BE016F5F23
:1019C0007F4F80E090E0A6DCCE0101964DDC6B9667
:1019D0000FB6F894DEBF0FBECDBFDF91CF911F9140
:1019E0000F910895CF93DF93CDB7DEB76B970FB606
:1019F000F894DEBF0FBECDBF81E08093B706109292
:101A0000B6061092B50640E050E0BA018BE798E0C8
:101A10000E947C998BE1EBE7F8E0DE0111960190E2
:101A20000D928A95E1F740E050E0BE016F5F7F4F75
:101A300080E090E06FDCCE01019616DC8091B50667
:101A40009091B6066B960FB6F894DEBF0FBECDBF71
:101A5000DF91CF9108952F923F924F925F926F92B4
:101A60007F928F929F92AF92BF92CF92DF92EF922E
:101A7000FF920F931F93CF93DF9300D01F92CDB7A8
:101A8000DEB77C018B01342E2DB73EB73C832B8310
:101A90008091AB0681110BC01092870610928A06C6
:101AA00081E08093AB068DE399E80E94223B809110
:101AB000A30681110BC010926C0610926F0681E094
:101AC0008093A3068AE399E80E94223BF801808173
:101AD0008F3251F486E998E0F70191838083109268
:101AE0006C070F5F1F4F05C08BE798E0F7019183EC
:101AF0008083F7010190F081E02DFA83E98327E8E4
:101B0000A22E26E0B22E3BE1232E0115110509F489
:101B10007FC04DB65EB66FE270E0C8010F943A55D3
:101B20003C010817190708F073C06C01C01AD10AEC
:101B3000DD24C60101962DB73EB7281B390B0FB621
:101B4000F8943EBF0FBE2DBF8DB79EB701964C01D6
:101B5000A601B8010F945A55F401EC0DFD1D108239
:101B6000332019F0C4010E9417A7F7016081718129
:101B700021E0A401C5010E94599C811111C0B4014A
:101B800080ED90E30E9425A18DEC90E30E9411A1CD
:101B90000FB6F8945EBE0FBE4DBE80E090E039C037
:101BA000F7018081918129813A818217930711F091
:101BB0000E945D9AF701B182A082A0916C07AA30C1
:101BC00078F481E08A0F80936C072A9ED00111245B
:101BD000A359B84FF501822D01900D928A95E1F736
:101BE000F701808191818758964029F49CE6A92EBF
:101BF00096E0B92E04C087E8A82E86E0B82E8301AF
:101C00000F5F1F4F0FB6F8945EBE0FBE4DBE7DCF67
